 aamG

 Timestamp is 540049c4 (Fri Aug 29 17:37:08 2014)

 Preferred load address is 00010000

 Start         Length     Name                   Class
 0001:00000000 000252b0H .text                   CODE
 0001:000252b0 000015a0H .text$yc                CODE
 0001:00026850 000000ccH .text$yd                CODE
 0002:00000000 00011b1cH .rdata                  DATA
 0002:00011b1c 0000016cH .rdata$r                DATA
 0002:00011c88 00000134H .xdata                  DATA
 0002:00011dbc 0000011cH .xdata$x                DATA
 0002:00011ed8 00000000H ATL$__a                 DATA
 0002:00011ed8 00000000H ATL$__z                 DATA
 0002:00011ed8 00000078H .idata$2                DATA
 0002:00011f50 00000014H .idata$3                DATA
 0002:00011f64 000002d0H .idata$4                DATA
 0002:00012234 000003c4H .idata$6                DATA
 0002:000125f8 00000000H .edata                  DATA
 0003:00000000 000002d0H .idata$5                DATA
 0003:000002d0 00000004H .CRT$XCA                DATA
 0003:000002d4 00000004H .CRT$XCAA               DATA
 0003:000002d8 00000010H .CRT$XCC                DATA
 0003:000002e8 0000005cH .CRT$XCL                DATA
 0003:00000344 00000160H .CRT$XCU                DATA
 0003:000004a4 00000004H .CRT$XCZ                DATA
 0003:000004a8 00000004H .CRT$XIA                DATA
 0003:000004ac 00000004H .CRT$XIZ                DATA
 0003:000004b0 00000004H .CRT$XPA                DATA
 0003:000004b4 00000004H .CRT$XPZ                DATA
 0003:000004b8 00000004H .CRT$XTA                DATA
 0003:000004bc 00000004H .CRT$XTZ                DATA
 0003:000004c0 000002a0H .data                   DATA
 0003:00000760 000016d0H .bss                    DATA
 0004:00000000 00001bd0H .pdata                  DATA
 0005:00000000 00000058H .rsrc$01                DATA
 0005:00000060 000003a0H .rsrc$02                DATA

  Address         Publics by Value              Rva+Base       Lib:Object

 0000:00000000       ___safe_se_handler_table   00000000     <absolute>
 0000:00000000       ___safe_se_handler_count   00000000     <absolute>
 0001:00000000       ?GetApp@@YAPAVCAAMApp@@XZ  00011000 f   aam.obj
 0001:0000001c       ?GetMainWnd@@YAPAVCMainFrame@@XZ 0001101c f   aam.obj
 0001:00000038       ?GetInstanceHandle@@YAPAUHINSTANCE__@@XZ 00011038 f   aam.obj
 0001:00000060       ?WaitForCalibrationDone@@YAXXZ 00011060 f   aam.obj
 0001:000000d0       WinMain                    000110d0 f   aam.obj
 0001:00000174       ??0CAAMApp@@QAA@XZ         00011174 f   aam.obj
 0001:000001e8       ?InitInstance@CAAMApp@@UAAHXZ 000111e8 f   aam.obj
 0001:0000051c       ?ExitInstance@CAAMApp@@UAAHXZ 0001151c f   aam.obj
 0001:00000578       ?ReadConnProfileName@CAAMApp@@QAAXXZ 00011578 f   aam.obj
 0001:000006a0       ?ReadModemName@CAAMApp@@QAAXXZ 000116a0 f   aam.obj
 0001:000007c0       ?ReadTimeSetting@CAAMApp@@QAAXXZ 000117c0 f   aam.obj
 0001:00000944       ?GetCarrier@CAAMApp@@QAAXXZ 00011944 f   aam.obj
 0001:00000984       ?SetDefaultProfile@CAAMApp@@QAAXXZ 00011984 f   aam.obj
 0001:000009c8       ?IsDynamicCarrierIndexSet@CAAMApp@@QAAHXZ 000119c8 f   aam.obj
 0001:00000a50       ?LoadResourceLibrary@CAAMApp@@QAAHXZ 00011a50 f   aam.obj
 0001:00000bcc       ?GetWindowHandle@CMainFrame@@QAAPAUHWND__@@XZ 00011bcc f i aam.obj
 0001:00000bf8       ?SetResourceHandle@CAAMApp@@QAAXPAUHINSTANCE__@@@Z 00011bf8 f i aam.obj
 0001:00000c20       ??1CAAMApp@@QAA@XZ         00011c20 f i aam.obj
 0001:00000c74       ??0CArbitrator@@QAA@XZ     00011c74 f   arbitrator.obj
 0001:00000ed4       ?StartThread@CArbitrator@@QAAXXZ 00011ed4 f   arbitrator.obj
 0001:00000f70       ?CloseThread@CArbitrator@@QAAXXZ 00011f70 f   arbitrator.obj
 0001:00000f98       ?RebootDevice@CArbitrator@@QAAXXZ 00011f98 f   arbitrator.obj
 0001:00001138       ?IsSpiderRunning@CArbitrator@@QAAHXZ 00012138 f   arbitrator.obj
 0001:0000126c       ?CheckProc@CArbitrator@@SAXPAX@Z 0001226c f   arbitrator.obj
 0001:000012b0       ?CheckProcRun@CArbitrator@@UAAXXZ 000122b0 f   arbitrator.obj
 0001:00001a5c       ??1CArbitrator@@UAA@XZ     00012a5c f   arbitrator.obj
 0001:00001b88       ?AppStartCheck@CArbitrator@@QAAKH@Z 00012b88 f   arbitrator.obj
 0001:00001bf8       ?CreateSession@CArbitrator@@QAAKH@Z 00012bf8 f   arbitrator.obj
 0001:00001c7c       ?DeleteSession@CArbitrator@@QAAXH@Z 00012c7c f   arbitrator.obj
 0001:00001ca0       ?ExitSession@CArbitrator@@QAAXXZ 00012ca0 f   arbitrator.obj
 0001:00001cb0       ?SetUpdaterInProgress@CArbitrator@@QAAX_N@Z 00012cb0 f   arbitrator.obj
 0001:00001ce8       ?GetUpdaterInProgress@CArbitrator@@QAA_NXZ 00012ce8 f   arbitrator.obj
 0001:00001d7c       ?SetProvisioningInProgress@CArbitrator@@QAAX_N@Z 00012d7c f   arbitrator.obj
 0001:00001db4       ?SetMDNchanged@CArbitrator@@QAAX_N@Z 00012db4 f   arbitrator.obj
 0001:00001dec       ?SetActivationInProgress@CArbitrator@@QAAX_N@Z 00012dec f   arbitrator.obj
 0001:00001e24       ?GetActivationStatus@CArbitrator@@QAA_NXZ 00012e24 f   arbitrator.obj
 0001:00001e70       ?GetMDNchanged@CArbitrator@@QAA_NXZ 00012e70 f   arbitrator.obj
 0001:00001ebc       ?GetProvisioningStatus@CArbitrator@@QAA_NXZ 00012ebc f   arbitrator.obj
 0001:00001f08       ?SetCheckPDP@CArbitrator@@QAAX_N@Z 00012f08 f   arbitrator.obj
 0001:00001f40       ?GetCheckPDP@CArbitrator@@QAA_NXZ 00012f40 f   arbitrator.obj
 0001:00001f8c       ?ResetState@CArbitrator@@QAAXXZ 00012f8c f   arbitrator.obj
 0001:00001f9c       ?LaunchIOTA@CArbitrator@@QAAXK@Z 00012f9c f   arbitrator.obj
 0001:00002358       ?IsRunning@CArbitrator@@QAAHPAG@Z 00013358 f   arbitrator.obj
 0001:0000253c       ??_ECArbitrator@@UAAPAXI@Z 0001353c f i arbitrator.obj
 0001:0000253c       ??_GCArbitrator@@UAAPAXI@Z 0001353c f i arbitrator.obj
 0001:0000257c       SetEvent                   0001357c f i arbitrator.obj
 0001:000025b0       ?GetResourceHandle@CAAMApp@@QAAPAUHINSTANCE__@@XZ 000135b0 f i arbitrator.obj
 0001:000025dc       ?wcsrchr@@YAPAGPAGG@Z      000135dc f i arbitrator.obj
 0001:00002610       ??0CIota24Dlg@@QAA@XZ      00013610 f   iota24dlg.obj
 0001:00002654       ??1CIota24Dlg@@UAA@XZ      00013654 f   iota24dlg.obj
 0001:00002674       ?Create@CIota24Dlg@@QAAHPAUHWND__@@@Z 00013674 f   iota24dlg.obj
 0001:000027cc       ?CIota24DlgProc@CIota24Dlg@@SAHPAUHWND__@@IIJ@Z 000137cc f   iota24dlg.obj
 0001:00002ad0       ?SetMessageText@CIota24Dlg@@QAAXIK@Z 00013ad0 f   iota24dlg.obj
 0001:00002b6c       ?ShowWindow@CIota24Dlg@@QAAXH@Z 00013b6c f   iota24dlg.obj
 0001:00002ba4       ?SetForegroundWindow@CIota24Dlg@@QAAHXZ 00013ba4 f   iota24dlg.obj
 0001:00002c00       ?Initialize@CIota24Dlg@@QAAXXZ 00013c00 f   iota24dlg.obj
 0001:00002d3c       ??_ECIota24Dlg@@UAAPAXI@Z  00013d3c f i iota24dlg.obj
 0001:00002d3c       ??_GCIota24Dlg@@UAAPAXI@Z  00013d3c f i iota24dlg.obj
 0001:00002d84       ??0CMainFrame@@QAA@XZ      00013d84 f   mainfrm.obj
 0001:00003274       ??1CMainFrame@@UAA@XZ      00014274 f   mainfrm.obj
 0001:000035e8       ?OnUSSDNotification@CMainFrame@@QAAJIJ@Z 000145e8 f   mainfrm.obj
 0001:000036d4       ?OnMIPFailEvent@CMainFrame@@QAAJIJ@Z 000146d4 f   mainfrm.obj
 0001:000042ac       ?WindowProc@CMainFrame@@UAAJIIJ@Z 000152ac f   mainfrm.obj
 0001:000054d0       ?InsertWPSBubble@CMainFrame@@QAAXXZ 000164d0 f   mainfrm.obj
 0001:00005750       ?RemoveWPSBubble@CMainFrame@@QAAXXZ 00016750 f   mainfrm.obj
 0001:0000586c       ?ExitEmergencyMode@CMainFrame@@QAAXXZ 0001686c f   mainfrm.obj
 0001:00005884       ?RemoveEmergencyICon@CMainFrame@@QAAXXZ 00016884 f   mainfrm.obj
 0001:000058f4       ?RemovePhoneBubbleICon@CMainFrame@@QAAXXZ 000168f4 f   mainfrm.obj
 0001:00005960       ?UpdateEmergencyICon@CMainFrame@@QAAXH@Z 00016960 f   mainfrm.obj
 0001:00005bdc       ?InsertEmergencyICon@CMainFrame@@QAAXXZ 00016bdc f   mainfrm.obj
 0001:00005ddc       ?OnAllCallStatusEvent@CMainFrame@@QAAJIJ@Z 00016ddc f   mainfrm.obj
 0001:00006cd4       ?OnEmergencyHangUp@CMainFrame@@QAAJIJ@Z 00017cd4 f   mainfrm.obj
 0001:00006e10       ?OnSubscriberNumber@CMainFrame@@QAAJIJ@Z 00017e10 f   mainfrm.obj
 0001:0000749c       ?OnDataCallStatusEvent@CMainFrame@@QAAJIJ@Z 0001849c f   mainfrm.obj
 0001:00007744       ?CheckForDataCall@CMainFrame@@QAA_NXZ 00018744 f   mainfrm.obj
 0001:0000791c       ?OnResultGetMinActiveState@CMainFrame@@QAAJIJ@Z 0001891c f   mainfrm.obj
 0001:00007df8       ?OnResultCallbackError@CMainFrame@@QAAJIJ@Z 00018df8 f   mainfrm.obj
 0001:00007ff0       ?On1XPdpInactFailEvent@CMainFrame@@QAAJIJ@Z 00018ff0 f   mainfrm.obj
 0001:00008328       ?OnMINActiveStateChanged@CMainFrame@@QAAJIJ@Z 00019328 f   mainfrm.obj
 0001:0000835c       ?OnResultGetSystemTime@CMainFrame@@QAAJIJ@Z 0001935c f   mainfrm.obj
 0001:00008440       ?OnPwrStateUpdate@CMainFrame@@QAAJIJ@Z 00019440 f   mainfrm.obj
 0001:00008538       ?OnCarrierChanged@CMainFrame@@QAAJIJ@Z 00019538 f   mainfrm.obj
 0001:00008590       ?OnSrvStateUpdate@CMainFrame@@QAAJIJ@Z 00019590 f   mainfrm.obj
 0001:000086d4       ?OnSIPNAIPWD@CMainFrame@@QAAJIJ@Z 000196d4 f   mainfrm.obj
 0001:000088bc       ?PopulateRegistrywithSIPNAIPWD@CMainFrame@@QAAJXZ 000198bc f   mainfrm.obj
 0001:00008c60       ?OnResultGetPDPForAnIndex@CMainFrame@@QAAJIJ@Z 00019c60 f   mainfrm.obj
 0001:00008c84       ?WndProc@@YAJPAUHWND__@@IIJ@Z 00019c84 f   mainfrm.obj
 0001:00008ce4       ?MyRegisterClass@@YAGPAUHINSTANCE__@@PAG@Z 00019ce4 f   mainfrm.obj
 0001:00008dac       ?Create@CMainFrame@@QAAHXZ 00019dac f   mainfrm.obj
 0001:00008edc       ??_ECMainFrame@@UAAPAXI@Z  00019edc f i mainfrm.obj
 0001:00008edc       ??_GCMainFrame@@UAAPAXI@Z  00019edc f i mainfrm.obj
 0001:00008f1c       ??0CMipErrorDlg@@QAA@K@Z   00019f1c f   miperrdlg.obj
 0001:00008f70       ??1CMipErrorDlg@@UAA@XZ    00019f70 f   miperrdlg.obj
 0001:00008f90       ?Create@CMipErrorDlg@@QAAHPAUHWND__@@@Z 00019f90 f   miperrdlg.obj
 0001:00009148       ?MipErrDlgProc@CMipErrorDlg@@SAHPAUHWND__@@IIJ@Z 0001a148 f   miperrdlg.obj
 0001:00009368       ?SetMessageText@CMipErrorDlg@@QAAXI@Z 0001a368 f   miperrdlg.obj
 0001:000093f4       ?SetErrId@CMipErrorDlg@@QAAXH@Z 0001a3f4 f   miperrdlg.obj
 0001:00009478       ?ShowWindow@CMipErrorDlg@@QAAXH@Z 0001a478 f   miperrdlg.obj
 0001:000094b0       ?BringWindowToTop@CMipErrorDlg@@QAAHXZ 0001a4b0 f   miperrdlg.obj
 0001:0000950c       ?Initialize@CMipErrorDlg@@QAAXXZ 0001a50c f   miperrdlg.obj
 0001:00009724       ??_ECMipErrorDlg@@UAAPAXI@Z 0001a724 f i miperrdlg.obj
 0001:00009724       ??_GCMipErrorDlg@@UAAPAXI@Z 0001a724 f i miperrdlg.obj
 0001:00009764       ??0CResultListElement@@QAA@XZ 0001a764 f   resultelement.obj
 0001:000097a8       ??1CResultListElement@@UAA@XZ 0001a7a8 f   resultelement.obj
 0001:000097c8       ?SetCallBackId@CResultListElement@@QAAXJ@Z 0001a7c8 f   resultelement.obj
 0001:000097e8       ?GetCallBackId@CResultListElement@@QAAJXZ 0001a7e8 f   resultelement.obj
 0001:00009814       ?SetFuncId@CResultListElement@@QAAXW4eFuncId@1@@Z 0001a814 f   resultelement.obj
 0001:00009834       ?GetFuncId@CResultListElement@@QAA?AW4eFuncId@1@XZ 0001a834 f   resultelement.obj
 0001:00009860       ??_ECResultListElement@@UAAPAXI@Z 0001a860 f i resultelement.obj
 0001:00009860       ??_GCResultListElement@@UAAPAXI@Z 0001a860 f i resultelement.obj
 0001:000098a0       ??0CSession@@QAA@XZ        0001a8a0 f   session.obj
 0001:00009910       ??1CSession@@UAA@XZ        0001a910 f   session.obj
 0001:00009950       ?GetSessionId@CSession@@QAAHXZ 0001a950 f   session.obj
 0001:0000999c       ?Create@CSession@@QAAKH@Z  0001a99c f   session.obj
 0001:000099f0       ?CheckDataPort@CSession@@QAA?AW4PortStatus@@XZ 0001a9f0 f   session.obj
 0001:00009a1c       ?CheckControlPort@CSession@@QAA?AW4PortStatus@@XZ 0001aa1c f   session.obj
 0001:00009a48       ?AppCheckTimer@@YAXPAUHWND__@@IIK@Z 0001aa48 f   session.obj
 0001:00009a58       ?GetSessionName@CSession@@QAAXPAG@Z 0001aa58 f   session.obj
 0001:00009a78       ?SetSessionName@CSession@@QAAXPBG@Z 0001aa78 f   session.obj
 0001:00009a98       ?CheckForModemStatus@CSession@@QAA_NXZ 0001aa98 f   session.obj
 0001:00009ae4       ?SetModemStatus@CSession@@QAAX_N@Z 0001aae4 f   session.obj
 0001:00009b1c       ?SetSessionId@CSession@@QAAXH@Z 0001ab1c f   session.obj
 0001:00009b54       ??_GCSession@@UAAPAXI@Z    0001ab54 f i session.obj
 0001:00009b54       ??_ECSession@@UAAPAXI@Z    0001ab54 f i session.obj
 0001:00009b94       ??0CSessionManager@@QAA@XZ 0001ab94 f   sessionmanager.obj
 0001:00009bec       ??1CSessionManager@@UAA@XZ 0001abec f   sessionmanager.obj
 0001:00009d9c       ?CreateSession@CSessionManager@@QAAKH@Z 0001ad9c f   sessionmanager.obj
 0001:00009f34       ?DeleteSession@CSessionManager@@QAA_NH@Z 0001af34 f   sessionmanager.obj
 0001:0000a1c0       ?IsAppRunning@CSessionManager@@QAA_NH@Z 0001b1c0 f   sessionmanager.obj
 0001:0000a404       ?Check@CSessionManager@@QAAKH@Z 0001b404 f   sessionmanager.obj
 0001:0000a880       ??_GCSessionManager@@UAAPAXI@Z 0001b880 f i sessionmanager.obj
 0001:0000a880       ??_ECSessionManager@@UAAPAXI@Z 0001b880 f i sessionmanager.obj
 0001:0000a8c0       ??1?$_Iterator@$00@?$list@PAVCSession@@V?$allocator@PAVCSession@@@std@@@std@@QAA@XZ 0001b8c0 f i sessionmanager.obj
 0001:0000a8d8       ??4?$_Iterator@$00@?$list@PAVCSession@@V?$allocator@PAVCSession@@@std@@@std@@QAAAAV012@ABV012@@Z 0001b8d8 f i sessionmanager.obj
 0001:0000a908       ??1?$_Const_iterator@$00@?$list@PAVCSession@@V?$allocator@PAVCSession@@@std@@@std@@QAA@XZ 0001b908 f i sessionmanager.obj
 0001:0000a920       ??4?$_Const_iterator@$00@?$list@PAVCSession@@V?$allocator@PAVCSession@@@std@@@std@@QAAAAV012@ABV012@@Z 0001b920 f i sessionmanager.obj
 0001:0000a968       ??1?$_Bidit@PAVCSession@@HPBQAV1@ABQAV1@@std@@QAA@XZ 0001b968 f i sessionmanager.obj
 0001:0000a988       ??1_Iterator_base@std@@QAA@XZ 0001b988 f i sessionmanager.obj
 0001:0000a9dc       ?_Orphan_me@_Iterator_base@std@@QAAXXZ 0001b9dc f i sessionmanager.obj
 0001:0000aaa4       ??4?$_Bidit@PAVCSession@@HPBQAV1@ABQAV1@@std@@QAAAAU01@ABU01@@Z 0001baa4 f i sessionmanager.obj
 0001:0000aadc       ??4_Iterator_base@std@@QAAAAV01@ABV01@@Z 0001badc f i sessionmanager.obj
 0001:0000ab6c       ?_Adopt@_Iterator_base@std@@QAAXPBV_Container_base@2@@Z 0001bb6c f i sessionmanager.obj
 0001:0000ac1c       ??0?$_Iterator@$00@?$list@PAVCSession@@V?$allocator@PAVCSession@@@std@@@std@@QAA@ABV012@@Z 0001bc1c f i sessionmanager.obj
 0001:0000ac50       ??0?$_Const_iterator@$00@?$list@PAVCSession@@V?$allocator@PAVCSession@@@std@@@std@@QAA@ABV012@@Z 0001bc50 f i sessionmanager.obj
 0001:0000ac9c       ??0?$_Bidit@PAVCSession@@HPBQAV1@ABQAV1@@std@@QAA@ABU01@@Z 0001bc9c f i sessionmanager.obj
 0001:0000acd0       ??0_Iterator_base@std@@QAA@ABV01@@Z 0001bcd0 f i sessionmanager.obj
 0001:0000ad24       ??0?$list@PAVCSession@@V?$allocator@PAVCSession@@@std@@@std@@QAA@XZ 0001bd24 f i sessionmanager.obj
 0001:0000adbc       ??1?$list@PAVCSession@@V?$allocator@PAVCSession@@@std@@@std@@QAA@XZ 0001bdbc f i sessionmanager.obj
 0001:0000adfc       ?begin@?$list@PAVCSession@@V?$allocator@PAVCSession@@@std@@@std@@QAA?AV?$_Iterator@$00@12@XZ 0001bdfc f i sessionmanager.obj
 0001:0000ae60       ?end@?$list@PAVCSession@@V?$allocator@PAVCSession@@@std@@@std@@QAA?AV?$_Iterator@$00@12@XZ 0001be60 f i sessionmanager.obj
 0001:0000aeb4       ?push_back@?$list@PAVCSession@@V?$allocator@PAVCSession@@@std@@@std@@QAAXABQAVCSession@@@Z 0001beb4 f i sessionmanager.obj
 0001:0000af04       ?erase@?$list@PAVCSession@@V?$allocator@PAVCSession@@@std@@@std@@QAA?AV?$_Iterator@$00@12@V312@@Z 0001bf04 f i sessionmanager.obj
 0001:0000b118       ??0?$_Iterator@$00@?$list@PAVCSession@@V?$allocator@PAVCSession@@@std@@@std@@QAA@XZ 0001c118 f i sessionmanager.obj
 0001:0000b148       ??D?$_Iterator@$00@?$list@PAVCSession@@V?$allocator@PAVCSession@@@std@@@std@@QBAAAPAVCSession@@XZ 0001c148 f i sessionmanager.obj
 0001:0000b178       ??E?$_Iterator@$00@?$list@PAVCSession@@V?$allocator@PAVCSession@@@std@@@std@@QAAAAV012@XZ 0001c178 f i sessionmanager.obj
 0001:0000b1a4       ??9?$_Const_iterator@$00@?$list@PAVCSession@@V?$allocator@PAVCSession@@@std@@@std@@QBA_NABV012@@Z 0001c1a4 f i sessionmanager.obj
 0001:0000b1fc       ??1?$_List_val@PAVCSession@@V?$allocator@PAVCSession@@@std@@@std@@QAA@XZ 0001c1fc f i sessionmanager.obj
 0001:0000b214       ??1?$_List_ptr@PAVCSession@@V?$allocator@PAVCSession@@@std@@@std@@QAA@XZ 0001c214 f i sessionmanager.obj
 0001:0000b22c       ??1?$_List_nod@PAVCSession@@V?$allocator@PAVCSession@@@std@@@std@@QAA@XZ 0001c22c f i sessionmanager.obj
 0001:0000b244       ??1_Container_base@std@@QAA@XZ 0001c244 f i sessionmanager.obj
 0001:0000b25c       ?_Orphan_all@_Container_base@std@@QBAXXZ 0001c25c f i sessionmanager.obj
 0001:0000b2f0       ?_Nextnode@?$list@PAVCSession@@V?$allocator@PAVCSession@@@std@@@std@@KAAAPAU_Node@?$_List_nod@PAVCSession@@V?$allocator@PAVCSession@@@std@@@2@PAU342@@Z 0001c2f0 f i sessionmanager.obj
 0001:0000b314       ?_Prevnode@?$list@PAVCSession@@V?$allocator@PAVCSession@@@std@@@std@@KAAAPAU_Node@?$_List_nod@PAVCSession@@V?$allocator@PAVCSession@@@std@@@2@PAU342@@Z 0001c314 f i sessionmanager.obj
 0001:0000b344       ?_Insert@?$list@PAVCSession@@V?$allocator@PAVCSession@@@std@@@std@@QAAXV?$_Iterator@$00@12@ABQAVCSession@@@Z 0001c344 f i sessionmanager.obj
 0001:0000b448       ?_Buynode@?$list@PAVCSession@@V?$allocator@PAVCSession@@@std@@@std@@IAAPAU_Node@?$_List_nod@PAVCSession@@V?$allocator@PAVCSession@@@std@@@2@XZ 0001c448 f i sessionmanager.obj
 0001:0000b54c       ?_Tidy@?$list@PAVCSession@@V?$allocator@PAVCSession@@@std@@@std@@IAAXXZ 0001c54c f i sessionmanager.obj
 0001:0000b5e0       ?_Orphan_ptr@?$list@PAVCSession@@V?$allocator@PAVCSession@@@std@@@std@@IBAXAAV12@PAU_Node@?$_List_nod@PAVCSession@@V?$allocator@PAVCSession@@@std@@@2@@Z 0001c5e0 f i sessionmanager.obj
 0001:0000b6b4       ??0?$_List_val@PAVCSession@@V?$allocator@PAVCSession@@@std@@@std@@QAA@V?$allocator@PAVCSession@@@1@@Z 0001c6b4 f i sessionmanager.obj
 0001:0000b710       ??0?$allocator@PAVCSession@@@std@@QAA@XZ 0001c710 f i sessionmanager.obj
 0001:0000b734       ?deallocate@?$allocator@U_Node@?$_List_nod@PAVCSession@@V?$allocator@PAVCSession@@@std@@@std@@@std@@QAAXPAU_Node@?$_List_nod@PAVCSession@@V?$allocator@PAVCSession@@@std@@@2@I@Z 0001c734 f i sessionmanager.obj
 0001:0000b74c       ?destroy@?$allocator@U_Node@?$_List_nod@PAVCSession@@V?$allocator@PAVCSession@@@std@@@std@@@std@@QAAXPAU_Node@?$_List_nod@PAVCSession@@V?$allocator@PAVCSession@@@std@@@2@@Z 0001c74c f i sessionmanager.obj
 0001:0000b764       ??0?$_Iterator@$00@?$list@PAVCSession@@V?$allocator@PAVCSession@@@std@@@std@@QAA@PAU_Node@?$_List_nod@PAVCSession@@V?$allocator@PAVCSession@@@std@@@2@PBV12@@Z 0001c764 f i sessionmanager.obj
 0001:0000b7a4       ??E?$_Iterator@$00@?$list@PAVCSession@@V?$allocator@PAVCSession@@@std@@@std@@QAA?AV012@H@Z 0001c7a4 f i sessionmanager.obj
 0001:0000b85c       ??0?$_Const_iterator@$00@?$list@PAVCSession@@V?$allocator@PAVCSession@@@std@@@std@@QAA@XZ 0001c85c f i sessionmanager.obj
 0001:0000b89c       ??D?$_Const_iterator@$00@?$list@PAVCSession@@V?$allocator@PAVCSession@@@std@@@std@@QBAABQAVCSession@@XZ 0001c89c f i sessionmanager.obj
 0001:0000b978       ??E?$_Const_iterator@$00@?$list@PAVCSession@@V?$allocator@PAVCSession@@@std@@@std@@QAAAAV012@XZ 0001c978 f i sessionmanager.obj
 0001:0000ba68       ??8?$_Const_iterator@$00@?$list@PAVCSession@@V?$allocator@PAVCSession@@@std@@@std@@QBA_NABV012@@Z 0001ca68 f i sessionmanager.obj
 0001:0000bad0       ?_Mynode@?$_Const_iterator@$00@?$list@PAVCSession@@V?$allocator@PAVCSession@@@std@@@std@@QBAPAU_Node@?$_List_nod@PAVCSession@@V?$allocator@PAVCSession@@@std@@@3@XZ 0001cad0 f i sessionmanager.obj
 0001:0000bafc       ??0?$_Bidit@PAVCSession@@HPBQAV1@ABQAV1@@std@@QAA@XZ 0001cafc f i sessionmanager.obj
 0001:0000bb2c       ??0_Iterator_base@std@@QAA@XZ 0001cb2c f i sessionmanager.obj
 0001:0000bb6c       ?_Myval@?$list@PAVCSession@@V?$allocator@PAVCSession@@@std@@@std@@KAAAPAVCSession@@PAU_Node@?$_List_nod@PAVCSession@@V?$allocator@PAVCSession@@@std@@@2@@Z 0001cb6c f i sessionmanager.obj
 0001:0000bb94       ?clear@?$list@PAVCSession@@V?$allocator@PAVCSession@@@std@@@std@@QAAXXZ 0001cb94 f i sessionmanager.obj
 0001:0000bca8       ?_Buynode@?$list@PAVCSession@@V?$allocator@PAVCSession@@@std@@@std@@IAAPAU_Node@?$_List_nod@PAVCSession@@V?$allocator@PAVCSession@@@std@@@2@PAU342@0ABQAVCSession@@@Z 0001cca8 f i sessionmanager.obj
 0001:0000be08       ?_Incsize@?$list@PAVCSession@@V?$allocator@PAVCSession@@@std@@@std@@IAAXI@Z 0001ce08 f i sessionmanager.obj
 0001:0000bed8       ??0length_error@std@@QAA@ABV?$basic_string@DU?$char_traits@D@std@@V?$allocator@D@2@@1@@Z 0001ced8 f i sessionmanager.obj
 0001:0000bf24       ??0logic_error@std@@QAA@ABV?$basic_string@DU?$char_traits@D@std@@V?$allocator@D@2@@1@@Z 0001cf24 f i sessionmanager.obj
 0001:0000bf94       ?what@logic_error@std@@UBAPBDXZ 0001cf94 f i sessionmanager.obj
 0001:0000bfc8       ??_Elogic_error@std@@UAAPAXI@Z 0001cfc8 f i sessionmanager.obj
 0001:0000bfc8       ??_Glogic_error@std@@UAAPAXI@Z 0001cfc8 f i sessionmanager.obj
 0001:0000c008       ??1logic_error@std@@UAA@XZ 0001d008 f i sessionmanager.obj
 0001:0000c03c       ??1length_error@std@@UAA@XZ 0001d03c f i sessionmanager.obj
 0001:0000c064       ??_Glength_error@std@@UAAPAXI@Z 0001d064 f i sessionmanager.obj
 0001:0000c064       ??_Elength_error@std@@UAAPAXI@Z 0001d064 f i sessionmanager.obj
 0001:0000c0ac       ??0?$basic_string@DU?$char_traits@D@std@@V?$allocator@D@2@@std@@QAA@ABV01@@Z 0001d0ac f i sessionmanager.obj
 0001:0000c14c       ??1?$basic_string@DU?$char_traits@D@std@@V?$allocator@D@2@@std@@QAA@XZ 0001d14c f i sessionmanager.obj
 0001:0000c194       ?c_str@?$basic_string@DU?$char_traits@D@std@@V?$allocator@D@2@@std@@QBAPBDXZ 0001d194 f i sessionmanager.obj
 0001:0000c1c4       ??1?$_String_val@DV?$allocator@D@std@@@std@@QAA@XZ 0001d1c4 f i sessionmanager.obj
 0001:0000c1dc       ??1_String_base@std@@QAA@XZ 0001d1dc f i sessionmanager.obj
 0001:0000c1f4       ?assign@?$basic_string@DU?$char_traits@D@std@@V?$allocator@D@2@@std@@QAAAAV12@ABV12@II@Z 0001d1f4 f i sessionmanager.obj
 0001:0000c318       ?_Tidy@?$basic_string@DU?$char_traits@D@std@@V?$allocator@D@2@@std@@IAAX_NI@Z 0001d318 f i sessionmanager.obj
 0001:0000c3c4       ?_Myptr@?$basic_string@DU?$char_traits@D@std@@V?$allocator@D@2@@std@@IBAPBDXZ 0001d3c4 f i sessionmanager.obj
 0001:0000c41c       ??0?$_String_val@DV?$allocator@D@std@@@std@@IAA@V?$allocator@D@1@@Z 0001d41c f i sessionmanager.obj
 0001:0000c45c       ??0?$allocator@D@std@@QAA@ABV01@@Z 0001d45c f i sessionmanager.obj
 0001:0000c480       ??0_String_base@std@@QAA@XZ 0001d480 f i sessionmanager.obj
 0001:0000c4b0       ??0_Container_base@std@@QAA@XZ 0001d4b0 f i sessionmanager.obj
 0001:0000c4e0       ?erase@?$basic_string@DU?$char_traits@D@std@@V?$allocator@D@2@@std@@QAAAAV12@II@Z 0001d4e0 f i sessionmanager.obj
 0001:0000c5f4       ?size@?$basic_string@DU?$char_traits@D@std@@V?$allocator@D@2@@std@@QBAIXZ 0001d5f4 f i sessionmanager.obj
 0001:0000c620       ?_Eos@?$basic_string@DU?$char_traits@D@std@@V?$allocator@D@2@@std@@IAAXI@Z 0001d620 f i sessionmanager.obj
 0001:0000c670       ?assign@?$char_traits@D@std@@SAXAADABD@Z 0001d670 f i sessionmanager.obj
 0001:0000c690       ?_Grow@?$basic_string@DU?$char_traits@D@std@@V?$allocator@D@2@@std@@IAA_NI_N@Z 0001d690 f i sessionmanager.obj
 0001:0000c7a4       ?_Myptr@?$basic_string@DU?$char_traits@D@std@@V?$allocator@D@2@@std@@IAAPADXZ 0001d7a4 f i sessionmanager.obj
 0001:0000c7fc       ?deallocate@?$allocator@D@std@@QAAXPADI@Z 0001d7fc f i sessionmanager.obj
 0001:0000c814       ??0?$_List_ptr@PAVCSession@@V?$allocator@PAVCSession@@@std@@@std@@IAA@V?$allocator@PAVCSession@@@1@@Z 0001d814 f i sessionmanager.obj
 0001:0000c870       ??0?$allocator@PAVCSession@@@std@@QAA@ABV01@@Z 0001d870 f i sessionmanager.obj
 0001:0000c894       ?allocate@?$allocator@U_Node@?$_List_nod@PAVCSession@@V?$allocator@PAVCSession@@@std@@@std@@@std@@QAAPAU_Node@?$_List_nod@PAVCSession@@V?$allocator@PAVCSession@@@std@@@2@I@Z 0001d894 f i sessionmanager.obj
 0001:0000c8c8       ?construct@?$allocator@PAU_Node@?$_List_nod@PAVCSession@@V?$allocator@PAVCSession@@@std@@@std@@@std@@QAAXPAPAU_Node@?$_List_nod@PAVCSession@@V?$allocator@PAVCSession@@@std@@@2@ABQAU342@@Z 0001d8c8 f i sessionmanager.obj
 0001:0000c8e4       ?destroy@?$allocator@PAU_Node@?$_List_nod@PAVCSession@@V?$allocator@PAVCSession@@@std@@@std@@@std@@QAAXPAPAU_Node@?$_List_nod@PAVCSession@@V?$allocator@PAVCSession@@@std@@@2@@Z 0001d8e4 f i sessionmanager.obj
 0001:0000c904       ??0?$_Const_iterator@$00@?$list@PAVCSession@@V?$allocator@PAVCSession@@@std@@@std@@QAA@PAU_Node@?$_List_nod@PAVCSession@@V?$allocator@PAVCSession@@@std@@@2@PBV12@@Z 0001d904 f i sessionmanager.obj
 0001:0000c96c       ?_Compat@?$_Const_iterator@$00@?$list@PAVCSession@@V?$allocator@PAVCSession@@@std@@@std@@QBAXABV123@@Z 0001d96c f i sessionmanager.obj
 0001:0000ca28       ??0length_error@std@@QAA@ABV01@@Z 0001da28 f i sessionmanager.obj
 0001:0000ca74       ??0logic_error@std@@QAA@ABV01@@Z 0001da74 f i sessionmanager.obj
 0001:0000caf4       ??0?$basic_string@DU?$char_traits@D@std@@V?$allocator@D@2@@std@@QAA@PBD@Z 0001daf4 f i sessionmanager.obj
 0001:0000cb74       ?max_size@?$basic_string@DU?$char_traits@D@std@@V?$allocator@D@2@@std@@QBAIXZ 0001db74 f i sessionmanager.obj
 0001:0000cbdc       ?_Copy@?$basic_string@DU?$char_traits@D@std@@V?$allocator@D@2@@std@@IAAXII@Z 0001dbdc f i sessionmanager.obj
 0001:0000ce10       ?max_size@?$list@PAVCSession@@V?$allocator@PAVCSession@@@std@@@std@@QBAIXZ 0001de10 f i sessionmanager.obj
 0001:0000ce44       ??0?$_List_nod@PAVCSession@@V?$allocator@PAVCSession@@@std@@@std@@IAA@V?$allocator@PAVCSession@@@1@@Z 0001de44 f i sessionmanager.obj
 0001:0000ce84       ?construct@?$allocator@PAVCSession@@@std@@QAAXPAPAVCSession@@ABQAV3@@Z 0001de84 f i sessionmanager.obj
 0001:0000cea0       ?assign@?$basic_string@DU?$char_traits@D@std@@V?$allocator@D@2@@std@@QAAAAV12@PBD@Z 0001dea0 f i sessionmanager.obj
 0001:0000cee4       ?length@?$char_traits@D@std@@SAIPBD@Z 0001dee4 f i sessionmanager.obj
 0001:0000cf14       ??0?$allocator@D@std@@QAA@XZ 0001df14 f i sessionmanager.obj
 0001:0000cf38       ?allocate@?$allocator@D@std@@QAAPADI@Z 0001df38 f i sessionmanager.obj
 0001:0000cf6c       ?max_size@?$allocator@D@std@@QBAIXZ 0001df6c f i sessionmanager.obj
 0001:0000cfb8       ?max_size@?$allocator@PAVCSession@@@std@@QBAIXZ 0001dfb8 f i sessionmanager.obj
 0001:0000d004       ?assign@?$basic_string@DU?$char_traits@D@std@@V?$allocator@D@2@@std@@QAAAAV12@PBDI@Z 0001e004 f i sessionmanager.obj
 0001:0000d0d0       ?_Inside@?$basic_string@DU?$char_traits@D@std@@V?$allocator@D@2@@std@@IAA_NPBD@Z 0001e0d0 f i sessionmanager.obj
 0001:0000d164       ??$_Debug_pointer@D@std@@YAXPBDPBGI@Z 0001e164 f i sessionmanager.obj
 0001:0000d194       ??$copy_s@U?$char_traits@D@std@@@_Traits_helper@std@@YAPADPADIPBDI@Z 0001e194 f i sessionmanager.obj
 0001:0000d1fc       ??$_Destroy@U_Node@?$_List_nod@PAVCSession@@V?$allocator@PAVCSession@@@std@@@std@@@std@@YAXPAU_Node@?$_List_nod@PAVCSession@@V?$allocator@PAVCSession@@@std@@@0@@Z 0001e1fc f i sessionmanager.obj
 0001:0000d20c       ??$move_s@U?$char_traits@D@std@@@_Traits_helper@std@@YAPADPADIPBDI@Z 0001e20c f i sessionmanager.obj
 0001:0000d274       ??$?0PAVCSession@@@?$allocator@PAU_Node@?$_List_nod@PAVCSession@@V?$allocator@PAVCSession@@@std@@@std@@@std@@QAA@ABV?$allocator@PAVCSession@@@1@@Z 0001e274 f i sessionmanager.obj
 0001:0000d298       ??$_Allocate@U_Node@?$_List_nod@PAVCSession@@V?$allocator@PAVCSession@@@std@@@std@@@std@@YAPAU_Node@?$_List_nod@PAVCSession@@V?$allocator@PAVCSession@@@std@@@0@IPAU120@@Z 0001e298 f i sessionmanager.obj
 0001:0000d328       ??0bad_alloc@std@@QAA@PBD@Z 0001e328 f i sessionmanager.obj
 0001:0000d36c       ??1bad_alloc@std@@UAA@XZ   0001e36c f i sessionmanager.obj
 0001:0000d394       ??_Ebad_alloc@std@@UAAPAXI@Z 0001e394 f i sessionmanager.obj
 0001:0000d394       ??_Gbad_alloc@std@@UAAPAXI@Z 0001e394 f i sessionmanager.obj
 0001:0000d3d4       ??$_Construct@PAU_Node@?$_List_nod@PAVCSession@@V?$allocator@PAVCSession@@@std@@@std@@PAU123@@std@@YAXPAPAU_Node@?$_List_nod@PAVCSession@@V?$allocator@PAVCSession@@@std@@@0@ABQAU120@@Z 0001e3d4 f i sessionmanager.obj
 0001:0000d43c       ??2@YAPAXIPAX@Z            0001e43c f i sessionmanager.obj
 0001:0000d460       ??$_Destroy@PAU_Node@?$_List_nod@PAVCSession@@V?$allocator@PAVCSession@@@std@@@std@@@std@@YAXPAPAU_Node@?$_List_nod@PAVCSession@@V?$allocator@PAVCSession@@@std@@@0@@Z 0001e460 f i sessionmanager.obj
 0001:0000d470       ??$?0PAVCSession@@@?$allocator@U_Node@?$_List_nod@PAVCSession@@V?$allocator@PAVCSession@@@std@@@std@@@std@@QAA@ABV?$allocator@PAVCSession@@@1@@Z 0001e470 f i sessionmanager.obj
 0001:0000d494       ??$_Construct@PAVCSession@@PAV1@@std@@YAXPAPAVCSession@@ABQAV1@@Z 0001e494 f i sessionmanager.obj
 0001:0000d4fc       ??$_Allocate@D@std@@YAPADIPAD@Z 0001e4fc f i sessionmanager.obj
 0001:0000d584       ??0bad_alloc@std@@QAA@ABV01@@Z 0001e584 f i sessionmanager.obj
 0001:0000d5c8       ??$_Char_traits_cat@U?$char_traits@D@std@@@std@@YA?AU_Secure_char_traits_tag@0@XZ 0001e5c8 f i sessionmanager.obj
 0001:0000d5fc       ??$copy_s@U?$char_traits@D@std@@@_Traits_helper@std@@YAPADPADIPBDIU_Secure_char_traits_tag@1@@Z 0001e5fc f i sessionmanager.obj
 0001:0000d638       ?_Copy_s@?$char_traits@D@std@@SAPADPADIPBDI@Z 0001e638 f i sessionmanager.obj
 0001:0000d670       ??$move_s@U?$char_traits@D@std@@@_Traits_helper@std@@YAPADPADIPBDIU_Secure_char_traits_tag@1@@Z 0001e670 f i sessionmanager.obj
 0001:0000d6ac       ?_Move_s@?$char_traits@D@std@@SAPADPADIPBDI@Z 0001e6ac f i sessionmanager.obj
 0001:0000d6e4       ??0CStateMachineMgr@@QAA@XZ 0001e6e4 f   statemachinemgr.obj
 0001:0000d80c       ??1CStateMachineMgr@@UAA@XZ 0001e80c f   statemachinemgr.obj
 0001:0000d838       ?CheckPhoneActivated@CStateMachineMgr@@QAA_NXZ 0001e838 f   statemachinemgr.obj
 0001:0000d884       ?UpdateStatusFromRIL@CStateMachineMgr@@QAAHXZ 0001e884 f   statemachinemgr.obj
 0001:0000d8fc       ?SetPhoneStatusCheck@CStateMachineMgr@@QAAX_N@Z 0001e8fc f   statemachinemgr.obj
 0001:0000d934       ?GetPhoneStatusCheck@CStateMachineMgr@@QAA_NXZ 0001e934 f   statemachinemgr.obj
 0001:0000d980       ?SetDeferredIOTATrigger@CStateMachineMgr@@QAAX_N@Z 0001e980 f   statemachinemgr.obj
 0001:0000d9b8       ?GetDeferredIOTATrigger@CStateMachineMgr@@QAA_NXZ 0001e9b8 f   statemachinemgr.obj
 0001:0000da04       ?GetServiceStatus@CStateMachineMgr@@QAA?AW4ServiceStatus@@XZ 0001ea04 f   statemachinemgr.obj
 0001:0000da50       ?CheckModemInUse@CStateMachineMgr@@QAA_NXZ 0001ea50 f   statemachinemgr.obj
 0001:0000da9c       ?SetModemInUse@CStateMachineMgr@@QAAX_N@Z 0001ea9c f   statemachinemgr.obj
 0001:0000dad4       ?Check@CStateMachineMgr@@QAAKH@Z 0001ead4 f   statemachinemgr.obj
 0001:0000e370       ?HangUpActiveDataCall@CStateMachineMgr@@QAA_NXZ 0001f370 f   statemachinemgr.obj
 0001:0000e610       ?GetControlPortStatus@CStateMachineMgr@@QAA?AW4PortStatus@@XZ 0001f610 f   statemachinemgr.obj
 0001:0000e65c       ?GetDataPortStatus@CStateMachineMgr@@QAA?AW4PortStatus@@XZ 0001f65c f   statemachinemgr.obj
 0001:0000e6a8       ?SetPhoneActiveState@CStateMachineMgr@@QAAX_N@Z 0001f6a8 f   statemachinemgr.obj
 0001:0000e6e0       ?SetSvcStatus@CStateMachineMgr@@QAAXW4ServiceStatus@@@Z 0001f6e0 f   statemachinemgr.obj
 0001:0000e718       ?SetDefaultSlotInfo@CStateMachineMgr@@QAA_NH@Z 0001f718 f   statemachinemgr.obj
 0001:0000e73c       ?SetDataCallStatus@CStateMachineMgr@@QAAXW4DataCallStatus@@@Z 0001f73c f   statemachinemgr.obj
 0001:0000e774       ?GetDataCallStatus@CStateMachineMgr@@QAA?AW4DataCallStatus@@XZ 0001f774 f   statemachinemgr.obj
 0001:0000e7c0       ?SetAALDeferredIOTATrigger@CStateMachineMgr@@QAAX_N@Z 0001f7c0 f   statemachinemgr.obj
 0001:0000e7f8       ?GetAALDeferredIOTATrigger@CStateMachineMgr@@QAA_NXZ 0001f7f8 f   statemachinemgr.obj
 0001:0000e844       ?SetCallStatus@CStateMachineMgr@@QAAXW4CallStatus@@@Z 0001f844 f   statemachinemgr.obj
 0001:0000e87c       ?GetCallStatus@CStateMachineMgr@@QAA?AW4CallStatus@@XZ 0001f87c f   statemachinemgr.obj
 0001:0000e8c8       ??_ECStateMachineMgr@@UAAPAXI@Z 0001f8c8 f i statemachinemgr.obj
 0001:0000e8c8       ??_GCStateMachineMgr@@UAAPAXI@Z 0001f8c8 f i statemachinemgr.obj
 0001:0000e908       ??0CUSSDDialog@@QAA@XZ     0001f908 f   USSDDialog.obj
 0001:0000e96c       ??1CUSSDDialog@@UAA@XZ     0001f96c f   USSDDialog.obj
 0001:0000e9c0       ?UpdateUSSDData@CUSSDDialog@@QAAXPAUrilsupservicedata_tag@@@Z 0001f9c0 f   USSDDialog.obj
 0001:0000ea98       ?Create@CUSSDDialog@@QAAHPAUHWND__@@PAUrilsupservicedata_tag@@@Z 0001fa98 f   USSDDialog.obj
 0001:0000ecf4       ?USSDDialogProc@CUSSDDialog@@SAHPAUHWND__@@IIJ@Z 0001fcf4 f   USSDDialog.obj
 0001:0000f050       ?SetMessageText@CUSSDDialog@@QAAXXZ 00020050 f   USSDDialog.obj
 0001:0000f360       ?ShowWindow@CUSSDDialog@@QAAXH@Z 00020360 f   USSDDialog.obj
 0001:0000f398       ?SetForegroundWindow@CUSSDDialog@@QAAHXZ 00020398 f   USSDDialog.obj
 0001:0000f3f4       ?Initialize@CUSSDDialog@@QAAXXZ 000203f4 f   USSDDialog.obj
 0001:0000f534       ??_GCUSSDDialog@@UAAPAXI@Z 00020534 f i USSDDialog.obj
 0001:0000f534       ??_ECUSSDDialog@@UAAPAXI@Z 00020534 f i USSDDialog.obj
 0001:0000f574       ??0CModemStatus@@QAA@XZ    00020574 f   winmodemstat.obj
 0001:0000f604       ??1CModemStatus@@UAA@XZ    00020604 f   winmodemstat.obj
 0001:0000f630       ?AddResultItem@CModemStatus@@KAXJW4eFuncId@CResultListElement@@K@Z 00020630 f   winmodemstat.obj
 0001:0000f768       ?Init@CModemStatus@@QAAJPAUHWND__@@@Z 00020768 f   winmodemstat.obj
 0001:0000f8b0       ?Deregister@CModemStatus@@SAXXZ 000208b0 f   winmodemstat.obj
 0001:0000f908       ?PrepareRilDevSpecificInfo@CModemStatus@@KAPAUtagDEVSPECIFICDATA@@KKAAK@Z 00020908 f   winmodemstat.obj
 0001:0000faac       ?ModGetSubscriberNumber@CModemStatus@@SAJXZ 00020aac f   winmodemstat.obj
 0001:0000fc6c       ?ModReadPDP@CModemStatus@@SAJK@Z 00020c6c f   winmodemstat.obj
 0001:0000fc98       ?SendSupServiceData@CModemStatus@@SAJPAGK@Z 00020c98 f   winmodemstat.obj
 0001:0000fd04       ?CancelSupServiceDataSession@CModemStatus@@SAJXZ 00020d04 f   winmodemstat.obj
 0001:0000fd58       ?ModGetOpState@CModemStatus@@SAJXZ 00020d58 f   winmodemstat.obj
 0001:0000fdb4       ?ModGetCallList@CModemStatus@@SAJXZ 00020db4 f   winmodemstat.obj
 0001:0000ff8c       ?ModGetRegistrationStatus@CModemStatus@@SAJXZ 00020f8c f   winmodemstat.obj
 0001:00010170       ?RilResultCallback@CModemStatus@@KAXKJPBXKK@Z 00021170 f   winmodemstat.obj
 0001:00010a04       ?RilNotifyCallback@CModemStatus@@KAXKPBXKK@Z 00021a04 f   winmodemstat.obj
 0001:0001115c       ?Read@CModemStatus@@SAJK@Z 0002215c f   winmodemstat.obj
 0001:000112ac       ?AddrStrToDW@CModemStatus@@KAKPBG@Z 000222ac f   winmodemstat.obj
 0001:000113c4       ?SetSlotInfo@CModemStatus@@SAHH@Z 000223c4 f   winmodemstat.obj
 0001:00011560       ?ExecNoParamDevSpecific@CModemStatus@@SAJK@Z 00022560 f   winmodemstat.obj
 0001:000117fc       ?Send2UI@CModemStatus@@SAJIIJ@Z 000227fc f   winmodemstat.obj
 0001:00011990       ?MessageBoxOnSeparateThread@CModemStatus@@QAAXPBG0I@Z 00022990 f   winmodemstat.obj
 0001:00011a7c       ?MessageBoxFunction@CModemStatus@@KAIPAX@Z 00022a7c f   winmodemstat.obj
 0001:00011afc       ?UpdateCallTypeAndStatus@CModemStatus@@KAKKKG@Z 00022afc f   winmodemstat.obj
 0001:00012640       ?ParseDetailErrorCode@CModemStatus@@SAHPAUtagRLE_RILDEVSPECIFIC_ErrorCode@@KG@Z 00023640 f   winmodemstat.obj
 0001:00012700       ?GetTestModeSettings@CModemStatus@@SAXXZ 00023700 f   winmodemstat.obj
 0001:000127a8       ?GetPowerSaveMode@CModemStatus@@SAXXZ 000237a8 f   winmodemstat.obj
 0001:00012850       ?PowerSaveExit@CModemStatus@@SAXXZ 00023850 f   winmodemstat.obj
 0001:000128f8       ?GetModemTime@CModemStatus@@SAHXZ 000238f8 f   winmodemstat.obj
 0001:0001295c       ?StartDMMode@CModemStatus@@SAHK@Z 0002395c f   winmodemstat.obj
 0001:00012a4c       ?StopDMMode@CModemStatus@@SAHXZ 00023a4c f   winmodemstat.obj
 0001:00012a94       ?IsDMMode@CModemStatus@@SAHXZ 00023a94 f   winmodemstat.obj
 0001:00012abc       ?StopEmergencyMode@CModemStatus@@SAJXZ 00023abc f   winmodemstat.obj
 0001:00012c98       ?ModSetEquipmentState@CModemStatus@@SAJK@Z 00023c98 f   winmodemstat.obj
 0001:00012ed0       ?HangUp@CModemStatus@@SAJXZ 00023ed0 f   winmodemstat.obj
 0001:00013074       ??_GCModemStatus@@UAAPAXI@Z 00024074 f i winmodemstat.obj
 0001:00013074       ??_ECModemStatus@@UAAPAXI@Z 00024074 f i winmodemstat.obj
 0001:000130b4       ??1?$_Iterator@$00@?$list@VCResultListElement@@V?$allocator@VCResultListElement@@@std@@@std@@QAA@XZ 000240b4 f i winmodemstat.obj
 0001:000130cc       ??0CResultListElement@@QAA@ABV0@@Z 000240cc f i winmodemstat.obj
 0001:00013148       ??1?$_Const_iterator@$00@?$list@VCResultListElement@@V?$allocator@VCResultListElement@@@std@@@std@@QAA@XZ 00024148 f i winmodemstat.obj
 0001:00013160       ??1?$_Bidit@VCResultListElement@@HPBV1@ABV1@@std@@QAA@XZ 00024160 f i winmodemstat.obj
 0001:00013178       GetCurrentProcess          00024178 f i winmodemstat.obj
 0001:00013190       ResetEvent                 00024190 f i winmodemstat.obj
 0001:000131c4       ?_AtlGetConversionACP@ATL@@YAIXZ 000241c4 f i winmodemstat.obj
 0001:000131dc       ?W2T@@YAPAGPAG@Z           000241dc f i winmodemstat.obj
 0001:00013200       ??4?$_Iterator@$00@?$list@VCResultListElement@@V?$allocator@VCResultListElement@@@std@@@std@@QAAAAV012@ABV012@@Z 00024200 f i winmodemstat.obj
 0001:00013230       ??4CResultListElement@@QAAAAV0@ABV0@@Z 00024230 f i winmodemstat.obj
 0001:0001329c       ??0?$_Iterator@$00@?$list@VCResultListElement@@V?$allocator@VCResultListElement@@@std@@@std@@QAA@ABV012@@Z 0002429c f i winmodemstat.obj
 0001:000132d0       ??4?$_Const_iterator@$00@?$list@VCResultListElement@@V?$allocator@VCResultListElement@@@std@@@std@@QAAAAV012@ABV012@@Z 000242d0 f i winmodemstat.obj
 0001:00013318       ??0?$_Const_iterator@$00@?$list@VCResultListElement@@V?$allocator@VCResultListElement@@@std@@@std@@QAA@ABV012@@Z 00024318 f i winmodemstat.obj
 0001:00013364       ??4?$_Bidit@VCResultListElement@@HPBV1@ABV1@@std@@QAAAAU01@ABU01@@Z 00024364 f i winmodemstat.obj
 0001:00013394       ??0?$_Bidit@VCResultListElement@@HPBV1@ABV1@@std@@QAA@ABU01@@Z 00024394 f i winmodemstat.obj
 0001:000133c8       ?begin@?$list@VCResultListElement@@V?$allocator@VCResultListElement@@@std@@@std@@QAA?AV?$_Iterator@$00@12@XZ 000243c8 f i winmodemstat.obj
 0001:0001342c       ?end@?$list@VCResultListElement@@V?$allocator@VCResultListElement@@@std@@@std@@QAA?AV?$_Iterator@$00@12@XZ 0002442c f i winmodemstat.obj
 0001:00013488       ?insert@?$list@VCResultListElement@@V?$allocator@VCResultListElement@@@std@@@std@@QAA?AV?$_Iterator@$00@12@V312@ABVCResultListElement@@@Z 00024488 f i winmodemstat.obj
 0001:0001356c       ?erase@?$list@VCResultListElement@@V?$allocator@VCResultListElement@@@std@@@std@@QAA?AV?$_Iterator@$00@12@V312@@Z 0002456c f i winmodemstat.obj
 0001:00013780       ??0?$_Iterator@$00@?$list@VCResultListElement@@V?$allocator@VCResultListElement@@@std@@@std@@QAA@XZ 00024780 f i winmodemstat.obj
 0001:000137b0       ??D?$_Iterator@$00@?$list@VCResultListElement@@V?$allocator@VCResultListElement@@@std@@@std@@QBAAAVCResultListElement@@XZ 000247b0 f i winmodemstat.obj
 0001:000137e8       ??E?$_Iterator@$00@?$list@VCResultListElement@@V?$allocator@VCResultListElement@@@std@@@std@@QAA?AV012@H@Z 000247e8 f i winmodemstat.obj
 0001:000138a0       ??9?$_Const_iterator@$00@?$list@VCResultListElement@@V?$allocator@VCResultListElement@@@std@@@std@@QBA_NABV012@@Z 000248a0 f i winmodemstat.obj
 0001:000138f8       ?_Nextnode@?$list@VCResultListElement@@V?$allocator@VCResultListElement@@@std@@@std@@KAAAPAU_Node@?$_List_nod@VCResultListElement@@V?$allocator@VCResultListElement@@@std@@@2@PAU342@@Z 000248f8 f i winmodemstat.obj
 0001:0001391c       ?_Prevnode@?$list@VCResultListElement@@V?$allocator@VCResultListElement@@@std@@@std@@KAAAPAU_Node@?$_List_nod@VCResultListElement@@V?$allocator@VCResultListElement@@@std@@@2@PAU342@@Z 0002491c f i winmodemstat.obj
 0001:0001394c       ?_Insert@?$list@VCResultListElement@@V?$allocator@VCResultListElement@@@std@@@std@@QAAXV?$_Iterator@$00@12@ABVCResultListElement@@@Z 0002494c f i winmodemstat.obj
 0001:00013a48       ?_Orphan_ptr@?$list@VCResultListElement@@V?$allocator@VCResultListElement@@@std@@@std@@IBAXAAV12@PAU_Node@?$_List_nod@VCResultListElement@@V?$allocator@VCResultListElement@@@std@@@2@@Z 00024a48 f i winmodemstat.obj
 0001:00013b1c       ?deallocate@?$allocator@U_Node@?$_List_nod@VCResultListElement@@V?$allocator@VCResultListElement@@@std@@@std@@@std@@QAAXPAU_Node@?$_List_nod@VCResultListElement@@V?$allocator@VCResultListElement@@@std@@@2@I@Z 00024b1c f i winmodemstat.obj
 0001:00013b34       ?destroy@?$allocator@U_Node@?$_List_nod@VCResultListElement@@V?$allocator@VCResultListElement@@@std@@@std@@@std@@QAAXPAU_Node@?$_List_nod@VCResultListElement@@V?$allocator@VCResultListElement@@@std@@@2@@Z 00024b34 f i winmodemstat.obj
 0001:00013b4c       ??0?$_Iterator@$00@?$list@VCResultListElement@@V?$allocator@VCResultListElement@@@std@@@std@@QAA@PAU_Node@?$_List_nod@VCResultListElement@@V?$allocator@VCResultListElement@@@std@@@2@PBV12@@Z 00024b4c f i winmodemstat.obj
 0001:00013b84       ??E?$_Iterator@$00@?$list@VCResultListElement@@V?$allocator@VCResultListElement@@@std@@@std@@QAAAAV012@XZ 00024b84 f i winmodemstat.obj
 0001:00013bb0       ??F?$_Iterator@$00@?$list@VCResultListElement@@V?$allocator@VCResultListElement@@@std@@@std@@QAAAAV012@XZ 00024bb0 f i winmodemstat.obj
 0001:00013bdc       ??0?$_Const_iterator@$00@?$list@VCResultListElement@@V?$allocator@VCResultListElement@@@std@@@std@@QAA@XZ 00024bdc f i winmodemstat.obj
 0001:00013c1c       ??D?$_Const_iterator@$00@?$list@VCResultListElement@@V?$allocator@VCResultListElement@@@std@@@std@@QBAABVCResultListElement@@XZ 00024c1c f i winmodemstat.obj
 0001:00013cf8       ??8?$_Const_iterator@$00@?$list@VCResultListElement@@V?$allocator@VCResultListElement@@@std@@@std@@QBA_NABV012@@Z 00024cf8 f i winmodemstat.obj
 0001:00013d60       ?_Mynode@?$_Const_iterator@$00@?$list@VCResultListElement@@V?$allocator@VCResultListElement@@@std@@@std@@QBAPAU_Node@?$_List_nod@VCResultListElement@@V?$allocator@VCResultListElement@@@std@@@3@XZ 00024d60 f i winmodemstat.obj
 0001:00013d8c       ??0?$_Bidit@VCResultListElement@@HPBV1@ABV1@@std@@QAA@XZ 00024d8c f i winmodemstat.obj
 0001:00013dbc       ?_Myval@?$list@VCResultListElement@@V?$allocator@VCResultListElement@@@std@@@std@@KAAAVCResultListElement@@PAU_Node@?$_List_nod@VCResultListElement@@V?$allocator@VCResultListElement@@@std@@@2@@Z 00024dbc f i winmodemstat.obj
 0001:00013dec       ?_Buynode@?$list@VCResultListElement@@V?$allocator@VCResultListElement@@@std@@@std@@IAAPAU_Node@?$_List_nod@VCResultListElement@@V?$allocator@VCResultListElement@@@std@@@2@PAU342@0ABVCResultListElement@@@Z 00024dec f i winmodemstat.obj
 0001:00013f4c       ?_Incsize@?$list@VCResultListElement@@V?$allocator@VCResultListElement@@@std@@@std@@IAAXI@Z 00024f4c f i winmodemstat.obj
 0001:0001401c       ?allocate@?$allocator@U_Node@?$_List_nod@VCResultListElement@@V?$allocator@VCResultListElement@@@std@@@std@@@std@@QAAPAU_Node@?$_List_nod@VCResultListElement@@V?$allocator@VCResultListElement@@@std@@@2@I@Z 0002501c f i winmodemstat.obj
 0001:00014050       ?construct@?$allocator@PAU_Node@?$_List_nod@VCResultListElement@@V?$allocator@VCResultListElement@@@std@@@std@@@std@@QAAXPAPAU_Node@?$_List_nod@VCResultListElement@@V?$allocator@VCResultListElement@@@std@@@2@ABQAU342@@Z 00025050 f i winmodemstat.obj
 0001:0001406c       ?destroy@?$allocator@PAU_Node@?$_List_nod@VCResultListElement@@V?$allocator@VCResultListElement@@@std@@@std@@@std@@QAAXPAPAU_Node@?$_List_nod@VCResultListElement@@V?$allocator@VCResultListElement@@@std@@@2@@Z 0002506c f i winmodemstat.obj
 0001:0001408c       ??0?$_Const_iterator@$00@?$list@VCResultListElement@@V?$allocator@VCResultListElement@@@std@@@std@@QAA@PAU_Node@?$_List_nod@VCResultListElement@@V?$allocator@VCResultListElement@@@std@@@2@PBV12@@Z 0002508c f i winmodemstat.obj
 0001:000140f4       ??E?$_Const_iterator@$00@?$list@VCResultListElement@@V?$allocator@VCResultListElement@@@std@@@std@@QAAAAV012@XZ 000250f4 f i winmodemstat.obj
 0001:000141e4       ??F?$_Const_iterator@$00@?$list@VCResultListElement@@V?$allocator@VCResultListElement@@@std@@@std@@QAAAAV012@XZ 000251e4 f i winmodemstat.obj
 0001:000142e0       ?_Compat@?$_Const_iterator@$00@?$list@VCResultListElement@@V?$allocator@VCResultListElement@@@std@@@std@@QBAXABV123@@Z 000252e0 f i winmodemstat.obj
 0001:0001439c       ?max_size@?$list@VCResultListElement@@V?$allocator@VCResultListElement@@@std@@@std@@QBAIXZ 0002539c f i winmodemstat.obj
 0001:000143d0       ?construct@?$allocator@VCResultListElement@@@std@@QAAXPAVCResultListElement@@ABV3@@Z 000253d0 f i winmodemstat.obj
 0001:000143ec       ?max_size@?$allocator@VCResultListElement@@@std@@QBAIXZ 000253ec f i winmodemstat.obj
 0001:00014438       ??$_Destroy@U_Node@?$_List_nod@VCResultListElement@@V?$allocator@VCResultListElement@@@std@@@std@@@std@@YAXPAU_Node@?$_List_nod@VCResultListElement@@V?$allocator@VCResultListElement@@@std@@@0@@Z 00025438 f i winmodemstat.obj
 0001:00014454       ??$_Allocate@U_Node@?$_List_nod@VCResultListElement@@V?$allocator@VCResultListElement@@@std@@@std@@@std@@YAPAU_Node@?$_List_nod@VCResultListElement@@V?$allocator@VCResultListElement@@@std@@@0@IPAU120@@Z 00025454 f i winmodemstat.obj
 0001:000144e4       ??$_Construct@PAU_Node@?$_List_nod@VCResultListElement@@V?$allocator@VCResultListElement@@@std@@@std@@PAU123@@std@@YAXPAPAU_Node@?$_List_nod@VCResultListElement@@V?$allocator@VCResultListElement@@@std@@@0@ABQAU120@@Z 000254e4 f i winmodemstat.obj
 0001:0001454c       ??$_Destroy@PAU_Node@?$_List_nod@VCResultListElement@@V?$allocator@VCResultListElement@@@std@@@std@@@std@@YAXPAPAU_Node@?$_List_nod@VCResultListElement@@V?$allocator@VCResultListElement@@@std@@@0@@Z 0002554c f i winmodemstat.obj
 0001:0001455c       ??$_Construct@VCResultListElement@@V1@@std@@YAXPAVCResultListElement@@ABV1@@Z 0002555c f i winmodemstat.obj
 0001:000145c4       ??_G_Node@?$_List_nod@VCResultListElement@@V?$allocator@VCResultListElement@@@std@@@std@@QAAPAXI@Z 000255c4 f i winmodemstat.obj
 0001:00014604       ??1_Node@?$_List_nod@VCResultListElement@@V?$allocator@VCResultListElement@@@std@@@std@@QAA@XZ 00025604 f i winmodemstat.obj
 0001:00014620       ??0CComCriticalSection@ATL@@QAA@XZ 00025620 f i winmodemstat.obj
 0001:00014654       ??1CComCriticalSection@ATL@@QAA@XZ 00025654 f i winmodemstat.obj
 0001:0001466c       ??0?$list@VCResultListElement@@V?$allocator@VCResultListElement@@@std@@@std@@QAA@XZ 0002566c f i winmodemstat.obj
 0001:000146fc       ??1?$_List_val@VCResultListElement@@V?$allocator@VCResultListElement@@@std@@@std@@QAA@XZ 000256fc f i winmodemstat.obj
 0001:00014714       ??1?$_List_ptr@VCResultListElement@@V?$allocator@VCResultListElement@@@std@@@std@@QAA@XZ 00025714 f i winmodemstat.obj
 0001:0001472c       ??1?$_List_nod@VCResultListElement@@V?$allocator@VCResultListElement@@@std@@@std@@QAA@XZ 0002572c f i winmodemstat.obj
 0001:0001474c       ?_Buynode@?$list@VCResultListElement@@V?$allocator@VCResultListElement@@@std@@@std@@IAAPAU_Node@?$_List_nod@VCResultListElement@@V?$allocator@VCResultListElement@@@std@@@2@XZ 0002574c f i winmodemstat.obj
 0001:00014850       ??0?$_List_val@VCResultListElement@@V?$allocator@VCResultListElement@@@std@@@std@@QAA@V?$allocator@VCResultListElement@@@1@@Z 00025850 f i winmodemstat.obj
 0001:000148ac       ??0?$allocator@VCResultListElement@@@std@@QAA@XZ 000258ac f i winmodemstat.obj
 0001:000148d0       ??0?$_List_ptr@VCResultListElement@@V?$allocator@VCResultListElement@@@std@@@std@@IAA@V?$allocator@VCResultListElement@@@1@@Z 000258d0 f i winmodemstat.obj
 0001:0001492c       ??0?$allocator@VCResultListElement@@@std@@QAA@ABV01@@Z 0002592c f i winmodemstat.obj
 0001:00014950       ??0?$_List_nod@VCResultListElement@@V?$allocator@VCResultListElement@@@std@@@std@@IAA@V?$allocator@VCResultListElement@@@1@@Z 00025950 f i winmodemstat.obj
 0001:00014990       ??$?0VCResultListElement@@@?$allocator@PAU_Node@?$_List_nod@VCResultListElement@@V?$allocator@VCResultListElement@@@std@@@std@@@std@@QAA@ABV?$allocator@VCResultListElement@@@1@@Z 00025990 f i winmodemstat.obj
 0001:000149b4       ??$?0VCResultListElement@@@?$allocator@U_Node@?$_List_nod@VCResultListElement@@V?$allocator@VCResultListElement@@@std@@@std@@@std@@QAA@ABV?$allocator@VCResultListElement@@@1@@Z 000259b4 f i winmodemstat.obj
 0001:000149d8       ?Term@CComCriticalSection@ATL@@QAAJXZ 000259d8 f i winmodemstat.obj
 0001:00014a04       ?_AtlRaiseException@ATL@@YAXKK@Z 00025a04 f i winmodemstat.obj
 0001:00014a30       ??1?$list@VCResultListElement@@V?$allocator@VCResultListElement@@@std@@@std@@QAA@XZ 00025a30 f i winmodemstat.obj
 0001:00014a70       ?_Tidy@?$list@VCResultListElement@@V?$allocator@VCResultListElement@@@std@@@std@@IAAXXZ 00025a70 f i winmodemstat.obj
 0001:00014b04       ?clear@?$list@VCResultListElement@@V?$allocator@VCResultListElement@@@std@@@std@@QAAXXZ 00025b04 f i winmodemstat.obj
 0001:00014c10       Process32Next              00025c10 f   toolhelp:toolhelp.dll
 0001:00014c20       CloseToolhelp32Snapshot    00025c20 f   toolhelp:toolhelp.dll
 0001:00014c30       Process32First             00025c30 f   toolhelp:toolhelp.dll
 0001:00014c40       CreateToolhelp32Snapshot   00025c40 f   toolhelp:toolhelp.dll
 0001:00014c50       Sleep                      00025c50 f   coredll:COREDLL.dll
 0001:00014c60       FindClose                  00025c60 f   coredll:COREDLL.dll
 0001:00014c70       FindFirstFileW             00025c70 f   coredll:COREDLL.dll
 0001:00014c80       DispatchMessageW           00025c80 f   coredll:COREDLL.dll
 0001:00014c90       TranslateMessage           00025c90 f   coredll:COREDLL.dll
 0001:00014ca0       GetMessageW                00025ca0 f   coredll:COREDLL.dll
 0001:00014cb0       wcscpy                     00025cb0 f   coredll:COREDLL.dll
 0001:00014cc0       GetLastError               00025cc0 f   coredll:COREDLL.dll
 0001:00014cd0       CreateMutexW               00025cd0 f   coredll:COREDLL.dll
 0001:00014ce0       WaitForSingleObject        00025ce0 f   coredll:COREDLL.dll
 0001:00014cf0       wcslen                     00025cf0 f   coredll:COREDLL.dll
 0001:00014d00       LoadLibraryW               00025d00 f   coredll:COREDLL.dll
 0001:00014d10       ??3@YAXPAX@Z               00025d10 f   coredll:COREDLL.dll
 0001:00014d20       CreateEventW               00025d20 f   coredll:COREDLL.dll
 0001:00014d30       InitializeCriticalSection  00025d30 f   coredll:COREDLL.dll
 0001:00014d40       ??2@YAPAXI@Z               00025d40 f   coredll:COREDLL.dll
 0001:00014d50       CloseHandle                00025d50 f   coredll:COREDLL.dll
 0001:00014d60       CreateThread               00025d60 f   coredll:COREDLL.dll
 0001:00014d70       EventModify                00025d70 f   coredll:COREDLL.dll
 0001:00014d80       MessageBoxW                00025d80 f   coredll:COREDLL.dll
 0001:00014d90       LoadStringW                00025d90 f   coredll:COREDLL.dll
 0001:00014da0       _wcsicmp                   00025da0 f   coredll:COREDLL.dll
 0001:00014db0       wcsrchr                    00025db0 f   coredll:COREDLL.dll
 0001:00014dc0       SystemIdleTimerReset       00025dc0 f   coredll:COREDLL.dll
 0001:00014dd0       PostMessageW               00025dd0 f   coredll:COREDLL.dll
 0001:00014de0       CreateProcessW             00025de0 f   coredll:COREDLL.dll
 0001:00014df0       DeleteCriticalSection      00025df0 f   coredll:COREDLL.dll
 0001:00014e00       OutputDebugStringW         00025e00 f   coredll:COREDLL.dll
 0001:00014e10       LeaveCriticalSection       00025e10 f   coredll:COREDLL.dll
 0001:00014e20       EnterCriticalSection       00025e20 f   coredll:COREDLL.dll
 0001:00014e30       NKDbgPrintfW               00025e30 f   coredll:COREDLL.dll
 0001:00014e40       RegisterWindowMessageW     00025e40 f   coredll:COREDLL.dll
 0001:00014e50       ShowWindow                 00025e50 f   coredll:COREDLL.dll
 0001:00014e60       EnableWindow               00025e60 f   coredll:COREDLL.dll
 0001:00014e70       GetDlgItem                 00025e70 f   coredll:COREDLL.dll
 0001:00014e80       SetWindowLongW             00025e80 f   coredll:COREDLL.dll
 0001:00014e90       CreateDialogIndirectParamW 00025e90 f   coredll:COREDLL.dll
 0001:00014ea0       LoadResource               00025ea0 f   coredll:COREDLL.dll
 0001:00014eb0       FindResourceW              00025eb0 f   coredll:COREDLL.dll
 0001:00014ec0       DestroyWindow              00025ec0 f   coredll:COREDLL.dll
 0001:00014ed0       GetWindowLongW             00025ed0 f   coredll:COREDLL.dll
 0001:00014ee0       SetDlgItemTextW            00025ee0 f   coredll:COREDLL.dll
 0001:00014ef0       wsprintfW                  00025ef0 f   coredll:COREDLL.dll
 0001:00014f00       SetForegroundWindow        00025f00 f   coredll:COREDLL.dll
 0001:00014f10       memset                     00025f10 f   coredll:COREDLL.dll
 0001:00014f20       DefWindowProcW             00025f20 f   coredll:COREDLL.dll
 0001:00014f30       KillTimer                  00025f30 f   coredll:COREDLL.dll
 0001:00014f40       memcpy                     00025f40 f   coredll:COREDLL.dll
 0001:00014f50       LoadImageW                 00025f50 f   coredll:COREDLL.dll
 0001:00014f60       SetTimer                   00025f60 f   coredll:COREDLL.dll
 0001:00014f70       RegCloseKey                00025f70 f   coredll:COREDLL.dll
 0001:00014f80       RegSetValueExW             00025f80 f   coredll:COREDLL.dll
 0001:00014f90       wcscmp                     00025f90 f   coredll:COREDLL.dll
 0001:00014fa0       wcsncpy                    00025fa0 f   coredll:COREDLL.dll
 0001:00014fb0       RegQueryValueExW           00025fb0 f   coredll:COREDLL.dll
 0001:00014fc0       RegOpenKeyExW              00025fc0 f   coredll:COREDLL.dll
 0001:00014fd0       RasEnumConnections         00025fd0 f   coredll:COREDLL.dll
 0001:00014fe0       SetSystemTime              00025fe0 f   coredll:COREDLL.dll
 0001:00014ff0       RasSetEntryDialParams      00025ff0 f   coredll:COREDLL.dll
 0001:00015000       RasGetEntryProperties      00026000 f   coredll:COREDLL.dll
 0001:00015010       RegisterClassW             00026010 f   coredll:COREDLL.dll
 0001:00015020       GetStockObject             00026020 f   coredll:COREDLL.dll
 0001:00015030       LoadIconW                  00026030 f   coredll:COREDLL.dll
 0001:00015040       CreateWindowExW            00026040 f   coredll:COREDLL.dll
 0001:00015050       SetWindowTextW             00026050 f   coredll:COREDLL.dll
 0001:00015060       BringWindowToTop           00026060 f   coredll:COREDLL.dll
 0001:00015070       __CxxThrowException        00026070 f   coredll:COREDLL.dll
 0001:00015080       ??_7type_info@@6B@         00026080 f   coredll:COREDLL.dll
 0001:00015090       ??0exception@std@@QAA@ABV01@@Z 00026090 f   coredll:COREDLL.dll
 0001:000150a0       ??1exception@std@@UAA@XZ   000260a0 f   coredll:COREDLL.dll
 0001:000150b0       ??0exception@std@@QAA@XZ   000260b0 f   coredll:COREDLL.dll
 0001:000150c0       strlen                     000260c0 f   coredll:COREDLL.dll
 0001:000150d0       ??0exception@std@@QAA@PBD@Z 000260d0 f   coredll:COREDLL.dll
 0001:000150e0       ?what@exception@std@@UBAPBDXZ 000260e0 f   coredll:COREDLL.dll
 0001:000150f0       FindWindowW                000260f0 f   coredll:COREDLL.dll
 0001:00015100       RasHangUp                  00026100 f   coredll:COREDLL.dll
 0001:00015110       RasGetConnectStatus        00026110 f   coredll:COREDLL.dll
 0001:00015120       ??_U@YAPAXI@Z              00026120 f   coredll:COREDLL.dll
 0001:00015130       GetDlgItemTextW            00026130 f   coredll:COREDLL.dll
 0001:00015140       wcscat                     00026140 f   coredll:COREDLL.dll
 0001:00015150       TerminateProcess           00026150 f   coredll:COREDLL.dll
 0001:00015160       ??_V@YAXPAX@Z              00026160 f   coredll:COREDLL.dll
 0001:00015170       swscanf                    00026170 f   coredll:COREDLL.dll
 0001:00015180       SendMessageTimeout         00026180 f   coredll:COREDLL.dll
 0001:00015190       free                       00026190 f   coredll:COREDLL.dll
 0001:000151a0       RaiseException             000261a0 f   coredll:COREDLL.dll
 0001:000151b0       ExitWindowsEx              000261b0 f   aygshell:AYGSHELL.dll
 0001:000151c0       SHInitDialog               000261c0 f   aygshell:AYGSHELL.dll
 0001:000151d0       SHCreateMenuBar            000261d0 f   aygshell:AYGSHELL.dll
 0001:000151e0       SHNotificationAdd          000261e0 f   aygshell:AYGSHELL.dll
 0001:000151f0       SHNotificationRemove       000261f0 f   aygshell:AYGSHELL.dll
 0001:00015200       SHNotificationUpdate       00026200 f   aygshell:AYGSHELL.dll
 0001:00015210       SHNotificationGetData      00026210 f   aygshell:AYGSHELL.dll
 0001:00015220       SHEnableSoftkey            00026220 f   aygshell:AYGSHELL.dll
 0001:00015230       RIL_Initialize             00026230 f   ril:ril.dll
 0001:00015240       RIL_Deinitialize           00026240 f   ril:ril.dll
 0001:00015250       RIL_GetSubscriberNumbers   00026250 f   ril:ril.dll
 0001:00015260       RIL_SendSupServiceData     00026260 f   ril:ril.dll
 0001:00015270       RIL_CancelSupServiceDataSession 00026270 f   ril:ril.dll
 0001:00015280       RIL_GetEquipmentState      00026280 f   ril:ril.dll
 0001:00015290       RIL_GetCallList            00026290 f   ril:ril.dll
 0001:000152a0       RIL_GetRegistrationStatus  000262a0 f   ril:ril.dll
 0001:000152b0       RIL_DevSpecific            000262b0 f   ril:ril.dll
 0001:000152c0       RIL_GetSystemTime          000262c0 f   ril:ril.dll
 0001:000152d0       RIL_SetEquipmentState      000262d0 f   ril:ril.dll
 0001:000152e0       RIL_Hangup                 000262e0 f   ril:ril.dll
 0001:000152f8       WinMainCRTStartup          000262f8 f   corelibc:pegwmain.obj
 0001:0001536c       __security_check_cookie    0002636c     corelibc:armsecgs.obj
 0001:00015380       __gsfailure                00026380     corelibc:armsecgs.obj
 0001:000153c4       _onexit                    000263c4 f   corelibc:onexit.obj
 0001:00015470       atexit                     00026470 f   corelibc:onexit.obj
 0001:00015490       _cinit                     00026490 f   corelibc:crt0dat.obj
 0001:00015600       exit                       00026600 f   corelibc:crt0dat.obj
 0001:00015618       _exit                      00026618 f   corelibc:crt0dat.obj
 0001:00015630       __security_init_cookie     00026630 f   corelibc:seccinit.obj
 0001:00015680       ??0_Init_locks@std@@QAA@XZ 00026680 f   libcpmtd:xlock.obj
 0001:000156e0       ??1_Init_locks@std@@QAA@XZ 000266e0 f   libcpmtd:xlock.obj
 0001:00015738       ??0_Lockit@std@@QAA@H@Z    00026738 f   libcpmtd:xlock.obj
 0001:00015774       ??1_Lockit@std@@QAA@XZ     00026774 f   libcpmtd:xlock.obj
 0001:000157a4       ?_Debug_message@std@@YAXPB_W0I@Z 000267a4 f   libcpmtd:stdthrow.obj
 0001:000157e4       ?_Debug_message@std@@YAXPBG0I@Z 000267e4 f   libcpmtd:stdthrow.obj
 0001:00015800       ??1out_of_range@std@@UAA@XZ 00026800 f i libcpmtd:string.obj
 0001:0001582c       ??_Eout_of_range@std@@UAAPAXI@Z 0002682c f i libcpmtd:string.obj
 0001:0001582c       ??_Gout_of_range@std@@UAAPAXI@Z 0002682c f i libcpmtd:string.obj
 0001:00015880       ?_Xlen@_String_base@std@@SAXXZ 00026880 f   libcpmtd:string.obj
 0001:00015910       ?_Xran@_String_base@std@@SAXXZ 00026910 f   libcpmtd:string.obj
 0001:00015998       ??0out_of_range@std@@QAA@ABV01@@Z 00026998 f i libcpmtd:string.obj
 0001:000159c8       _Mtxinit                   000269c8 f   libcpmtd:xmtx.obj
 0001:000159e4       _Mtxdst                    000269e4 f   libcpmtd:xmtx.obj
 0001:00015a00       _Mtxlock                   00026a00 f   libcpmtd:xmtx.obj
 0001:00015a1c       _Mtxunlock                 00026a1c f   libcpmtd:xmtx.obj
 0001:00015a38       __GSHandlerCheckCommon     00026a38 f   LIBCMTD:gshandler.obj
 0001:00015a80       __GSHandlerCheck           00026a80 f   LIBCMTD:gshandler.obj
 0001:00015ab0       __InternalCxxFrameHandler  00026ab0 f   LIBCMTD:frame_ce.obj
 0001:00015c8c       __CxxFrameHandler3         00026c8c f   LIBCMTD:frame_ce.obj
 0001:00016468       __FrameUnwindToState       00027468 f   LIBCMTD:frame_ce.obj
 0001:00017214       ?_DestructExceptionObject@@YAXPAUEHExceptionRecord@@E@Z 00028214 f   LIBCMTD:frame_ce.obj
 0001:00017364       ?_OffsetToAddress@@YAPAXHPAKK@Z 00028364 f   LIBCMTD:frame_ce.obj
 0001:000173f0       ?FindFrameInfo@@YAPAU_FrameInfo@@PAK@Z 000283f0 f   LIBCMTD:frame_ce.obj
 0001:00017478       ?FindCatchFrameInfo@@YAPAU_FrameInfo@@PAK@Z 00028478 f   LIBCMTD:frame_ce.obj
 0001:000174fc       ?_GetRangeOfTrysToCheck@@YAPBU_s_TryBlockMapEntry@@PBU_s_FuncInfo@@HHPAI1@Z 000284fc f   LIBCMTD:frame_ce.obj
 0001:000175f4       __GSHandlerCheck_EH        000285f4 f   LIBCMTD:gshandlereh.obj
 0001:00017688       _invalid_parameter         00028688 f   LIBCMTD:invarginternal.obj
 0001:000176cc       _CrtDbgReportW             000286cc f   LIBCMTD:dbgrpt.obj
 0001:00017744       _CrtDbgReportTV            00028744 f i LIBCMTD:dbgrpt.obj
 0001:000177a0       __crtMessageWindowW        000287a0 f   LIBCMTD:dbgrpt.obj
 0001:00017e78       _invoke_watson_if_error    00028e78 f i LIBCMTD:dbgrpt.obj
 0001:00017ecc       memcpy_s                   00028ecc f   LIBCMTD:memcpy_s.obj
 0001:00018184       memmove_s                  00029184 f   LIBCMTD:memmove_s.obj
 0001:000183f8       GetCRTStorage              000293f8 f   LIBCMTD:corecrt.obj
 0001:00018508       TlsAlloc                   00029508 f i LIBCMTD:corecrt.obj
 0001:00018544       TlsFree                    00029544 f i LIBCMTD:corecrt.obj
 0001:00018588       ?FindFrameForUnwind@@YAPAKPAKPBU_s_FuncInfo@@@Z 00029588 f   LIBCMTD:mdframe_arm.obj
 0001:00018620       ?FindCatchFrame@@YAPAKPAKK@Z 00029620 f   LIBCMTD:mdframe_arm.obj
 0001:000186b8       ?AdjustFrameForCatch@@YAPAKPAKPBU_s_FuncInfo@@@Z 000296b8 f   LIBCMTD:mdframe_arm.obj
 0001:00018758       ?GetCurrentState@@YAHPAKPAU_DISPATCHER_CONTEXT@@PBU_s_FuncInfo@@@Z 00029758 f   LIBCMTD:ehstate_arm_mips.obj
 0001:00018834       _CallSettingFrame          00029834     LIBCMTD:handlers_arm.obj
 0001:00018878       _invoke_watson             00029878 f   LIBCMTD:invarg.obj
 0001:000188ac       _mtinitlocks               000298ac f   LIBCMTD:mlock.obj
 0001:000189cc       _mtinitlocknum             000299cc f   LIBCMTD:mlock.obj
 0001:00018b34       _lock                      00029b34 f   LIBCMTD:mlock.obj
 0001:00018c30       _unlock                    00029c30 f   LIBCMTD:mlock.obj
 0001:00018c70       _lockerr_exit              00029c70 f   LIBCMTD:mlock.obj
 0001:00018c98       _CrtDbgBreak               00029c98 f   LIBCMTD:dbgrptt.obj
 0001:00018ca8       _VCrtDbgReportW            00029ca8 f   LIBCMTD:dbgrptt.obj
 0001:00019860       __crtMessageBoxW           0002a860 f   LIBCMTD:crtmbox.obj
 0001:00019ac4       wcsncpy_s                  0002aac4 f   LIBCMTD:wcsncpy_s.obj
 0001:0001a0c4       wcscpy_s                   0002b0c4 f   LIBCMTD:wcscpy_s.obj
 0001:0001a540       __crtInitCritSecAndSpinCount 0002b540 f   LIBCMTD:initcrit.obj
 0001:0001a670       _amsg_exit                 0002b670 f   LIBCMTD:crt0dat.obj
 0001:0001a69c       __crtExitProcess           0002b69c f   LIBCMTD:crt0dat.obj
 0001:0001a6e4       strcpy_s                   0002b6e4 f   LIBCMTD:strcpy_s.obj
 0001:0001ab38       wcscat_s                   0002bb38 f   LIBCMTD:wcscat_s.obj
 0001:0001b11c       _itow_s                    0002c11c f   LIBCMTD:xtows.obj
 0001:0001b7a8       _encode_pointer            0002c7a8 f   LIBCMTD:tidtable.obj
 0001:0001b7d0       _encoded_null              0002c7d0 f   LIBCMTD:tidtable.obj
 0001:0001b808       _decode_pointer            0002c808 f   LIBCMTD:tidtable.obj
 0001:0001b830       ?AtlAdvise@ATL@@YAJPAUIUnknown@@0ABU_GUID@@PAK@Z 0002c830 f   atlsd:atlfuncs.obj
 0001:0001b9ec       ?AtlUnadvise@ATL@@YAJPAUIUnknown@@ABU_GUID@@K@Z 0002c9ec f   atlsd:atlfuncs.obj
 0001:0001bba4       ?AtlFreeMarshalStream@ATL@@YAJPAUIStream@@@Z 0002cba4 f   atlsd:atlfuncs.obj
 0001:0001bc5c       ?AtlMarshalPtrInProc@ATL@@YAJPAUIUnknown@@ABU_GUID@@PAPAUIStream@@@Z 0002cc5c f   atlsd:atlfuncs.obj
 0001:0001bda0       ?AtlUnmarshalPtr@ATL@@YAJPAUIStream@@ABU_GUID@@PAPAUIUnknown@@@Z 0002cda0 f   atlsd:atlfuncs.obj
 0001:0001bec0       ?AtlComModuleGetClassObject@ATL@@YAJPAU_ATL_COM_MODULE70@1@ABU_GUID@@1PAPAX@Z 0002cec0 f   atlsd:atlfuncs.obj
 0001:0001c238       ?AtlComModuleRegisterClassObjects@ATL@@YAJPAU_ATL_COM_MODULE70@1@KK@Z 0002d238 f   atlsd:atlfuncs.obj
 0001:0001c358       ?AtlComModuleRevokeClassObjects@ATL@@YAJPAU_ATL_COM_MODULE70@1@@Z 0002d358 f   atlsd:atlfuncs.obj
 0001:0001c470       ?AtlWaitWithMessageLoop@ATL@@YAHPAX@Z 0002d470 f   atlsd:atlfuncs.obj
 0001:0001c608       ?AtlInternalQueryInterface@ATL@@YAJPAXPBU_ATL_INTMAP_ENTRY@1@ABU_GUID@@PAPAX@Z 0002d608 f   atlsd:atlfuncs.obj
 0001:0001c990       ?AtlGetVersion@ATL@@YAKPAX@Z 0002d990 f   atlsd:atlfuncs.obj
 0001:0001c9b8       ?AtlWinModuleAddCreateWndData@ATL@@YAXPAU_ATL_WIN_MODULE70@1@PAU_AtlCreateWndData@1@PAX@Z 0002d9b8 f   atlsd:atlfuncs.obj
 0001:0001cbf4       ?AtlWinModuleExtractCreateWndData@ATL@@YAPAXPAU_ATL_WIN_MODULE70@1@@Z 0002dbf4 f   atlsd:atlfuncs.obj
 0001:0001ce40       ?AtlWinModuleInit@ATL@@YAJPAU_ATL_WIN_MODULE70@1@@Z 0002de40 f   atlsd:atlfuncs.obj
 0001:0001cf90       ?AtlModuleAddTermFunc@ATL@@YAJPAU_ATL_MODULE70@1@P6AXK@ZK@Z 0002df90 f   atlsd:atlfuncs.obj
 0001:0001d19c       ?AtlCallTermFunc@ATL@@YAXPAU_ATL_MODULE70@1@@Z 0002e19c f   atlsd:atlfuncs.obj
 0001:0001d264       ??1?$CComPtr@UIConnectionPointContainer@@@ATL@@QAA@XZ 0002e264 f i atlsd:atlfuncs.obj
 0001:0001d28c       ??1?$CComPtr@UIConnectionPoint@@@ATL@@QAA@XZ 0002e28c f i atlsd:atlfuncs.obj
 0001:0001d2b4       GetCurrentThreadId         0002e2b4 f i atlsd:atlfuncs.obj
 0001:0001d2d4       ?IsWindowUnicode@ATL@@YAHPAUHWND__@@@Z 0002e2d4 f i atlsd:atlfuncs.obj
 0001:0001d2fc       ??0?$CComPtr@UIConnectionPointContainer@@@ATL@@QAA@XZ 0002e2fc f i atlsd:atlfuncs.obj
 0001:0001d33c       ??1?$CComPtrBase@UIConnectionPointContainer@@@ATL@@QAA@XZ 0002e33c f i atlsd:atlfuncs.obj
 0001:0001d384       ??I?$CComPtrBase@UIConnectionPointContainer@@@ATL@@QAAPAPAUIConnectionPointContainer@@XZ 0002e384 f i atlsd:atlfuncs.obj
 0001:0001d400       ??C?$CComPtrBase@UIConnectionPointContainer@@@ATL@@QBAPAV?$_NoAddRefReleaseOnCComPtr@UIConnectionPointContainer@@@1@XZ 0002e400 f i atlsd:atlfuncs.obj
 0001:0001d480       ??0?$CComPtr@UIConnectionPoint@@@ATL@@QAA@XZ 0002e480 f i atlsd:atlfuncs.obj
 0001:0001d4c0       ??1?$CComPtrBase@UIConnectionPoint@@@ATL@@QAA@XZ 0002e4c0 f i atlsd:atlfuncs.obj
 0001:0001d508       ??I?$CComPtrBase@UIConnectionPoint@@@ATL@@QAAPAPAUIConnectionPoint@@XZ 0002e508 f i atlsd:atlfuncs.obj
 0001:0001d584       ??C?$CComPtrBase@UIConnectionPoint@@@ATL@@QBAPAV?$_NoAddRefReleaseOnCComPtr@UIConnectionPoint@@@1@XZ 0002e584 f i atlsd:atlfuncs.obj
 0001:0001d604       ??0?$CComPtrBase@UIConnectionPointContainer@@@ATL@@IAA@XZ 0002e604 f i atlsd:atlfuncs.obj
 0001:0001d638       ??0?$CComPtrBase@UIConnectionPoint@@@ATL@@IAA@XZ 0002e638 f i atlsd:atlfuncs.obj
 0001:0001d66c       ?InlineIsEqualGUID@ATL@@YAHABU_GUID@@0@Z 0002e66c f i atlsd:atlfuncs.obj
 0001:0001d720       ??0CTraceFileAndLineInfo@ATL@@QAA@PBDH@Z 0002e720 f i atlsd:atlfuncs.obj
 0001:0001d764       ??RCTraceFileAndLineInfo@ATL@@QBAXKIPB_WZZ 0002e764 f i atlsd:atlfuncs.obj
 0001:0001d7dc       ?TraceV@CTrace@ATL@@QBAXPBDHKIPB_WPAD@Z 0002e7dc f i atlsd:atlfuncs.obj
 0001:0001d838       ??BCTraceCategory@ATL@@QBAKXZ 0002e838 f i atlsd:atlfuncs.obj
 0001:0001d86c       ?Init@CComCriticalSection@ATL@@QAAJXZ 0002e86c f i atlsd:atlfuncs.obj
 0001:0001d910       ?RevokeClassObject@_ATL_OBJMAP_ENTRY30@ATL@@QAAJXZ 0002e910 f i atlsd:atlfuncs.obj
 0001:0001d978       ?RegisterClassObject@_ATL_OBJMAP_ENTRY30@ATL@@QAAJKK@Z 0002e978 f i atlsd:atlfuncs.obj
 0001:0001da70       ?InlineIsEqualUnknown@ATL@@YAHABU_GUID@@@Z 0002ea70 f i atlsd:atlfuncs.obj
 0001:0001daf8       ??0?$CComCritSecLock@VCComCriticalSection@ATL@@@ATL@@QAA@AAVCComCriticalSection@1@_N@Z 0002eaf8 f i atlsd:atlfuncs.obj
 0001:0001db88       ?AtlThrowImpl@ATL@@YAXJ@Z  0002eb88 f i atlsd:atlfuncs.obj
 0001:0001dc98       ??1?$CComCritSecLock@VCComCriticalSection@ATL@@@ATL@@QAA@XZ 0002ec98 f i atlsd:atlfuncs.obj
 0001:0001dcd4       ?Unlock@?$CComCritSecLock@VCComCriticalSection@ATL@@@ATL@@QAAXXZ 0002ecd4 f i atlsd:atlfuncs.obj
 0001:0001dd74       ?Unlock@CComCriticalSection@ATL@@QAAJXZ 0002ed74 f i atlsd:atlfuncs.obj
 0001:0001ddb0       ?Lock@?$CComCritSecLock@VCComCriticalSection@ATL@@@ATL@@QAAJXZ 0002edb0 f i atlsd:atlfuncs.obj
 0001:0001de80       ?Lock@CComCriticalSection@ATL@@QAAJXZ 0002ee80 f i atlsd:atlfuncs.obj
 0001:0001debc       AtlRawDllMain              0002eebc f   atlsd:atlbase.obj
 0001:0001dfbc       ?CoDisconnectObject@ATL@@YAJPAUIUnknown@@K@Z 0002efbc f   atlsd:atlbase.obj
 0001:0001e110       ?CoInitialize@ATL@@YAJPAX@Z 0002f110 f   atlsd:atlbase.obj
 0001:0001e1c4       ?CoRevokeClassObject@ATL@@YAJK@Z 0002f1c4 f   atlsd:atlbase.obj
 0001:0001e278       ?CoRegisterClassObject@ATL@@YAJABU_GUID@@PAUIUnknown@@KKPAK@Z 0002f278 f   atlsd:atlbase.obj
 0001:0001e340       ?CoMarshalInterface@ATL@@YAJPAUIStream@@ABU_GUID@@PAUIUnknown@@KPAXK@Z 0002f340 f   atlsd:atlbase.obj
 0001:0001e410       ?CoUnmarshalInterface@ATL@@YAJPAUIStream@@ABU_GUID@@PAPAX@Z 0002f410 f   atlsd:atlbase.obj
 0001:0001e4cc       ?CoReleaseMarshalData@ATL@@YAJPAUIStream@@@Z 0002f4cc f   atlsd:atlbase.obj
 0001:0001e580       ?OleSaveToStream@ATL@@YAJPAUIPersistStream@@PAUIStream@@@Z 0002f580 f   atlsd:atlbase.obj
 0001:0001e738       ?OleLoadFromStream@ATL@@YAJPAUIStream@@ABU_GUID@@PAPAX@Z 0002f738 f   atlsd:atlbase.obj
 0001:0001ea64       ??0CAtlBaseModule@ATL@@QAA@XZ 0002fa64 f   atlsd:atlbase.obj
 0001:0001ebf0       ??1CAtlBaseModule@ATL@@QAA@XZ 0002fbf0 f   atlsd:atlbase.obj
 0001:0001ec30       ?AddResourceInstance@CAtlBaseModule@ATL@@QAA_NPAUHINSTANCE__@@@Z 0002fc30 f   atlsd:atlbase.obj
 0001:0001edcc       ?RemoveResourceInstance@CAtlBaseModule@ATL@@QAA_NPAUHINSTANCE__@@@Z 0002fdcc f   atlsd:atlbase.obj
 0001:0001efe0       ?GetHInstanceAt@CAtlBaseModule@ATL@@QAAPAUHINSTANCE__@@H@Z 0002ffe0 f   atlsd:atlbase.obj
 0001:0001f214       ??0_ATL_BASE_MODULE70@ATL@@QAA@XZ 00030214 f i atlsd:atlbase.obj
 0001:0001f274       ??1_ATL_BASE_MODULE70@ATL@@QAA@XZ 00030274 f i atlsd:atlbase.obj
 0001:0001f2b8       ?_AtlGetThisModuleHandle@ATL@@YAPAUHINSTANCE__@@XZ 000302b8 f i atlsd:atlbase.obj
 0001:0001f318       ??0?$CSimpleArray@PAUHINSTANCE__@@V?$CSimpleArrayEqualHelper@PAUHINSTANCE__@@@ATL@@@ATL@@QAA@XZ 00030318 f i atlsd:atlbase.obj
 0001:0001f36c       ?GetSize@?$CSimpleArray@PAUHINSTANCE__@@V?$CSimpleArrayEqualHelper@PAUHINSTANCE__@@@ATL@@@ATL@@QBAHXZ 0003036c f i atlsd:atlbase.obj
 0001:0001f39c       ?Add@?$CSimpleArray@PAUHINSTANCE__@@V?$CSimpleArrayEqualHelper@PAUHINSTANCE__@@@ATL@@@ATL@@QAAHABQAUHINSTANCE__@@@Z 0003039c f i atlsd:atlbase.obj
 0001:0001f4ec       ?RemoveAt@?$CSimpleArray@PAUHINSTANCE__@@V?$CSimpleArrayEqualHelper@PAUHINSTANCE__@@@ATL@@@ATL@@QAAHH@Z 000304ec f i atlsd:atlbase.obj
 0001:0001f664       ??A?$CSimpleArray@PAUHINSTANCE__@@V?$CSimpleArrayEqualHelper@PAUHINSTANCE__@@@ATL@@@ATL@@QAAAAPAUHINSTANCE__@@H@Z 00030664 f i atlsd:atlbase.obj
 0001:0001f748       ?InternalSetAtIndex@?$CSimpleArray@PAUHINSTANCE__@@V?$CSimpleArrayEqualHelper@PAUHINSTANCE__@@@ATL@@@ATL@@QAAXHABQAUHINSTANCE__@@@Z 00030748 f i atlsd:atlbase.obj
 0001:0001f7d8       ??0Wrapper@?$CSimpleArray@PAUHINSTANCE__@@V?$CSimpleArrayEqualHelper@PAUHINSTANCE__@@@ATL@@@ATL@@QAA@ABQAUHINSTANCE__@@@Z 000307d8 f i atlsd:atlbase.obj
 0001:0001f810       ??1?$CSimpleArray@PAUHINSTANCE__@@V?$CSimpleArrayEqualHelper@PAUHINSTANCE__@@@ATL@@@ATL@@QAA@XZ 00030810 f i atlsd:atlbase.obj
 0001:0001f838       ??$?2PAUHINSTANCE__@@@Wrapper@?$CSimpleArray@PAUHINSTANCE__@@V?$CSimpleArrayEqualHelper@PAUHINSTANCE__@@@ATL@@@ATL@@SAPAXIPAPAUHINSTANCE__@@@Z 00030838 f i atlsd:atlbase.obj
 0001:0001f860       ?RemoveAll@?$CSimpleArray@PAUHINSTANCE__@@V?$CSimpleArrayEqualHelper@PAUHINSTANCE__@@@ATL@@@ATL@@QAAXXZ 00030860 f i atlsd:atlbase.obj
 0001:0001f904       ?memmove_s@Checked@ATL@@YAXPAXIPBXI@Z 00030904 f i atlsd:atlbase.obj
 0001:0001f958       ?AtlCrtErrorCheck@ATL@@YAHH@Z 00030958 f i atlsd:atlbase.obj
 0001:0001fa24       ??1?$CComPtr@UIUnknown@@@ATL@@QAA@XZ 00030a24 f i atlsd:atlbase.obj
 0001:0001fa4c       ??1?$CComPtr@UIPersistStream@@@ATL@@QAA@XZ 00030a4c f i atlsd:atlbase.obj
 0001:0001fa74       ??0?$CComPtr@UIUnknown@@@ATL@@QAA@XZ 00030a74 f i atlsd:atlbase.obj
 0001:0001fab4       ??1?$CComPtrBase@UIUnknown@@@ATL@@QAA@XZ 00030ab4 f i atlsd:atlbase.obj
 0001:0001fafc       ??I?$CComPtrBase@UIUnknown@@@ATL@@QAAPAPAUIUnknown@@XZ 00030afc f i atlsd:atlbase.obj
 0001:0001fb78       ??C?$CComPtrBase@UIUnknown@@@ATL@@QBAPAV?$_NoAddRefReleaseOnCComPtr@UIUnknown@@@1@XZ 00030b78 f i atlsd:atlbase.obj
 0001:0001fbf8       ??0?$CComPtr@UIPersistStream@@@ATL@@QAA@XZ 00030bf8 f i atlsd:atlbase.obj
 0001:0001fc38       ??1?$CComPtrBase@UIPersistStream@@@ATL@@QAA@XZ 00030c38 f i atlsd:atlbase.obj
 0001:0001fc80       ??I?$CComPtrBase@UIPersistStream@@@ATL@@QAAPAPAUIPersistStream@@XZ 00030c80 f i atlsd:atlbase.obj
 0001:0001fcfc       ??C?$CComPtrBase@UIPersistStream@@@ATL@@QBAPAV?$_NoAddRefReleaseOnCComPtr@UIPersistStream@@@1@XZ 00030cfc f i atlsd:atlbase.obj
 0001:0001fd7c       ??0?$CComPtrBase@UIUnknown@@@ATL@@IAA@XZ 00030d7c f i atlsd:atlbase.obj
 0001:0001fdb0       ??0?$CComPtrBase@UIPersistStream@@@ATL@@IAA@XZ 00030db0 f i atlsd:atlbase.obj
 0001:0001fde4       ??0CTraceCategory@ATL@@QAA@PB_WI@Z 00030de4 f i atlsd:atltrace.obj
 0001:0001fe68       ?ChangeCategory@CTrace@ATL@@QAA_NKIW4ATLTRACESTATUS@2@@Z 00030e68 f i atlsd:atltrace.obj
 0001:0001fed8       ?RegisterCategory@CTrace@ATL@@QAAKPB_W@Z 00030ed8 f i atlsd:atltrace.obj
 0001:0001ff24       ??0CAtlAllocator@@QAA@XZ   00030f24 f i atlsd:Externs.obj
 0001:0001ffb4       ??0CTraceSnapshot@@QAA@XZ  00030fb4 f i atlsd:Externs.obj
 0001:00020010       ??0?$CSimpleArray@UCModuleInfo@CTraceSnapshot@@V?$CSimpleArrayEqualHelper@UCModuleInfo@CTraceSnapshot@@@ATL@@@ATL@@QAA@XZ 00031010 f i atlsd:Externs.obj
 0001:00020064       ??0?$CSimpleArray@KV?$CSimpleArrayEqualHelper@K@ATL@@@ATL@@QAA@XZ 00031064 f i atlsd:Externs.obj
 0001:00020228       GetCurrentProcessId        00031228 f i atlsd:Externs.obj
 0001:00020248       ??0CAtlException@ATL@@QAA@J@Z 00031248 f i atlsd:Externs.obj
 0001:0002027c       ??0CTrace@ATL@@AAA@P6AHHPB_WH00ZZ@Z 0003127c f i atlsd:Externs.obj
 0001:00020304       ??1CAtlAllocator@@QAA@XZ   00031304 f i atlsd:Externs.obj
 0001:00020344       ??1CTraceSnapshot@@QAA@XZ  00031344 f i atlsd:Externs.obj
 0001:00020384       ??1?$CSimpleArray@UCModuleInfo@CTraceSnapshot@@V?$CSimpleArrayEqualHelper@UCModuleInfo@CTraceSnapshot@@@ATL@@@ATL@@QAA@XZ 00031384 f i atlsd:Externs.obj
 0001:000203ac       ??1?$CSimpleArray@KV?$CSimpleArrayEqualHelper@K@ATL@@@ATL@@QAA@XZ 000313ac f i atlsd:Externs.obj
 0001:000203d4       ?RemoveAll@?$CSimpleArray@UCModuleInfo@CTraceSnapshot@@V?$CSimpleArrayEqualHelper@UCModuleInfo@CTraceSnapshot@@@ATL@@@ATL@@QAAXXZ 000313d4 f i atlsd:Externs.obj
 0001:00020478       ?RemoveAll@?$CSimpleArray@KV?$CSimpleArrayEqualHelper@K@ATL@@@ATL@@QAAXXZ 00031478 f i atlsd:Externs.obj
 0001:0002051c       ??1CTrace@ATL@@AAA@XZ      0003151c f i atlsd:Externs.obj
 0001:0002054c       ?NotifyTool@ATL@@YAXXZ     0003154c f   atlsd:AtlDebugAPI.obj
 0001:000205c4       AtlTraceRegister           000315c4 f   atlsd:AtlDebugAPI.obj
 0001:000206c0       AtlTraceUnregister         000316c0 f   atlsd:AtlDebugAPI.obj
 0001:00020720       AtlTraceRegisterCategoryU  00031720 f   atlsd:AtlDebugAPI.obj
 0001:000207ac       AtlTraceModifyProcess      000317ac f   atlsd:AtlDebugAPI.obj
 0001:0002092c       AtlTraceModifyModule       0003192c f   atlsd:AtlDebugAPI.obj
 0001:00020acc       AtlTraceModifyCategory     00031acc f   atlsd:AtlDebugAPI.obj
 0001:00020c0c       AtlTraceGetProcess         00031c0c f   atlsd:AtlDebugAPI.obj
 0001:00020dac       AtlTraceGetModule          00031dac f   atlsd:AtlDebugAPI.obj
 0001:00020f9c       AtlTraceGetCategory        00031f9c f   atlsd:AtlDebugAPI.obj
 0001:00021140       AtlTraceGetUpdateEventNameU 00032140 f   atlsd:AtlDebugAPI.obj
 0001:00021194       AtlTraceGetUpdateEventNameU_s 00032194 f   atlsd:AtlDebugAPI.obj
 0001:000211ec       AtlTraceVU                 000321ec f   atlsd:AtlDebugAPI.obj
 0001:000214fc       AtlTraceOpenProcess        000324fc f   atlsd:AtlDebugAPI.obj
 0001:00021558       AtlTraceCloseProcess       00032558 f   atlsd:AtlDebugAPI.obj
 0001:00021694       AtlTraceSnapshotProcess    00032694 f   atlsd:AtlDebugAPI.obj
 0001:0002176c       AtlTraceGetProcessInfo     0003276c f   atlsd:AtlDebugAPI.obj
 0001:00021a9c       AtlTraceGetModuleInfo      00032a9c f   atlsd:AtlDebugAPI.obj
 0001:00021d90       AtlTraceGetCategoryInfo    00032d90 f   atlsd:AtlDebugAPI.obj
 0001:00022448       ?GetProcess@CAtlAllocator@@QBAPAVCAtlTraceProcess@@XZ 00033448 f i atlsd:AtlDebugAPI.obj
 0001:00022478       ?Name@CAtlTraceCategory@@QBAPB_WXZ 00033478 f i atlsd:AtlDebugAPI.obj
 0001:000224a4       ?Path@CAtlTraceModuleInfo@@QBAPB_WXZ 000334a4 f i atlsd:AtlDebugAPI.obj
 0001:000224d0       ?Name@CAtlTraceModuleInfo@@QBAPB_WXZ 000334d0 f i atlsd:AtlDebugAPI.obj
 0001:000224fc       ?Id@CAtlTraceProcess@@QBAKXZ 000334fc f i atlsd:AtlDebugAPI.obj
 0001:00022530       ?CrtDbgReport@CAtlTraceModule@@QBAP6AHHPB_WH00ZZXZ 00033530 f i atlsd:AtlDebugAPI.obj
 0001:00022564       ?GetSize@?$CSimpleArray@UCModuleInfo@CTraceSnapshot@@V?$CSimpleArrayEqualHelper@UCModuleInfo@CTraceSnapshot@@@ATL@@@ATL@@QBAHXZ 00033564 f i atlsd:AtlDebugAPI.obj
 0001:00022594       ??A?$CSimpleArray@UCModuleInfo@CTraceSnapshot@@V?$CSimpleArrayEqualHelper@UCModuleInfo@CTraceSnapshot@@@ATL@@@ATL@@QAAAAUCModuleInfo@CTraceSnapshot@@H@Z 00033594 f i atlsd:AtlDebugAPI.obj
 0001:00022678       ?wcscpy_s@Checked@ATL@@YAXPA_WIPB_W@Z 00033678 f i atlsd:AtlDebugAPI.obj
 0001:000226d0       ?Init@CAtlAllocator@@QAA_NPB_WK@Z 000336d0 f   atlsd:Allocate.obj
 0001:00022ba8       ?Close@CAtlAllocator@@QAAX_N@Z 00033ba8 f   atlsd:Allocate.obj
 0001:00022c78       ?GetModule@CAtlAllocator@@QBAPAVCAtlTraceModule@@H@Z 00033c78 f   atlsd:Allocate.obj
 0001:00022d8c       ?GetCategory@CAtlAllocator@@QBAPAVCAtlTraceCategory@@H@Z 00033d8c f   atlsd:Allocate.obj
 0001:00022ed4       ?GetCategoryCount@CAtlAllocator@@QBAHH@Z 00033ed4 f   atlsd:Allocate.obj
 0001:00022fac       ?GetCategoryCount@CAtlAllocator@@QBAHABVCAtlTraceModule@@@Z 00033fac f   atlsd:Allocate.obj
 0001:00023048       ?GetModuleCount@CAtlAllocator@@QBAHXZ 00034048 f   atlsd:Allocate.obj
 0001:000230e8       ?FindModule@CAtlAllocator@@QBA_NPB_WPAI@Z 000340e8 f   atlsd:Allocate.obj
 0001:000231dc       ?AddModule@CAtlAllocator@@QAAHPAUHINSTANCE__@@@Z 000341dc f   atlsd:Allocate.obj
 0001:00023524       ?AddCategory@CAtlAllocator@@QAAHHPB_W@Z 00034524 f   atlsd:Allocate.obj
 0001:0002392c       ?RemoveModule@CAtlAllocator@@QAA_NH@Z 0003492c f   atlsd:Allocate.obj
 0001:00023a60       ?CleanUp@CAtlAllocator@@QAAXXZ 00034a60 f   atlsd:Allocate.obj
 0001:00023a8c       ?TakeSnapshot@CAtlAllocator@@QAAXXZ 00034a8c f   atlsd:Allocate.obj
 0001:00023dc8       ?ReleaseSnapshot@CAtlAllocator@@QAAXXZ 00034dc8 f   atlsd:Allocate.obj
 0001:00023f68       ?IncRef@CAtlTraceProcess@@QAAIXZ 00034f68 f i atlsd:Allocate.obj
 0001:00023fc0       ?Base@CAtlTraceProcess@@QBAPAXXZ 00034fc0 f i atlsd:Allocate.obj
 0001:00023ff4       ?DecRef@CAtlTraceProcess@@QAAIXZ 00034ff4 f i atlsd:Allocate.obj
 0001:0002404c       ?ModuleCount@CAtlTraceProcess@@QBAHXZ 0003504c f i atlsd:Allocate.obj
 0001:00024080       ?MaxSize@CAtlTraceProcess@@QBAKXZ 00035080 f i atlsd:Allocate.obj
 0001:000240b0       ?CategoryCount@CAtlTraceProcess@@QBAHXZ 000350b0 f i atlsd:Allocate.obj
 0001:000240e0       ?TryAllocate@CAtlTraceSettings@@QAA_NXZ 000350e0 f i atlsd:Allocate.obj
 0001:00024164       ?MarkValid@CAtlTraceSettings@@QAAXJ@Z 00035164 f i atlsd:Allocate.obj
 0001:000241e0       ?IncModuleCount@CAtlTraceProcess@@QAAXI@Z 000351e0 f i atlsd:Allocate.obj
 0001:0002421c       ?TryAddRef@CAtlTraceSettings@@QAA_NXZ 0003521c f i atlsd:Allocate.obj
 0001:000242ac       ?Release@CAtlTraceSettings@@QAAXXZ 000352ac f i atlsd:Allocate.obj
 0001:00024308       ?IncCategoryCount@CAtlTraceProcess@@QAAXI@Z 00035308 f i atlsd:Allocate.obj
 0001:0002433c       ?Add@?$CSimpleArray@UCModuleInfo@CTraceSnapshot@@V?$CSimpleArrayEqualHelper@UCModuleInfo@CTraceSnapshot@@@ATL@@@ATL@@QAAHABUCModuleInfo@CTraceSnapshot@@@Z 0003533c f i atlsd:Allocate.obj
 0001:00024494       ?GetSize@?$CSimpleArray@KV?$CSimpleArrayEqualHelper@K@ATL@@@ATL@@QBAHXZ 00035494 f i atlsd:Allocate.obj
 0001:000244c4       ?Add@?$CSimpleArray@KV?$CSimpleArrayEqualHelper@K@ATL@@@ATL@@QAAHABK@Z 000354c4 f i atlsd:Allocate.obj
 0001:00024614       ?RemoveAt@?$CSimpleArray@KV?$CSimpleArrayEqualHelper@K@ATL@@@ATL@@QAAHH@Z 00035614 f i atlsd:Allocate.obj
 0001:0002478c       ??A?$CSimpleArray@KV?$CSimpleArrayEqualHelper@K@ATL@@@ATL@@QAAAAKH@Z 0003578c f i atlsd:Allocate.obj
 0001:00024870       ?InternalSetAtIndex@?$CSimpleArray@UCModuleInfo@CTraceSnapshot@@V?$CSimpleArrayEqualHelper@UCModuleInfo@CTraceSnapshot@@@ATL@@@ATL@@QAAXHABUCModuleInfo@CTraceSnapshot@@@Z 00035870 f i atlsd:Allocate.obj
 0001:00024900       ?InternalSetAtIndex@?$CSimpleArray@KV?$CSimpleArrayEqualHelper@K@ATL@@@ATL@@QAAXHABK@Z 00035900 f i atlsd:Allocate.obj
 0001:00024990       ??0Wrapper@?$CSimpleArray@UCModuleInfo@CTraceSnapshot@@V?$CSimpleArrayEqualHelper@UCModuleInfo@CTraceSnapshot@@@ATL@@@ATL@@QAA@ABUCModuleInfo@CTraceSnapshot@@@Z 00035990 f i atlsd:Allocate.obj
 0001:000249c8       ??0Wrapper@?$CSimpleArray@KV?$CSimpleArrayEqualHelper@K@ATL@@@ATL@@QAA@ABK@Z 000359c8 f i atlsd:Allocate.obj
 0001:00024a00       ??$?2UCModuleInfo@CTraceSnapshot@@@Wrapper@?$CSimpleArray@UCModuleInfo@CTraceSnapshot@@V?$CSimpleArrayEqualHelper@UCModuleInfo@CTraceSnapshot@@@ATL@@@ATL@@SAPAXIPAUCModuleInfo@CTraceSnapshot@@@Z 00035a00 f i atlsd:Allocate.obj
 0001:00024a28       ??$?2K@Wrapper@?$CSimpleArray@KV?$CSimpleArrayEqualHelper@K@ATL@@@ATL@@SAPAXIPAK@Z 00035a28 f i atlsd:Allocate.obj
 0001:00024a50       ??0CAtlTraceModuleInfo@@QAA@XZ 00035a50 f   atlsd:AtlTraceModuleManager.obj
 0001:00024ac4       ?Reset@CAtlTraceModuleInfo@@QAAXPAUHINSTANCE__@@@Z 00035ac4 f   atlsd:AtlTraceModuleManager.obj
 0001:00024c60       ??0CAtlTraceCategory@@QAA@XZ 00035c60 f   atlsd:AtlTraceModuleManager.obj
 0001:00024ccc       ?Reset@CAtlTraceCategory@@QAAXPB_WJ@Z 00035ccc f   atlsd:AtlTraceModuleManager.obj
 0001:00024d4c       ??0CAtlTraceModule@@QAA@XZ 00035d4c f   atlsd:AtlTraceModuleManager.obj
 0001:00024db8       ?CrtDbgReport@CAtlTraceModule@@QAAXP6AHHPB_WH00ZZ@Z 00035db8 f   atlsd:AtlTraceModuleManager.obj
 0001:00024e0c       ??0CAtlTraceProcess@@QAA@K@Z 00035e0c f   atlsd:AtlTraceModuleManager.obj
 0001:00024f84       ?GetNextCookie@CAtlTraceProcess@@QAAJXZ 00035f84 f   atlsd:AtlTraceModuleManager.obj
 0001:00024fcc       ??0CAtlTraceSettings@@QAA@XZ 00035fcc f i atlsd:AtlTraceModuleManager.obj
 0001:00025030       _XcptFilter                00036030 f   coredll:COREDLL.dll
 0001:00025040       __C_specific_handler       00036040 f   coredll:COREDLL.dll
 0001:00025050       __report_gsfailure         00036050 f   coredll:COREDLL.dll
 0001:00025060       LocalReAlloc               00036060 f   coredll:COREDLL.dll
 0001:00025070       LocalAlloc                 00036070 f   coredll:COREDLL.dll
 0001:00025080       LocalSize                  00036080 f   coredll:COREDLL.dll
 0001:00025090       LocalFree                  00036090 f   coredll:COREDLL.dll
 0001:000250a0       __security_gen_cookie      000360a0 f   coredll:COREDLL.dll
 0001:000250b0       InterlockedIncrement       000360b0 f   coredll:COREDLL.dll
 0001:000250c0       InterlockedDecrement       000360c0 f   coredll:COREDLL.dll
 0001:000250d0       strcmp                     000360d0 f   coredll:COREDLL.dll
 0001:000250e0       ?terminate@std@@YAXXZ      000360e0 f   coredll:COREDLL.dll
 0001:000250f0       memmove                    000360f0 f   coredll:COREDLL.dll
 0001:00025100       malloc                     00036100 f   coredll:COREDLL.dll
 0001:00025110       _snwprintf                 00036110 f   coredll:COREDLL.dll
 0001:00025120       GetModuleFileNameW         00036120 f   coredll:COREDLL.dll
 0001:00025130       TlsSetValue                00036130 f   coredll:COREDLL.dll
 0001:00025140       TlsGetValue                00036140 f   coredll:COREDLL.dll
 0001:00025150       InterlockedCompareExchange 00036150 f   coredll:COREDLL.dll
 0001:00025160       TlsCall                    00036160 f   coredll:COREDLL.dll
 0001:00025170       WriteFile                  00036170 f   coredll:COREDLL.dll
 0001:00025180       wcstombs                   00036180 f   coredll:COREDLL.dll
 0001:00025190       _vsnwprintf                00036190 f   coredll:COREDLL.dll
 0001:000251a0       GetProcAddressW            000361a0 f   coredll:COREDLL.dll
 0001:000251b0       SetLastError               000361b0 f   coredll:COREDLL.dll
 0001:000251c0       PeekMessageW               000361c0 f   coredll:COREDLL.dll
 0001:000251d0       MsgWaitForMultipleObjectsEx 000361d0 f   coredll:COREDLL.dll
 0001:000251e0       GetModuleHandleW           000361e0 f   coredll:COREDLL.dll
 0001:000251f0       realloc                    000361f0 f   coredll:COREDLL.dll
 0001:00025200       OpenEventW                 00036200 f   coredll:COREDLL.dll
 0001:00025210       VirtualAlloc               00036210 f   coredll:COREDLL.dll
 0001:00025220       UnmapViewOfFile            00036220 f   coredll:COREDLL.dll
 0001:00025230       memcmp                     00036230 f   coredll:COREDLL.dll
 0001:00025240       GetSystemInfo              00036240 f   coredll:COREDLL.dll
 0001:00025250       MapViewOfFile              00036250 f   coredll:COREDLL.dll
 0001:00025260       CreateFileMappingW         00036260 f   coredll:COREDLL.dll
 0001:00025270       CreateStreamOnHGlobal      00036270 f   ole32:ole32.dll
 0001:00025280       WriteClassStm              00036280 f   ole32:ole32.dll
 0001:00025290       CoCreateInstance           00036290 f   ole32:ole32.dll
 0001:000252a0       ReadClassStm               000362a0 f   ole32:ole32.dll
 0002:000005f8       ??_7CAAMApp@@6B@           000385f8     aam.obj
 0002:000014e4       ??_7CArbitrator@@6B@       000394e4     arbitrator.obj
 0002:000015f4       ??_7CIota24Dlg@@6B@        000395f4     iota24dlg.obj
 0002:000052a0       ??_7CMainFrame@@6B@        0003d2a0     mainfrm.obj
 0002:00005334       ??_7CMipErrorDlg@@6B@      0003d334     miperrdlg.obj
 0002:00005338       ??_7CResultListElement@@6B@ 0003d338     resultelement.obj
 0002:00005388       ??_7CSession@@6B@          0003d388     session.obj
 0002:00005d64       ??_7CSessionManager@@6B@   0003dd64     sessionmanager.obj
 0002:00005da4       ??_C@_1DC@POOIKBAO@?$AAI?$AAT?$AAE?$AAR?$AAA?$AAT?$AAO?$AAR?$AA?5?$AAL?$AAI?$AAS?$AAT?$AA?5?$AAC?$AAO?$AAR?$AAR?$AAU?$AAP?$AAT?$AAE?$AAD?$AA?$CB?$AA?$AA@ 0003dda4     sessionmanager.obj
 0002:00005dd8       ??_C@_1IE@BKKAAKCG@?$AAC?$AA?3?$AA?2?$AAP?$AAr?$AAo?$AAg?$AAr?$AAa?$AAm?$AA?5?$AAF?$AAi?$AAl?$AAe?$AAs?$AA?2?$AAM?$AAi?$AAc?$AAr?$AAo?$AAs?$AAo?$AAf?$AAt?$AA?5?$AAV?$AAi?$AAs?$AAu?$AAa@ 0003ddd8     sessionmanager.obj
 0002:00005f58       ??_C@_1EE@BBMFLDOC@?$AAl?$AAi?$AAs?$AAt?$AA?5?$AAe?$AAr?$AAa?$AAs?$AAe?$AA?5?$AAi?$AAt?$AAe?$AAr?$AAa?$AAt?$AAo?$AAr?$AA?5?$AAo?$AAu?$AAt?$AAs?$AAi?$AAd?$AAe?$AA?5?$AAr?$AAa?$AAn?$AAg@ 0003df58     sessionmanager.obj
 0002:00005fa0       ??_C@_1HM@HPOOGGJN@?$AAC?$AA?3?$AA?2?$AAP?$AAr?$AAo?$AAg?$AAr?$AAa?$AAm?$AA?5?$AAF?$AAi?$AAl?$AAe?$AAs?$AA?2?$AAM?$AAi?$AAc?$AAr?$AAo?$AAs?$AAo?$AAf?$AAt?$AA?5?$AAV?$AAi?$AAs?$AAu?$AAa@ 0003dfa0     sessionmanager.obj
 0002:00006080       ??_C@_1EG@BPNHNPIG@?$AAl?$AAi?$AAs?$AAt?$AA?5?$AAi?$AAn?$AAs?$AAe?$AAr?$AAt?$AA?5?$AAi?$AAt?$AAe?$AAr?$AAa?$AAt?$AAo?$AAr?$AA?5?$AAo?$AAu?$AAt?$AAs?$AAi?$AAd?$AAe?$AA?5?$AAr?$AAa?$AAn@ 0003e080     sessionmanager.obj
 0002:000061bc       ??_C@_1BO@MEPPHOO@?$AA?$CC?$AAo?$AAu?$AAt?$AA?5?$AAo?$AAf?$AA?5?$AAr?$AAa?$AAn?$AAg?$AAe?$AA?$CC?$AA?$AA@ 0003e1bc     sessionmanager.obj
 0002:000061e0       ??_C@_1MI@FDDKHILP@?$AAs?$AAt?$AAd?$AA?3?$AA?3?$AAl?$AAi?$AAs?$AAt?$AA?$DM?$AAc?$AAl?$AAa?$AAs?$AAs?$AA?5?$AAC?$AAS?$AAe?$AAs?$AAs?$AAi?$AAo?$AAn?$AA?5?$AA?$CK?$AA?0?$AAc?$AAl?$AAa?$AAs?$AAs@ 0003e1e0     sessionmanager.obj
 0002:000062a8       ??_C@_1FG@CMLDHNON@?$AA?$CI?$AA?$CC?$AAS?$AAt?$AAa?$AAn?$AAd?$AAa?$AAr?$AAd?$AA?5?$AAC?$AA?$CL?$AA?$CL?$AA?5?$AAL?$AAi?$AAb?$AAr?$AAa?$AAr?$AAi?$AAe?$AAs?$AA?5?$AAO?$AAu?$AAt?$AA?5?$AAo?$AAf?$AA?5@ 0003e2a8     sessionmanager.obj
 0002:00006300       ??_C@_1EC@HILJLMMC@?$AAl?$AAi?$AAs?$AAt?$AA?5?$AAi?$AAt?$AAe?$AAr?$AAa?$AAt?$AAo?$AAr?$AA?5?$AAn?$AAo?$AAt?$AA?5?$AAd?$AAe?$AAr?$AAe?$AAf?$AAe?$AAr?$AAe?$AAn?$AAc?$AAa?$AAb?$AAl?$AAe@ 0003e300     sessionmanager.obj
 0002:00006348       ??_C@_1MK@IBOMODNJ@?$AAs?$AAt?$AAd?$AA?3?$AA?3?$AAl?$AAi?$AAs?$AAt?$AA?$DM?$AAc?$AAl?$AAa?$AAs?$AAs?$AA?5?$AAC?$AAS?$AAe?$AAs?$AAs?$AAi?$AAo?$AAn?$AA?5?$AA?$CK?$AA?0?$AAc?$AAl?$AAa?$AAs?$AAs@ 0003e348     sessionmanager.obj
 0002:00006418       ??_C@_1EA@DOGAGKDH@?$AAl?$AAi?$AAs?$AAt?$AA?5?$AAi?$AAt?$AAe?$AAr?$AAa?$AAt?$AAo?$AAr?$AA?5?$AAn?$AAo?$AAt?$AA?5?$AAi?$AAn?$AAc?$AAr?$AAe?$AAm?$AAe?$AAn?$AAt?$AAa?$AAb?$AAl?$AAe?$AA?$AA@ 0003e418     sessionmanager.obj
 0002:000064c4       ??_C@_0BB@MOGOBHAF@list?$DMT?$DO?5too?5long?$AA@ 0003e4c4     sessionmanager.obj
 0002:0000654c       ?npos@?$basic_string@DU?$char_traits@D@std@@V?$allocator@D@2@@std@@2IB 0003e54c     sessionmanager.obj
 0002:000065fc       ??_C@_1CG@JNLFBNGN@?$AA?$CC?$AAi?$AAn?$AAv?$AAa?$AAl?$AAi?$AAd?$AA?5?$AAa?$AAr?$AAg?$AAu?$AAm?$AAe?$AAn?$AAt?$AA?$CC?$AA?$AA@ 0003e5fc     sessionmanager.obj
 0002:00006628       ??_C@_1MC@LGNMKBFJ@?$AAs?$AAt?$AAd?$AA?3?$AA?3?$AAl?$AAi?$AAs?$AAt?$AA?$DM?$AAc?$AAl?$AAa?$AAs?$AAs?$AA?5?$AAC?$AAS?$AAe?$AAs?$AAs?$AAi?$AAo?$AAn?$AA?5?$AA?$CK?$AA?0?$AAc?$AAl?$AAa?$AAs?$AAs@ 0003e628     sessionmanager.obj
 0002:000066f0       ??_C@_1FO@OCPOOAIA@?$AA?$CI?$AA?$CC?$AAS?$AAt?$AAa?$AAn?$AAd?$AAa?$AAr?$AAd?$AA?5?$AAC?$AA?$CL?$AA?$CL?$AA?5?$AAL?$AAi?$AAb?$AAr?$AAa?$AAr?$AAi?$AAe?$AAs?$AA?5?$AAI?$AAn?$AAv?$AAa?$AAl?$AAi?$AAd@ 0003e6f0     sessionmanager.obj
 0002:00006750       ??_C@_1DI@MDELDGPI@?$AAl?$AAi?$AAs?$AAt?$AA?5?$AAi?$AAt?$AAe?$AAr?$AAa?$AAt?$AAo?$AAr?$AAs?$AA?5?$AAi?$AAn?$AAc?$AAo?$AAm?$AAp?$AAa?$AAt?$AAi?$AAb?$AAl?$AAe?$AA?$AA@ 0003e750     sessionmanager.obj
 0002:000068b0       ??_C@_1IC@HKDJIJDA@?$AAC?$AA?3?$AA?2?$AAP?$AAr?$AAo?$AAg?$AAr?$AAa?$AAm?$AA?5?$AAF?$AAi?$AAl?$AAe?$AAs?$AA?2?$AAM?$AAi?$AAc?$AAr?$AAo?$AAs?$AAo?$AAf?$AAt?$AA?5?$AAV?$AAi?$AAs?$AAu?$AAa@ 0003e8b0     sessionmanager.obj
 0002:00006934       ??_C@_1CK@EOPGIILJ@?$AAi?$AAn?$AAv?$AAa?$AAl?$AAi?$AAd?$AA?5?$AAn?$AAu?$AAl?$AAl?$AA?5?$AAp?$AAo?$AAi?$AAn?$AAt?$AAe?$AAr?$AA?$AA@ 0003e934     sessionmanager.obj
 0002:0000753c       ??_7CStateMachineMgr@@6B@  0003f53c     statemachinemgr.obj
 0002:00007e48       ??_7CUSSDDialog@@6B@       0003fe48     USSDDialog.obj
 0002:0000b7c4       ??_7CModemStatus@@6B@      000437c4     winmodemstat.obj
 0002:0000b8f8       ??_C@_1OI@CFPJBECN@?$AAs?$AAt?$AAd?$AA?3?$AA?3?$AAl?$AAi?$AAs?$AAt?$AA?$DM?$AAc?$AAl?$AAa?$AAs?$AAs?$AA?5?$AAC?$AAR?$AAe?$AAs?$AAu?$AAl?$AAt?$AAL?$AAi?$AAs?$AAt?$AAE?$AAl?$AAe?$AAm?$AAe@ 000438f8     winmodemstat.obj
 0002:0000bac8       ??_C@_1OK@IGJPFAPB@?$AAs?$AAt?$AAd?$AA?3?$AA?3?$AAl?$AAi?$AAs?$AAt?$AA?$DM?$AAc?$AAl?$AAa?$AAs?$AAs?$AA?5?$AAC?$AAR?$AAe?$AAs?$AAu?$AAl?$AAt?$AAL?$AAi?$AAs?$AAt?$AAE?$AAl?$AAe?$AAm?$AAe@ 00043ac8     winmodemstat.obj
 0002:0000bbb8       ??_C@_1OK@HFKNOMDA@?$AAs?$AAt?$AAd?$AA?3?$AA?3?$AAl?$AAi?$AAs?$AAt?$AA?$DM?$AAc?$AAl?$AAa?$AAs?$AAs?$AA?5?$AAC?$AAR?$AAe?$AAs?$AAu?$AAl?$AAt?$AAL?$AAi?$AAs?$AAt?$AAE?$AAl?$AAe?$AAm?$AAe@ 00043bb8     winmodemstat.obj
 0002:0000bca8       ??_C@_1EA@JDNDELPC@?$AAl?$AAi?$AAs?$AAt?$AA?5?$AAi?$AAt?$AAe?$AAr?$AAa?$AAt?$AAo?$AAr?$AA?5?$AAn?$AAo?$AAt?$AA?5?$AAd?$AAe?$AAc?$AAr?$AAe?$AAm?$AAe?$AAn?$AAt?$AAa?$AAb?$AAl?$AAe?$AA?$AA@ 00043ca8     winmodemstat.obj
 0002:0000bce8       ??_C@_1OC@OBKBLNGA@?$AAs?$AAt?$AAd?$AA?3?$AA?3?$AAl?$AAi?$AAs?$AAt?$AA?$DM?$AAc?$AAl?$AAa?$AAs?$AAs?$AA?5?$AAC?$AAR?$AAe?$AAs?$AAu?$AAl?$AAt?$AAL?$AAi?$AAs?$AAt?$AAE?$AAl?$AAe?$AAm?$AAe@ 00043ce8     winmodemstat.obj
 0002:0000be78       ??_C@_1EA@JHMKKLFC@?$AAn?$AAI?$AAn?$AAd?$AAe?$AAx?$AA?5?$AA?$DO?$AA?$DN?$AA?5?$AA0?$AA?5?$AA?$CG?$AA?$CG?$AA?5?$AAn?$AAI?$AAn?$AAd?$AAe?$AAx?$AA?5?$AA?$DM?$AA?5?$AAm?$AA_?$AAn?$AAS?$AAi?$AAz?$AAe?$AA?$AA@ 00043e78     winmodemstat.obj
 0002:0000bef4       ??_C@_0P@GHFPNOJB@bad?5allocation?$AA@ 00043ef4     libcpmtd:stdthrow.obj
 0002:0000bf08       ??_7bad_alloc@std@@6B@     00043f08     libcpmtd:string.obj
 0002:0000bf14       ??_7logic_error@std@@6B@   00043f14     libcpmtd:string.obj
 0002:0000bf20       ??_7length_error@std@@6B@  00043f20     libcpmtd:string.obj
 0002:0000bf2c       ??_7out_of_range@std@@6B@  00043f2c     libcpmtd:string.obj
 0002:0000bf80       ??_C@_0BA@JFNIOLAK@string?5too?5long?$AA@ 00043f80     libcpmtd:string.obj
 0002:0000bfdc       ??_C@_0BI@CFPLBAOH@invalid?5string?5position?$AA@ 00043fdc     libcpmtd:string.obj
 0002:0000bff4       ??_C@_17LGKOMLJ@?$AA?4?$AA?4?$AA?4?$AA?$AA@ 00043ff4     LIBCMTD:dbgrpt.obj
 0002:0000bffc       ??_C@_1CC@CGHMNGDG@?$AAA?$AAs?$AAs?$AAe?$AAr?$AAt?$AAi?$AAo?$AAn?$AA?5?$AAF?$AAa?$AAi?$AAl?$AAe?$AAd?$AA?$AA@ 00043ffc     LIBCMTD:dbgrpt.obj
 0002:0000c020       ??_C@_1M@ILHOPKA@?$AAE?$AAr?$AAr?$AAo?$AAr?$AA?$AA@ 00044020     LIBCMTD:dbgrpt.obj
 0002:0000c02c       ??_C@_1BA@GLMCNLEM@?$AAW?$AAa?$AAr?$AAn?$AAi?$AAn?$AAg?$AA?$AA@ 0004402c     LIBCMTD:dbgrpt.obj
 0002:0000c040       ??_C@_1FC@DDJKODKC@?$AAf?$AA?3?$AA?2?$AAs?$AAp?$AA?2?$AAv?$AAc?$AAt?$AAo?$AAo?$AAl?$AAs?$AA?2?$AAc?$AAr?$AAt?$AAc?$AAe?$AA?2?$AAc?$AAr?$AAt?$AAw?$AA3?$AA2?$AA?2?$AAm?$AAi?$AAs?$AAc?$AA?2@ 00044040     LIBCMTD:dbgrpt.obj
 0002:0000c098       ??_C@_1EG@PEOEAKBB@?$AAM?$AAi?$AAc?$AAr?$AAo?$AAs?$AAo?$AAf?$AAt?$AA?5?$AAV?$AAi?$AAs?$AAu?$AAa?$AAl?$AA?5?$AAC?$AA?$CL?$AA?$CL?$AA?5?$AAD?$AAe?$AAb?$AAu?$AAg?$AA?5?$AAL?$AAi?$AAb?$AAr?$AAa@ 00044098     LIBCMTD:dbgrpt.obj
 0002:0000c0e0       ??_C@_1JI@EACPGHID@?$AAw?$AAc?$AAs?$AAc?$AAp?$AAy?$AA_?$AAs?$AA?$CI?$AAs?$AAz?$AAO?$AAu?$AAt?$AAM?$AAe?$AAs?$AAs?$AAa?$AAg?$AAe?$AA?0?$AA?5?$AA4?$AA0?$AA9?$AA6?$AA?0?$AA?5?$AAL?$AA?$CC?$AA_@ 000440e0     LIBCMTD:dbgrpt.obj
 0002:0000c178       ??_C@_1FG@BBOLDHGF@?$AA_?$AAC?$AAr?$AAt?$AAD?$AAb?$AAg?$AAR?$AAe?$AAp?$AAo?$AAr?$AAt?$AA?3?$AA?5?$AAS?$AAt?$AAr?$AAi?$AAn?$AAg?$AA?5?$AAt?$AAo?$AAo?$AA?5?$AAl?$AAo?$AAn?$AAg?$AA?5?$AAo@ 00044178     LIBCMTD:dbgrpt.obj
 0002:0000c1d0       ??_C@_1KG@MFHGLLO@?$AAD?$AAe?$AAb?$AAu?$AAg?$AA?5?$AA?$CF?$AAs?$AA?$CB?$AA?6?$AA?6?$AAP?$AAr?$AAo?$AAg?$AAr?$AAa?$AAm?$AA?3?$AA?5?$AA?$CF?$AAs?$AA?$CF?$AAs?$AA?$CF?$AAs?$AA?$CF?$AAs?$AA?$CF?$AAs?$AA?$CF?$AAs@ 000441d0     LIBCMTD:dbgrpt.obj
 0002:0000c278       ??_C@_1BE@CGCJKGHI@?$AA?6?$AAM?$AAo?$AAd?$AAu?$AAl?$AAe?$AA?3?$AA?5?$AA?$AA@ 00044278     LIBCMTD:dbgrpt.obj
 0002:0000c28c       ??_C@_1BA@LNHECFIM@?$AA?6?$AAF?$AAi?$AAl?$AAe?$AA?3?$AA?5?$AA?$AA@ 0004428c     LIBCMTD:dbgrpt.obj
 0002:0000c29c       ??_C@_1BA@GLLGCPCK@?$AA?6?$AAL?$AAi?$AAn?$AAe?$AA?3?$AA?5?$AA?$AA@ 0004429c     LIBCMTD:dbgrpt.obj
 0002:0000c2ac       ??_C@_13LBAGMAIH@?$AA?6?$AA?$AA@ 000442ac     LIBCMTD:dbgrpt.obj
 0002:0000c2b0       ??_C@_1BK@PEDCIPMA@?$AAE?$AAx?$AAp?$AAr?$AAe?$AAs?$AAs?$AAi?$AAo?$AAn?$AA?3?$AA?5?$AA?$AA@ 000442b0     LIBCMTD:dbgrpt.obj
 0002:0000c2cc       ??_C@_11LOCGONAA@?$AA?$AA@ 000442cc     LIBCMTD:dbgrpt.obj
 0002:0000c2d0       ??_C@_1JM@GKDPCMEA@?$AAw?$AAc?$AAs?$AAn?$AAc?$AAp?$AAy?$AA_?$AAs?$AA?$CI?$AAs?$AAz?$AAS?$AAh?$AAo?$AAr?$AAt?$AAP?$AAr?$AAo?$AAg?$AAN?$AAa?$AAm?$AAe?$AA?0?$AA?5?$AA2?$AA6?$AA0?$AA?5?$AA?9@ 000442d0     LIBCMTD:dbgrpt.obj
 0002:0000c370       ??_C@_1GI@DEDNNLCI@?$AAw?$AAc?$AAs?$AAc?$AAp?$AAy?$AA_?$AAs?$AA?$CI?$AAs?$AAz?$AAE?$AAx?$AAe?$AAN?$AAa?$AAm?$AAe?$AA?0?$AA?5?$AA2?$AA6?$AA0?$AA?0?$AA?5?$AAL?$AA?$CC?$AA?$DM?$AAp?$AAr?$AAo?$AAg@ 00044370     LIBCMTD:dbgrpt.obj
 0002:0000c3d8       ??_C@_1CI@PGJIFDEK@?$AA_?$AA_?$AAc?$AAr?$AAt?$AAM?$AAe?$AAs?$AAs?$AAa?$AAg?$AAe?$AAW?$AAi?$AAn?$AAd?$AAo?$AAw?$AAW?$AA?$AA@ 000443d8     LIBCMTD:dbgrpt.obj
 0002:0000c400       ??_C@_1CO@EAEJAADC@?$AA?$DM?$AAp?$AAr?$AAo?$AAg?$AAr?$AAa?$AAm?$AA?5?$AAn?$AAa?$AAm?$AAe?$AA?5?$AAu?$AAn?$AAk?$AAn?$AAo?$AAw?$AAn?$AA?$DO?$AA?$AA@ 00044400     LIBCMTD:dbgrpt.obj
 0002:0000c430       ??_C@_1CK@DDKKOLAN@?$AAs?$AAi?$AAz?$AAe?$AAI?$AAn?$AAB?$AAy?$AAt?$AAe?$AAs?$AA?5?$AA?$DO?$AA?$DN?$AA?5?$AAc?$AAo?$AAu?$AAn?$AAt?$AA?$AA@ 00044430     LIBCMTD:memcpy_s.obj
 0002:0000c45c       ??_C@_1BI@DCHLDCPP@?$AAs?$AAr?$AAc?$AA?5?$AA?$CB?$AA?$DN?$AA?5?$AAN?$AAU?$AAL?$AAL?$AA?$AA@ 0004445c     LIBCMTD:memcpy_s.obj
 0002:0000c474       ??_C@_1BC@GKHDJMGB@?$AAm?$AAe?$AAm?$AAc?$AAp?$AAy?$AA_?$AAs?$AA?$AA@ 00044474     LIBCMTD:memcpy_s.obj
 0002:0000c488       ??_C@_1FK@BOBCAACJ@?$AAf?$AA?3?$AA?2?$AAs?$AAp?$AA?2?$AAv?$AAc?$AAt?$AAo?$AAo?$AAl?$AAs?$AA?2?$AAc?$AAr?$AAt?$AAc?$AAe?$AA?2?$AAc?$AAr?$AAt?$AAw?$AA3?$AA2?$AA?2?$AAs?$AAt?$AAr?$AAi?$AAn@ 00044488     LIBCMTD:memcpy_s.obj
 0002:0000c4e4       ??_C@_1BI@GKKCBDMD@?$AAd?$AAs?$AAt?$AA?5?$AA?$CB?$AA?$DN?$AA?5?$AAN?$AAU?$AAL?$AAL?$AA?$AA@ 000444e4     LIBCMTD:memcpy_s.obj
 0002:0000c4fc       ??_C@_1BE@NMKKBGPA@?$AAm?$AAe?$AAm?$AAm?$AAo?$AAv?$AAe?$AA_?$AAs?$AA?$AA@ 000444fc     LIBCMTD:memmove_s.obj
 0002:0000c510       ??_C@_1FM@JMDLOEFB@?$AAf?$AA?3?$AA?2?$AAs?$AAp?$AA?2?$AAv?$AAc?$AAt?$AAo?$AAo?$AAl?$AAs?$AA?2?$AAc?$AAr?$AAt?$AAc?$AAe?$AA?2?$AAc?$AAr?$AAt?$AAw?$AA3?$AA2?$AA?2?$AAs?$AAt?$AAr?$AAi?$AAn@ 00044510     LIBCMTD:memmove_s.obj
 0002:0000c56c       ??_C@_0BJ@IPHDMCNM@fatal?5error?5in?5_lock?5?$CD0?6?$AA@ 0004456c     LIBCMTD:mlock.obj
 0002:0000c588       ??_C@_1FE@PLIBPAGC@?$AAf?$AA?3?$AA?2?$AAs?$AAp?$AA?2?$AAv?$AAc?$AAt?$AAo?$AAo?$AAl?$AAs?$AA?2?$AAc?$AAr?$AAt?$AAc?$AAe?$AA?2?$AAc?$AAr?$AAt?$AAw?$AA3?$AA2?$AA?2?$AAm?$AAi?$AAs?$AAc?$AA?2@ 00044588     LIBCMTD:dbgrptt.obj
 0002:0000c5e0       ??_C@_1MA@LBAMNNOB@?$AAs?$AAt?$AAr?$AAc?$AAp?$AAy?$AA_?$AAs?$AA?$CI?$AAs?$AAz?$AAO?$AAu?$AAt?$AAM?$AAe?$AAs?$AAs?$AAa?$AAg?$AAe?$AA2?$AA?0?$AA?5?$AA4?$AA0?$AA9?$AA6?$AA?0?$AA?5?$AA?$CC?$AA_@ 000445e0     LIBCMTD:dbgrptt.obj
 0002:0000c6a0       ??_C@_0DP@GNPEPHJD@_CrtDbgReport?3?5String?5too?5long?5o@ 000446a0     LIBCMTD:dbgrptt.obj
 0002:0000c6e0       ??_C@_1FI@DBAIJPJE@?$AAw?$AAc?$AAs?$AAc?$AAp?$AAy?$AA_?$AAs?$AA?$CI?$AAs?$AAz?$AAO?$AAu?$AAt?$AAM?$AAe?$AAs?$AAs?$AAa?$AAg?$AAe?$AA?0?$AA?5?$AA4?$AA0?$AA9?$AA6?$AA?0?$AA?5?$AAs?$AAz?$AAL@ 000446e0     LIBCMTD:dbgrptt.obj
 0002:0000c738       ??_C@_1BI@JIDBEPIG@?$AA?$CF?$AAs?$AA?$CI?$AA?$CF?$AAd?$AA?$CJ?$AA?5?$AA?3?$AA?5?$AA?$CF?$AAs?$AA?$AA@ 00044738     LIBCMTD:dbgrptt.obj
 0002:0000c750       ??_C@_1EK@PHCBEDKB@?$AAw?$AAc?$AAs?$AAc?$AAa?$AAt?$AA_?$AAs?$AA?$CI?$AAs?$AAz?$AAL?$AAi?$AAn?$AAe?$AAM?$AAe?$AAs?$AAs?$AAa?$AAg?$AAe?$AA?0?$AA?5?$AA4?$AA0?$AA9?$AA6?$AA?0?$AA?5?$AAL?$AA?$CC@ 00044750     LIBCMTD:dbgrptt.obj
 0002:0000c7a0       ??_C@_1EK@NMDFGHMF@?$AAw?$AAc?$AAs?$AAc?$AAa?$AAt?$AA_?$AAs?$AA?$CI?$AAs?$AAz?$AAL?$AAi?$AAn?$AAe?$AAM?$AAe?$AAs?$AAs?$AAa?$AAg?$AAe?$AA?0?$AA?5?$AA4?$AA0?$AA9?$AA6?$AA?0?$AA?5?$AAL?$AA?$CC@ 000447a0     LIBCMTD:dbgrptt.obj
 0002:0000c7ec       ??_C@_13CMNBPIDO@?$AA?$AN?$AA?$AA@ 000447ec     LIBCMTD:dbgrptt.obj
 0002:0000c7f0       ??_C@_1FK@HPADHBBD@?$AAw?$AAc?$AAs?$AAc?$AAa?$AAt?$AA_?$AAs?$AA?$CI?$AAs?$AAz?$AAL?$AAi?$AAn?$AAe?$AAM?$AAe?$AAs?$AAs?$AAa?$AAg?$AAe?$AA?0?$AA?5?$AA4?$AA0?$AA9?$AA6?$AA?0?$AA?5?$AAs?$AAz@ 000447f0     LIBCMTD:dbgrptt.obj
 0002:0000c850       ??_C@_1KO@DGAHENCH@?$AAw?$AAc?$AAs?$AAc?$AAp?$AAy?$AA_?$AAs?$AA?$CI?$AAs?$AAz?$AAL?$AAi?$AAn?$AAe?$AAM?$AAe?$AAs?$AAs?$AAa?$AAg?$AAe?$AA?0?$AA?5?$AA4?$AA0?$AA9?$AA6?$AA?0?$AA?5?$AAs?$AAz@ 00044850     LIBCMTD:dbgrptt.obj
 0002:0000c900       ??_C@_1CE@OJBNHDMO@?$AAA?$AAs?$AAs?$AAe?$AAr?$AAt?$AAi?$AAo?$AAn?$AA?5?$AAf?$AAa?$AAi?$AAl?$AAe?$AAd?$AA?$CB?$AA?$AA@ 00044900     LIBCMTD:dbgrptt.obj
 0002:0000c924       ??_C@_1CG@FFFGGODN@?$AAA?$AAs?$AAs?$AAe?$AAr?$AAt?$AAi?$AAo?$AAn?$AA?5?$AAf?$AAa?$AAi?$AAl?$AAe?$AAd?$AA?3?$AA?5?$AA?$AA@ 00044924     LIBCMTD:dbgrptt.obj
 0002:0000c950       ??_C@_1JK@KHFABAEO@?$AAw?$AAc?$AAs?$AAc?$AAp?$AAy?$AA_?$AAs?$AA?$CI?$AAs?$AAz?$AAU?$AAs?$AAe?$AAr?$AAM?$AAe?$AAs?$AAs?$AAa?$AAg?$AAe?$AA?0?$AA?5?$AA4?$AA0?$AA9?$AA6?$AA?0?$AA?5?$AAL?$AA?$CC@ 00044950     LIBCMTD:dbgrptt.obj
 0002:0000c9ec       ??_C@_1BA@ELMMDCFC@?$AA?0?$AA?5?$AAL?$AAi?$AAn?$AAe?$AA?5?$AA?$AA@ 000449ec     LIBCMTD:dbgrptt.obj
 0002:0000c9fc       ??_C@_1BO@OCHMLCAG@?$AA?$DM?$AAf?$AAi?$AAl?$AAe?$AA?5?$AAu?$AAn?$AAk?$AAn?$AAo?$AAw?$AAn?$AA?$DO?$AA?$AA@ 000449fc     LIBCMTD:dbgrptt.obj
 0002:0000ca20       ??_C@_1EM@MJFLEDMB@?$AAS?$AAe?$AAc?$AAo?$AAn?$AAd?$AA?5?$AAC?$AAh?$AAa?$AAn?$AAc?$AAe?$AA?5?$AAA?$AAs?$AAs?$AAe?$AAr?$AAt?$AAi?$AAo?$AAn?$AA?5?$AAF?$AAa?$AAi?$AAl?$AAe?$AAd?$AA?3?$AA?5@ 00044a20     LIBCMTD:dbgrptt.obj
 0002:0000ca70       ??_C@_1FA@CNLLOMHI@?$AA_?$AAi?$AAt?$AAo?$AAw?$AA_?$AAs?$AA?$CI?$AAn?$AAL?$AAi?$AAn?$AAe?$AA?0?$AA?5?$AAs?$AAz?$AAL?$AAi?$AAn?$AAe?$AAM?$AAe?$AAs?$AAs?$AAa?$AAg?$AAe?$AA?0?$AA?5?$AA4?$AA0@ 00044a70     LIBCMTD:dbgrptt.obj
 0002:0000cac0       ??_C@_1CA@HPALHDOD@?$AA_?$AAV?$AAC?$AAr?$AAt?$AAD?$AAb?$AAg?$AAR?$AAe?$AAp?$AAo?$AAr?$AAt?$AAW?$AA?$AA@ 00044ac0     LIBCMTD:dbgrptt.obj
 0002:0000cae0       ??_C@_1CG@MKBKDNCP@?$AAG?$AAe?$AAt?$AAL?$AAa?$AAs?$AAt?$AAA?$AAc?$AAt?$AAi?$AAv?$AAe?$AAP?$AAo?$AAp?$AAu?$AAp?$AA?$AA@ 00044ae0     LIBCMTD:crtmbox.obj
 0002:0000cb08       ??_C@_1CA@HNKPMKAN@?$AAG?$AAe?$AAt?$AAA?$AAc?$AAt?$AAi?$AAv?$AAe?$AAW?$AAi?$AAn?$AAd?$AAo?$AAw?$AA?$AA@ 00044b08     LIBCMTD:crtmbox.obj
 0002:0000cb28       ??_C@_1BI@OGPGOOGK@?$AAM?$AAe?$AAs?$AAs?$AAa?$AAg?$AAe?$AAB?$AAo?$AAx?$AAW?$AA?$AA@ 00044b28     LIBCMTD:crtmbox.obj
 0002:0000cb40       ??_C@_1BI@IENOMFML@?$AAC?$AAO?$AAR?$AAE?$AAD?$AAL?$AAL?$AA?4?$AAD?$AAL?$AAL?$AA?$AA@ 00044b40     LIBCMTD:crtmbox.obj
 0002:0000cb58       ??_C@_1DM@MADKGDLO@?$AA?$CI?$AAL?$AA?$CC?$AAB?$AAu?$AAf?$AAf?$AAe?$AAr?$AA?5?$AAi?$AAs?$AA?5?$AAt?$AAo?$AAo?$AA?5?$AAs?$AAm?$AAa?$AAl?$AAl?$AA?$CC?$AA?5?$AA?$CG?$AA?$CG?$AA?5?$AA0?$AA?$CJ?$AA?$AA@ 00044b58     LIBCMTD:wcsncpy_s.obj
 0002:0000cb94       ??_C@_1CI@HCPHDDLE@?$AAB?$AAu?$AAf?$AAf?$AAe?$AAr?$AA?5?$AAi?$AAs?$AA?5?$AAt?$AAo?$AAo?$AA?5?$AAs?$AAm?$AAa?$AAl?$AAl?$AA?$AA@ 00044b94     LIBCMTD:wcsncpy_s.obj
 0002:0000cbbc       ??_C@_1CG@OFBJMIGJ@?$AA?$CI?$AA?$CI?$AA?$CI?$AA_?$AAS?$AAr?$AAc?$AA?$CJ?$AA?$CJ?$AA?$CJ?$AA?5?$AA?$CB?$AA?$DN?$AA?5?$AAN?$AAU?$AAL?$AAL?$AA?$AA@ 00044bbc     LIBCMTD:wcsncpy_s.obj
 0002:0000cbe4       ??_C@_1BE@PMMBFFCC@?$AAw?$AAc?$AAs?$AAn?$AAc?$AAp?$AAy?$AA_?$AAs?$AA?$AA@ 00044be4     LIBCMTD:wcsncpy_s.obj
 0002:0000cbf8       ??_C@_1FG@OHHBDIEA@?$AAf?$AA?3?$AA?2?$AAs?$AAp?$AA?2?$AAv?$AAc?$AAt?$AAo?$AAo?$AAl?$AAs?$AA?2?$AAc?$AAr?$AAt?$AAc?$AAe?$AA?2?$AAc?$AAr?$AAt?$AAw?$AA3?$AA2?$AA?2?$AAh?$AA?2?$AAt?$AAc?$AAs@ 00044bf8     LIBCMTD:wcsncpy_s.obj
 0002:0000cc50       ??_C@_1FC@PFMLEHKI@?$AA?$CI?$AA?$CI?$AA_?$AAD?$AAs?$AAt?$AA?$CJ?$AA?$CJ?$AA?5?$AA?$CB?$AA?$DN?$AA?5?$AAN?$AAU?$AAL?$AAL?$AA?5?$AA?$CG?$AA?$CG?$AA?5?$AA?$CI?$AA?$CI?$AA_?$AAS?$AAi?$AAz?$AAe?$AAI?$AAn?$AAW?$AAo?$AAr@ 00044c50     LIBCMTD:wcsncpy_s.obj
 0002:0000cca4       ??_C@_1BC@KIONAFPO@?$AAw?$AAc?$AAs?$AAc?$AAp?$AAy?$AA_?$AAs?$AA?$AA@ 00044ca4     LIBCMTD:wcscpy_s.obj
 0002:0000ccb8       ??_C@_1FE@IPADLOPJ@?$AAf?$AA?3?$AA?2?$AAs?$AAp?$AA?2?$AAv?$AAc?$AAt?$AAo?$AAo?$AAl?$AAs?$AA?2?$AAc?$AAr?$AAt?$AAc?$AAe?$AA?2?$AAc?$AAr?$AAt?$AAw?$AA3?$AA2?$AA?2?$AAh?$AA?2?$AAt?$AAc?$AAs@ 00044cb8     LIBCMTD:wcscpy_s.obj
 0002:0000cd0c       ??_C@_1BC@CFJEPFGF@?$AAs?$AAt?$AAr?$AAc?$AAp?$AAy?$AA_?$AAs?$AA?$AA@ 00044d0c     LIBCMTD:strcpy_s.obj
 0002:0000cd20       ??_C@_1FC@NCPEPIBI@?$AA?$CI?$AA?$CI?$AA_?$AAD?$AAs?$AAt?$AA?$CJ?$AA?$CJ?$AA?5?$AA?$CB?$AA?$DN?$AA?5?$AAN?$AAU?$AAL?$AAL?$AA?5?$AA?$CG?$AA?$CG?$AA?5?$AA?$CI?$AA?$CI?$AA_?$AAS?$AAi?$AAz?$AAe?$AAI?$AAn?$AAB?$AAy?$AAt@ 00044d20     LIBCMTD:strcpy_s.obj
 0002:0000cd78       ??_C@_1FA@MJKDNFFB@?$AA?$CI?$AAL?$AA?$CC?$AAS?$AAt?$AAr?$AAi?$AAn?$AAg?$AA?5?$AAi?$AAs?$AA?5?$AAn?$AAo?$AAt?$AA?5?$AAn?$AAu?$AAl?$AAl?$AA?5?$AAt?$AAe?$AAr?$AAm?$AAi?$AAn?$AAa?$AAt?$AAe?$AAd@ 00044d78     LIBCMTD:wcscat_s.obj
 0002:0000cdc8       ??_C@_1DM@FHLMIEG@?$AAS?$AAt?$AAr?$AAi?$AAn?$AAg?$AA?5?$AAi?$AAs?$AA?5?$AAn?$AAo?$AAt?$AA?5?$AAn?$AAu?$AAl?$AAl?$AA?5?$AAt?$AAe?$AAr?$AAm?$AAi?$AAn?$AAa?$AAt?$AAe?$AAd?$AA?$AA@ 00044dc8     LIBCMTD:wcscat_s.obj
 0002:0000ce04       ??_C@_1BC@PLIEPKPJ@?$AAw?$AAc?$AAs?$AAc?$AAa?$AAt?$AA_?$AAs?$AA?$AA@ 00044e04     LIBCMTD:wcscat_s.obj
 0002:0000ce18       ??_C@_1FE@EHLIBGFJ@?$AAf?$AA?3?$AA?2?$AAs?$AAp?$AA?2?$AAv?$AAc?$AAt?$AAo?$AAo?$AAl?$AAs?$AA?2?$AAc?$AAr?$AAt?$AAc?$AAe?$AA?2?$AAc?$AAr?$AAt?$AAw?$AA3?$AA2?$AA?2?$AAh?$AA?2?$AAt?$AAc?$AAs@ 00044e18     LIBCMTD:wcscat_s.obj
 0002:0000ce6c       ??_C@_1CM@HABGDNLJ@?$AAl?$AAe?$AAn?$AAg?$AAt?$AAh?$AA?5?$AA?$DM?$AA?5?$AAs?$AAi?$AAz?$AAe?$AAI?$AAn?$AAT?$AAC?$AAh?$AAa?$AAr?$AAs?$AA?$AA@ 00044e6c     LIBCMTD:xtows.obj
 0002:0000ce98       ??_C@_1DE@PCJGDBBD@?$AA2?$AA?5?$AA?$DM?$AA?$DN?$AA?5?$AAr?$AAa?$AAd?$AAi?$AAx?$AA?5?$AA?$CG?$AA?$CG?$AA?5?$AAr?$AAa?$AAd?$AAi?$AAx?$AA?5?$AA?$DM?$AA?$DN?$AA?5?$AA3?$AA6?$AA?$AA@ 00044e98     LIBCMTD:xtows.obj
 0002:0000ced0       ??_C@_1FA@MKGGAGEI@?$AAs?$AAi?$AAz?$AAe?$AAI?$AAn?$AAT?$AAC?$AAh?$AAa?$AAr?$AAs?$AA?5?$AA?$DO?$AA?5?$AA?$CI?$AAs?$AAi?$AAz?$AAe?$AA_?$AAt?$AA?$CJ?$AA?$CI?$AAi?$AAs?$AA_?$AAn?$AAe?$AAg?$AA?5?$AA?$DP@ 00044ed0     LIBCMTD:xtows.obj
 0002:0000cf20       ??_C@_1CC@JNJFIMGE@?$AAs?$AAi?$AAz?$AAe?$AAI?$AAn?$AAT?$AAC?$AAh?$AAa?$AAr?$AAs?$AA?5?$AA?$DO?$AA?5?$AA0?$AA?$AA@ 00044f20     LIBCMTD:xtows.obj
 0002:0000cf44       ??_C@_1O@NCBFODOE@?$AAx?$AAt?$AAo?$AAw?$AA_?$AAs?$AA?$AA@ 00044f44     LIBCMTD:xtows.obj
 0002:0000cf58       ??_C@_1FE@LAGNOOBA@?$AAf?$AA?3?$AA?2?$AAs?$AAp?$AA?2?$AAv?$AAc?$AAt?$AAo?$AAo?$AAl?$AAs?$AA?2?$AAc?$AAr?$AAt?$AAc?$AAe?$AA?2?$AAc?$AAr?$AAt?$AAw?$AA3?$AA2?$AA?2?$AAc?$AAo?$AAn?$AAv?$AAe@ 00044f58     LIBCMTD:xtows.obj
 0002:0000cfac       ??_C@_1BI@ICGGMGLK@?$AAb?$AAu?$AAf?$AA?5?$AA?$CB?$AA?$DN?$AA?5?$AAN?$AAU?$AAL?$AAL?$AA?$AA@ 00044fac     LIBCMTD:xtows.obj
 0002:0000dfac       _GUID_b196b284_bab4_101a_b69c_00aa00341d07 00045fac     atlsd:atlfuncs.obj
 0002:0000dfbc       _GUID_00000000_0000_0000_c000_000000000046 00045fbc     atlsd:atlfuncs.obj
 0002:0000dfd0       ??_C@_1HA@FENMNPLO@?$AAf?$AA?3?$AA?2?$AAd?$AAd?$AA?2?$AAv?$AAc?$AAt?$AAo?$AAo?$AAl?$AAs?$AA?2?$AAv?$AAc?$AA7?$AAl?$AAi?$AAb?$AAs?$AAc?$AAe?$AA?2?$AAs?$AAh?$AAi?$AAp?$AA?2?$AAa?$AAt?$AAl@ 00045fd0     atlsd:atlfuncs.obj
 0002:0000e040       ??_C@_19LMDLLIGP@?$AAp?$AA?$DN?$AA?$DN?$AA0?$AA?$AA@ 00046040     atlsd:atlfuncs.obj
 0002:0000e04c       ??_C@_19JHCPJMAL@?$AAp?$AA?$CB?$AA?$DN?$AA0?$AA?$AA@ 0004604c     atlsd:atlfuncs.obj
 0002:0000e058       ??_C@_1HA@LPPEBACM@?$AAf?$AA?3?$AA?2?$AAd?$AAd?$AA?2?$AAv?$AAc?$AAt?$AAo?$AAo?$AAl?$AAs?$AA?2?$AAv?$AAc?$AA7?$AAl?$AAi?$AAb?$AAs?$AAc?$AAe?$AA?2?$AAs?$AAh?$AAi?$AAp?$AA?2?$AAa?$AAt?$AAl@ 00046058     atlsd:atlfuncs.obj
 0002:0000e0c8       ??_C@_1M@HLGKFCJM@?$AAf?$AAa?$AAl?$AAs?$AAe?$AA?$AA@ 000460c8     atlsd:atlfuncs.obj
 0002:0000e0d4       ??_C@_1CK@DFMKPFAK@?$AAA?$AAt?$AAl?$AAT?$AAh?$AAr?$AAo?$AAw?$AA?3?$AA?5?$AAh?$AAr?$AA?5?$AA?$DN?$AA?5?$AA0?$AAx?$AA?$CF?$AAx?$AA?6?$AA?$AA@ 000460d4     atlsd:atlfuncs.obj
 0002:0000e100       ??_C@_0DI@MHBOGIL@f?3?2dd?2vctools?2vc7libsce?2ship?2atl@ 00046100     atlsd:atlfuncs.obj
 0002:0000e138       ??_C@_1GM@IDLEHDFG@?$AAf?$AA?3?$AA?2?$AAd?$AAd?$AA?2?$AAv?$AAc?$AAt?$AAo?$AAo?$AAl?$AAs?$AA?2?$AAv?$AAc?$AA7?$AAl?$AAi?$AAb?$AAs?$AAc?$AAe?$AA?2?$AAs?$AAh?$AAi?$AAp?$AA?2?$AAa?$AAt?$AAl@ 00046138     atlsd:atlfuncs.obj
 0002:0000e1a4       ??_C@_1BE@NPGJNKLA@?$AAm?$AA_?$AAb?$AAL?$AAo?$AAc?$AAk?$AAe?$AAd?$AA?$AA@ 000461a4     atlsd:atlfuncs.obj
 0002:0000e1b8       ??_C@_1BG@OHCCAGNO@?$AA?$CB?$AAm?$AA_?$AAb?$AAL?$AAo?$AAc?$AAk?$AAe?$AAd?$AA?$AA@ 000461b8     atlsd:atlfuncs.obj
 0002:0000e1d0       ??_C@_1HE@LMFAHKHJ@?$AAf?$AA?3?$AA?2?$AAd?$AAd?$AA?2?$AAv?$AAc?$AAt?$AAo?$AAo?$AAl?$AAs?$AA?2?$AAv?$AAc?$AA7?$AAl?$AAi?$AAb?$AAs?$AAc?$AAe?$AA?2?$AAs?$AAh?$AAi?$AAp?$AA?2?$AAa?$AAt?$AAl@ 000461d0     atlsd:atlfuncs.obj
 0002:0000e3b8       GUID_ATLVer30              000463b8     atlsd:atlbase.obj
 0002:0000e3c8       GUID_ATLVer70              000463c8     atlsd:atlbase.obj
 0002:00011678       ??_C@_1JC@IHNNLNKC@?$AAf?$AA?3?$AA?2?$AAd?$AAd?$AA?2?$AAv?$AAc?$AAt?$AAo?$AAo?$AAl?$AAs?$AA?2?$AAv?$AAc?$AA7?$AAl?$AAi?$AAb?$AAs?$AAc?$AAe?$AA?2?$AAs?$AAh?$AAi?$AAp?$AA?2?$AAa?$AAt?$AAl@ 00049678     atlsd:Allocate.obj
 0002:0001170c       ??_C@_1BK@GFEAMNLJ@?$AAn?$AAC?$AAo?$AAo?$AAk?$AAi?$AAe?$AA?5?$AA?$CB?$AA?$DN?$AA?5?$AA0?$AA?$AA@ 0004970c     atlsd:Allocate.obj
 0002:00011b0c       IID_IPersistStream         00049b0c     uuid:objidl_i_guid12.obj
 0002:00011b1c       ??_R4bad_alloc@std@@6B@    00049b1c     libcpmtd:string.obj
 0002:00011b30       ??_R3bad_alloc@std@@8      00049b30     libcpmtd:string.obj
 0002:00011b40       ??_R2bad_alloc@std@@8      00049b40     libcpmtd:string.obj
 0002:00011b4c       ??_R1A@?0A@EA@bad_alloc@std@@8 00049b4c     libcpmtd:string.obj
 0002:00011b68       ??_R1A@?0A@EA@exception@std@@8 00049b68     libcpmtd:string.obj
 0002:00011b84       ??_R3exception@std@@8      00049b84     libcpmtd:string.obj
 0002:00011b94       ??_R2exception@std@@8      00049b94     libcpmtd:string.obj
 0002:00011b9c       ??_R4logic_error@std@@6B@  00049b9c     libcpmtd:string.obj
 0002:00011bb0       ??_R3logic_error@std@@8    00049bb0     libcpmtd:string.obj
 0002:00011bc0       ??_R2logic_error@std@@8    00049bc0     libcpmtd:string.obj
 0002:00011bcc       ??_R1A@?0A@EA@logic_error@std@@8 00049bcc     libcpmtd:string.obj
 0002:00011be8       ??_R4length_error@std@@6B@ 00049be8     libcpmtd:string.obj
 0002:00011bfc       ??_R3length_error@std@@8   00049bfc     libcpmtd:string.obj
 0002:00011c0c       ??_R2length_error@std@@8   00049c0c     libcpmtd:string.obj
 0002:00011c1c       ??_R1A@?0A@EA@length_error@std@@8 00049c1c     libcpmtd:string.obj
 0002:00011c38       ??_R4out_of_range@std@@6B@ 00049c38     libcpmtd:string.obj
 0002:00011c4c       ??_R3out_of_range@std@@8   00049c4c     libcpmtd:string.obj
 0002:00011c5c       ??_R2out_of_range@std@@8   00049c5c     libcpmtd:string.obj
 0002:00011c6c       ??_R1A@?0A@EA@out_of_range@std@@8 00049c6c     libcpmtd:string.obj
 0002:00011dbc       _TI3?AVlength_error@std@@  00049dbc     sessionmanager.obj
 0002:00011dcc       _CTA3?AVlength_error@std@@ 00049dcc     sessionmanager.obj
 0002:00011ddc       _CT??_R0?AVlength_error@std@@@8??0length_error@std@@QAA@ABV01@@Z44 00049ddc     sessionmanager.obj
 0002:00011df8       _CT??_R0?AVlogic_error@std@@@8??0logic_error@std@@QAA@ABV01@@Z44 00049df8     sessionmanager.obj
 0002:00011e14       _CT??_R0?AVexception@std@@@8??0exception@std@@QAA@ABV01@@Z12 00049e14     sessionmanager.obj
 0002:00011e30       _TI2?AVbad_alloc@std@@     00049e30     sessionmanager.obj
 0002:00011e40       _CTA2?AVbad_alloc@std@@    00049e40     sessionmanager.obj
 0002:00011e4c       _CT??_R0?AVbad_alloc@std@@@8??0bad_alloc@std@@QAA@ABV01@@Z12 00049e4c     sessionmanager.obj
 0002:00011e68       _TI3?AVout_of_range@std@@  00049e68     libcpmtd:string.obj
 0002:00011e78       _CTA3?AVout_of_range@std@@ 00049e78     libcpmtd:string.obj
 0002:00011e88       _CT??_R0?AVout_of_range@std@@@8??0out_of_range@std@@QAA@ABV01@@Z44 00049e88     libcpmtd:string.obj
 0002:00011ea4       _TI1?AVCAtlException@ATL@@ 00049ea4     atlsd:Externs.obj
 0002:00011eb4       _CTA1?AVCAtlException@ATL@@ 00049eb4     atlsd:Externs.obj
 0002:00011ebc       _CT??_R0?AVCAtlException@ATL@@@84 00049ebc     atlsd:Externs.obj
 0002:00011ed8       __IMPORT_DESCRIPTOR_sw_utilityG 00049ed8     sw_utilityG:sw_utilityG.dll
 0002:00011eec       __IMPORT_DESCRIPTOR_toolhelp 00049eec     toolhelp:toolhelp.dll
 0002:00011f00       __IMPORT_DESCRIPTOR_COREDLL 00049f00     coredll:COREDLL.dll
 0002:00011f14       __IMPORT_DESCRIPTOR_AYGSHELL 00049f14     aygshell:AYGSHELL.dll
 0002:00011f28       __IMPORT_DESCRIPTOR_ril    00049f28     ril:ril.dll
 0002:00011f3c       __IMPORT_DESCRIPTOR_ole32  00049f3c     ole32:ole32.dll
 0002:00011f50       __NULL_IMPORT_DESCRIPTOR   00049f50     sw_utilityG:sw_utilityG.dll
 0003:00000000       __imp_SHNotificationGetData 0004b000     aygshell:AYGSHELL.dll
 0003:00000004       __imp_SHNotificationUpdate 0004b004     aygshell:AYGSHELL.dll
 0003:00000008       __imp_SHNotificationRemove 0004b008     aygshell:AYGSHELL.dll
 0003:0000000c       __imp_SHNotificationAdd    0004b00c     aygshell:AYGSHELL.dll
 0003:00000010       __imp_SHCreateMenuBar      0004b010     aygshell:AYGSHELL.dll
 0003:00000014       __imp_SHInitDialog         0004b014     aygshell:AYGSHELL.dll
 0003:00000018       __imp_ExitWindowsEx        0004b018     aygshell:AYGSHELL.dll
 0003:0000001c       __imp_SHEnableSoftkey      0004b01c     aygshell:AYGSHELL.dll
 0003:00000020       \177AYGSHELL_NULL_THUNK_DATA 0004b020     aygshell:AYGSHELL.dll
 0003:00000024       __imp_UnmapViewOfFile      0004b024     coredll:COREDLL.dll
 0003:00000028       __imp_VirtualAlloc         0004b028     coredll:COREDLL.dll
 0003:0000002c       __imp_OpenEventW           0004b02c     coredll:COREDLL.dll
 0003:00000030       __imp_realloc              0004b030     coredll:COREDLL.dll
 0003:00000034       __imp_GetModuleHandleW     0004b034     coredll:COREDLL.dll
 0003:00000038       __imp_MsgWaitForMultipleObjectsEx 0004b038     coredll:COREDLL.dll
 0003:0000003c       __imp_PeekMessageW         0004b03c     coredll:COREDLL.dll
 0003:00000040       __imp_SetLastError         0004b040     coredll:COREDLL.dll
 0003:00000044       __imp_GetProcAddressW      0004b044     coredll:COREDLL.dll
 0003:00000048       __imp__vsnwprintf          0004b048     coredll:COREDLL.dll
 0003:0000004c       __imp_wcstombs             0004b04c     coredll:COREDLL.dll
 0003:00000050       __imp_WriteFile            0004b050     coredll:COREDLL.dll
 0003:00000054       __imp_TlsCall              0004b054     coredll:COREDLL.dll
 0003:00000058       __imp_InterlockedCompareExchange 0004b058     coredll:COREDLL.dll
 0003:0000005c       __imp_TlsGetValue          0004b05c     coredll:COREDLL.dll
 0003:00000060       __imp_TlsSetValue          0004b060     coredll:COREDLL.dll
 0003:00000064       __imp_GetModuleFileNameW   0004b064     coredll:COREDLL.dll
 0003:00000068       __imp__snwprintf           0004b068     coredll:COREDLL.dll
 0003:0000006c       __imp_malloc               0004b06c     coredll:COREDLL.dll
 0003:00000070       __imp_memmove              0004b070     coredll:COREDLL.dll
 0003:00000074       __imp_Sleep                0004b074     coredll:COREDLL.dll
 0003:00000078       __imp_FindClose            0004b078     coredll:COREDLL.dll
 0003:0000007c       __imp_FindFirstFileW       0004b07c     coredll:COREDLL.dll
 0003:00000080       __imp_DispatchMessageW     0004b080     coredll:COREDLL.dll
 0003:00000084       __imp_TranslateMessage     0004b084     coredll:COREDLL.dll
 0003:00000088       __imp_GetMessageW          0004b088     coredll:COREDLL.dll
 0003:0000008c       __imp_wcscpy               0004b08c     coredll:COREDLL.dll
 0003:00000090       __imp_GetLastError         0004b090     coredll:COREDLL.dll
 0003:00000094       __imp_CreateMutexW         0004b094     coredll:COREDLL.dll
 0003:00000098       __imp_WaitForSingleObject  0004b098     coredll:COREDLL.dll
 0003:0000009c       __imp_wcslen               0004b09c     coredll:COREDLL.dll
 0003:000000a0       __imp_LoadLibraryW         0004b0a0     coredll:COREDLL.dll
 0003:000000a4       __imp_??3@YAXPAX@Z         0004b0a4     coredll:COREDLL.dll
 0003:000000a8       __imp_CreateEventW         0004b0a8     coredll:COREDLL.dll
 0003:000000ac       __imp_InitializeCriticalSection 0004b0ac     coredll:COREDLL.dll
 0003:000000b0       __imp_??2@YAPAXI@Z         0004b0b0     coredll:COREDLL.dll
 0003:000000b4       __imp_CloseHandle          0004b0b4     coredll:COREDLL.dll
 0003:000000b8       __imp_CreateThread         0004b0b8     coredll:COREDLL.dll
 0003:000000bc       __imp_EventModify          0004b0bc     coredll:COREDLL.dll
 0003:000000c0       __imp_MessageBoxW          0004b0c0     coredll:COREDLL.dll
 0003:000000c4       __imp_LoadStringW          0004b0c4     coredll:COREDLL.dll
 0003:000000c8       __imp__wcsicmp             0004b0c8     coredll:COREDLL.dll
 0003:000000cc       __imp_wcsrchr              0004b0cc     coredll:COREDLL.dll
 0003:000000d0       __imp_SystemIdleTimerReset 0004b0d0     coredll:COREDLL.dll
 0003:000000d4       __imp_PostMessageW         0004b0d4     coredll:COREDLL.dll
 0003:000000d8       __imp_CreateProcessW       0004b0d8     coredll:COREDLL.dll
 0003:000000dc       __imp_DeleteCriticalSection 0004b0dc     coredll:COREDLL.dll
 0003:000000e0       __imp_OutputDebugStringW   0004b0e0     coredll:COREDLL.dll
 0003:000000e4       __imp_LeaveCriticalSection 0004b0e4     coredll:COREDLL.dll
 0003:000000e8       __imp_EnterCriticalSection 0004b0e8     coredll:COREDLL.dll
 0003:000000ec       __imp_NKDbgPrintfW         0004b0ec     coredll:COREDLL.dll
 0003:000000f0       __imp_RegisterWindowMessageW 0004b0f0     coredll:COREDLL.dll
 0003:000000f4       __imp_ShowWindow           0004b0f4     coredll:COREDLL.dll
 0003:000000f8       __imp_EnableWindow         0004b0f8     coredll:COREDLL.dll
 0003:000000fc       __imp_memcmp               0004b0fc     coredll:COREDLL.dll
 0003:00000100       __imp_SetWindowLongW       0004b100     coredll:COREDLL.dll
 0003:00000104       __imp_CreateDialogIndirectParamW 0004b104     coredll:COREDLL.dll
 0003:00000108       __imp_LoadResource         0004b108     coredll:COREDLL.dll
 0003:0000010c       __imp_FindResourceW        0004b10c     coredll:COREDLL.dll
 0003:00000110       __imp_DestroyWindow        0004b110     coredll:COREDLL.dll
 0003:00000114       __imp_GetWindowLongW       0004b114     coredll:COREDLL.dll
 0003:00000118       __imp_SetDlgItemTextW      0004b118     coredll:COREDLL.dll
 0003:0000011c       __imp_wsprintfW            0004b11c     coredll:COREDLL.dll
 0003:00000120       __imp_SetForegroundWindow  0004b120     coredll:COREDLL.dll
 0003:00000124       __imp_memset               0004b124     coredll:COREDLL.dll
 0003:00000128       __imp_DefWindowProcW       0004b128     coredll:COREDLL.dll
 0003:0000012c       __imp_KillTimer            0004b12c     coredll:COREDLL.dll
 0003:00000130       __imp_memcpy               0004b130     coredll:COREDLL.dll
 0003:00000134       __imp_LoadImageW           0004b134     coredll:COREDLL.dll
 0003:00000138       __imp_SetTimer             0004b138     coredll:COREDLL.dll
 0003:0000013c       __imp_RegCloseKey          0004b13c     coredll:COREDLL.dll
 0003:00000140       __imp_RegSetValueExW       0004b140     coredll:COREDLL.dll
 0003:00000144       __imp_wcscmp               0004b144     coredll:COREDLL.dll
 0003:00000148       __imp_wcsncpy              0004b148     coredll:COREDLL.dll
 0003:0000014c       __imp_RegQueryValueExW     0004b14c     coredll:COREDLL.dll
 0003:00000150       __imp_RegOpenKeyExW        0004b150     coredll:COREDLL.dll
 0003:00000154       __imp_RasEnumConnections   0004b154     coredll:COREDLL.dll
 0003:00000158       __imp_SetSystemTime        0004b158     coredll:COREDLL.dll
 0003:0000015c       __imp_RasSetEntryDialParams 0004b15c     coredll:COREDLL.dll
 0003:00000160       __imp_RasGetEntryProperties 0004b160     coredll:COREDLL.dll
 0003:00000164       __imp_RegisterClassW       0004b164     coredll:COREDLL.dll
 0003:00000168       __imp_GetStockObject       0004b168     coredll:COREDLL.dll
 0003:0000016c       __imp_LoadIconW            0004b16c     coredll:COREDLL.dll
 0003:00000170       __imp_LocalSize            0004b170     coredll:COREDLL.dll
 0003:00000174       __imp_SetWindowTextW       0004b174     coredll:COREDLL.dll
 0003:00000178       __imp_BringWindowToTop     0004b178     coredll:COREDLL.dll
 0003:0000017c       __imp___CxxThrowException  0004b17c     coredll:COREDLL.dll
 0003:00000180       __imp_??_7type_info@@6B@   0004b180     coredll:COREDLL.dll
 0003:00000184       __imp_??0exception@std@@QAA@ABV01@@Z 0004b184     coredll:COREDLL.dll
 0003:00000188       __imp_??1exception@std@@UAA@XZ 0004b188     coredll:COREDLL.dll
 0003:0000018c       __imp_??0exception@std@@QAA@XZ 0004b18c     coredll:COREDLL.dll
 0003:00000190       __imp___rt_udiv            0004b190     coredll:COREDLL.dll
 0003:00000194       __imp_strlen               0004b194     coredll:COREDLL.dll
 0003:00000198       __imp_??0exception@std@@QAA@PBD@Z 0004b198     coredll:COREDLL.dll
 0003:0000019c       __imp_?what@exception@std@@UBAPBDXZ 0004b19c     coredll:COREDLL.dll
 0003:000001a0       __imp_FindWindowW          0004b1a0     coredll:COREDLL.dll
 0003:000001a4       __imp_RasHangUp            0004b1a4     coredll:COREDLL.dll
 0003:000001a8       __imp_RasGetConnectStatus  0004b1a8     coredll:COREDLL.dll
 0003:000001ac       __imp_??_U@YAPAXI@Z        0004b1ac     coredll:COREDLL.dll
 0003:000001b0       __imp_GetDlgItemTextW      0004b1b0     coredll:COREDLL.dll
 0003:000001b4       __imp_wcscat               0004b1b4     coredll:COREDLL.dll
 0003:000001b8       __imp_TerminateProcess     0004b1b8     coredll:COREDLL.dll
 0003:000001bc       __imp_??_V@YAXPAX@Z        0004b1bc     coredll:COREDLL.dll
 0003:000001c0       __imp_swscanf              0004b1c0     coredll:COREDLL.dll
 0003:000001c4       __imp_SendMessageTimeout   0004b1c4     coredll:COREDLL.dll
 0003:000001c8       __imp_free                 0004b1c8     coredll:COREDLL.dll
 0003:000001cc       __imp_RaiseException       0004b1cc     coredll:COREDLL.dll
 0003:000001d0       __imp_GetSystemInfo        0004b1d0     coredll:COREDLL.dll
 0003:000001d4       __imp_MapViewOfFile        0004b1d4     coredll:COREDLL.dll
 0003:000001d8       __imp_CreateFileMappingW   0004b1d8     coredll:COREDLL.dll
 0003:000001dc       __imp_LocalAlloc           0004b1dc     coredll:COREDLL.dll
 0003:000001e0       __imp_LocalReAlloc         0004b1e0     coredll:COREDLL.dll
 0003:000001e4       __imp__XcptFilter          0004b1e4     coredll:COREDLL.dll
 0003:000001e8       __imp___C_specific_handler 0004b1e8     coredll:COREDLL.dll
 0003:000001ec       __imp_GetDlgItem           0004b1ec     coredll:COREDLL.dll
 0003:000001f0       __imp_CreateWindowExW      0004b1f0     coredll:COREDLL.dll
 0003:000001f4       __imp_?terminate@std@@YAXXZ 0004b1f4     coredll:COREDLL.dll
 0003:000001f8       __imp_strcmp               0004b1f8     coredll:COREDLL.dll
 0003:000001fc       __imp_InterlockedDecrement 0004b1fc     coredll:COREDLL.dll
 0003:00000200       __imp_InterlockedIncrement 0004b200     coredll:COREDLL.dll
 0003:00000204       __imp___security_gen_cookie 0004b204     coredll:COREDLL.dll
 0003:00000208       __imp_LocalFree            0004b208     coredll:COREDLL.dll
 0003:0000020c       __imp___report_gsfailure   0004b20c     coredll:COREDLL.dll
 0003:00000210       \177COREDLL_NULL_THUNK_DATA 0004b210     coredll:COREDLL.dll
 0003:00000214       __imp_WriteClassStm        0004b214     ole32:ole32.dll
 0003:00000218       __imp_CoCreateInstance     0004b218     ole32:ole32.dll
 0003:0000021c       __imp_ReadClassStm         0004b21c     ole32:ole32.dll
 0003:00000220       __imp_CreateStreamOnHGlobal 0004b220     ole32:ole32.dll
 0003:00000224       \177ole32_NULL_THUNK_DATA  0004b224     ole32:ole32.dll
 0003:00000228       __imp_RIL_Hangup           0004b228     ril:ril.dll
 0003:0000022c       __imp_RIL_SetEquipmentState 0004b22c     ril:ril.dll
 0003:00000230       __imp_RIL_GetSystemTime    0004b230     ril:ril.dll
 0003:00000234       __imp_RIL_DevSpecific      0004b234     ril:ril.dll
 0003:00000238       __imp_RIL_GetRegistrationStatus 0004b238     ril:ril.dll
 0003:0000023c       __imp_RIL_GetCallList      0004b23c     ril:ril.dll
 0003:00000240       __imp_RIL_GetEquipmentState 0004b240     ril:ril.dll
 0003:00000244       __imp_RIL_CancelSupServiceDataSession 0004b244     ril:ril.dll
 0003:00000248       __imp_RIL_SendSupServiceData 0004b248     ril:ril.dll
 0003:0000024c       __imp_RIL_GetSubscriberNumbers 0004b24c     ril:ril.dll
 0003:00000250       __imp_RIL_Deinitialize     0004b250     ril:ril.dll
 0003:00000254       __imp_RIL_Initialize       0004b254     ril:ril.dll
 0003:00000258       \177ril_NULL_THUNK_DATA    0004b258     ril:ril.dll
 0003:0000025c       __imp_?GetProductFeatures@@YAHAAK@Z 0004b25c     sw_utilityG:sw_utilityG.dll
 0003:00000260       __imp_?LogV@@YAXPBGZZ      0004b260     sw_utilityG:sw_utilityG.dll
 0003:00000264       __imp_?GetVerInfo@@YAPAGPAUHINSTANCE__@@@Z 0004b264     sw_utilityG:sw_utilityG.dll
 0003:00000268       __imp_?InitLog@@YAXPAUHINSTANCE__@@@Z 0004b268     sw_utilityG:sw_utilityG.dll
 0003:0000026c       __imp_?WriteLog@@YAXKPBGZZ 0004b26c     sw_utilityG:sw_utilityG.dll
 0003:00000270       __imp_GetVersionInfo       0004b270     sw_utilityG:sw_utilityG.dll
 0003:00000274       __imp_?GetRegValue@@YAJPAUHKEY__@@PBG1AAK@Z 0004b274     sw_utilityG:sw_utilityG.dll
 0003:00000278       __imp_?GetRegValue@@YAJPAUHKEY__@@PBG1PAGPAK@Z 0004b278     sw_utilityG:sw_utilityG.dll
 0003:0000027c       __imp_?SetRegValue@@YAJPAUHKEY__@@PBG11@Z 0004b27c     sw_utilityG:sw_utilityG.dll
 0003:00000280       __imp_?InWideMode@@YAHXZ   0004b280     sw_utilityG:sw_utilityG.dll
 0003:00000284       __imp_?RelayoutDialog@@YAHPAUHINSTANCE__@@PAUHWND__@@PBG@Z 0004b284     sw_utilityG:sw_utilityG.dll
 0003:00000288       __imp_?GetActWizDisabled@@YAKXZ 0004b288     sw_utilityG:sw_utilityG.dll
 0003:0000028c       __imp_?GetResolution@@YAHXZ 0004b28c     sw_utilityG:sw_utilityG.dll
 0003:00000290       __imp_?LogC@@YAXPBGZZ      0004b290     sw_utilityG:sw_utilityG.dll
 0003:00000294       __imp_?SWAI_GetRegValue@@YAJPAUHKEY__@@PBG1AAK@Z 0004b294     sw_utilityG:sw_utilityG.dll
 0003:00000298       __imp_?SetConnectionProfile@@YAJXZ 0004b298     sw_utilityG:sw_utilityG.dll
 0003:0000029c       __imp_?GetCarrierIndex@@YAKXZ 0004b29c     sw_utilityG:sw_utilityG.dll
 0003:000002a0       __imp_?GetAutoUpdateTimeUI@@YAKXZ 0004b2a0     sw_utilityG:sw_utilityG.dll
 0003:000002a4       __imp_?GetAutoUpdateTime@@YAKXZ 0004b2a4     sw_utilityG:sw_utilityG.dll
 0003:000002a8       __imp_?SetAutoUpdateTime@@YAXH@Z 0004b2a8     sw_utilityG:sw_utilityG.dll
 0003:000002ac       __imp_?SWAI_GetRegValue@@YAJPAUHKEY__@@PBG1PAEPAK@Z 0004b2ac     sw_utilityG:sw_utilityG.dll
 0003:000002b0       __imp_?LogStoreFileLine@@YAXPAGH@Z 0004b2b0     sw_utilityG:sw_utilityG.dll
 0003:000002b4       __imp_?LogW@@YAXPBGZZ      0004b2b4     sw_utilityG:sw_utilityG.dll
 0003:000002b8       \177sw_utilityG_NULL_THUNK_DATA 0004b2b8     sw_utilityG:sw_utilityG.dll
 0003:000002bc       __imp_Process32First       0004b2bc     toolhelp:toolhelp.dll
 0003:000002c0       __imp_CreateToolhelp32Snapshot 0004b2c0     toolhelp:toolhelp.dll
 0003:000002c4       __imp_CloseToolhelp32Snapshot 0004b2c4     toolhelp:toolhelp.dll
 0003:000002c8       __imp_Process32Next        0004b2c8     toolhelp:toolhelp.dll
 0003:000002cc       \177toolhelp_NULL_THUNK_DATA 0004b2cc     toolhelp:toolhelp.dll
 0003:000002d0       __xc_a                     0004b2d0     corelibc:crt0init.obj
 0003:000004a4       __xc_z                     0004b4a4     corelibc:crt0init.obj
 0003:000004a8       __xi_a                     0004b4a8     corelibc:crt0init.obj
 0003:000004ac       __xi_z                     0004b4ac     corelibc:crt0init.obj
 0003:000004b0       __xp_a                     0004b4b0     corelibc:crt0init.obj
 0003:000004b4       __xp_z                     0004b4b4     corelibc:crt0init.obj
 0003:000004b8       __xt_a                     0004b4b8     corelibc:crt0init.obj
 0003:000004bc       __xt_z                     0004b4bc     corelibc:crt0init.obj
 0003:000004d0       ?TRAY_NOTIFYICON@@3IA      0004b4d0     mainfrm.obj
 0003:0000050c       ?szAppName@CSession@@2PAPBGA 0004b50c     session.obj
 0003:00000520       ??_R0?AVlength_error@std@@@8 0004b520     sessionmanager.obj
 0003:00000540       ??_R0?AVlogic_error@std@@@8 0004b540     sessionmanager.obj
 0003:00000560       ??_R0?AVexception@std@@@8  0004b560     sessionmanager.obj
 0003:0000057c       ??_R0?AVbad_alloc@std@@@8  0004b57c     sessionmanager.obj
 0003:000005a4       ?m_SrvState@CModemStatus@@2KA 0004b5a4     winmodemstat.obj
 0003:000005a8       __security_cookie_complement 0004b5a8     corelibc:seccook.obj
 0003:000005ac       __security_cookie          0004b5ac     corelibc:seccook.obj
 0003:000005bc       ??_R0?AVout_of_range@std@@@8 0004b5bc     libcpmtd:string.obj
 0003:00000710       _crtAssertBusy             0004b710     LIBCMTD:dbgrptt.obj
 0003:00000714       _CrtDbgMode                0004b714     LIBCMTD:dbgrptt.obj
 0003:00000720       _CrtDbgFile                0004b720     LIBCMTD:dbgrptt.obj
 0003:0000072c       _aexit_rtn                 0004b72c     LIBCMTD:crt0dat.obj
 0003:00000730       _pRawDllMain               0004b730     atlsd:atlbase.obj
 0003:00000734       ?g_pszUpdateEventName@@3PB_WB 0004b734     atlsd:Externs.obj
 0003:00000738       ?g_pszAllocFileMapName@@3PB_WB 0004b738     atlsd:Externs.obj
 0003:0000073c       ?g_pszKernelObjFmt@@3PB_WB 0004b73c     atlsd:Externs.obj
 0003:00000740       ??_R0?AVCAtlException@ATL@@@8 0004b740     atlsd:Externs.obj
 0003:00000760       ?hInst@@3PAUHINSTANCE__@@A 0004b760     aam.obj
 0003:00000764       ?theApp@@3VCAAMApp@@A      0004b764     aam.obj
 0003:00000bc8       ?theMainWnd@@3VCMainFrame@@A 0004bbc8     aam.obj
 0003:000016f0       ?m_MsgBoxBuffer@CModemStatus@@1UtagMsgBoxContent@@A 0004c6f0     winmodemstat.obj
 0003:00001b04       ?m_NonDataCallStatus@CModemStatus@@2KA 0004cb04     winmodemstat.obj
 0003:00001b08       ?m_DataCallStatus@CModemStatus@@2KA 0004cb08     winmodemstat.obj
 0003:00001b0c       ?m_CallType@CModemStatus@@2KA 0004cb0c     winmodemstat.obj
 0003:00001b10       ?m_PwrState@CModemStatus@@2W4ePowerState@1@A 0004cb10     winmodemstat.obj
 0003:00001b14       ?m_RoamState@CModemStatus@@2KA 0004cb14     winmodemstat.obj
 0003:00001b18       ?m_IsOTASPCommited@CModemStatus@@2HA 0004cb18     winmodemstat.obj
 0003:00001b1c       ?m_LastCallEndStatus@CModemStatus@@2GA 0004cb1c     winmodemstat.obj
 0003:00001b20       ?m_hApi@CModemStatus@@1PAXA 0004cb20     winmodemstat.obj
 0003:00001b24       ?m_hActiveWindow@CModemStatus@@2PAUHWND__@@A 0004cb24     winmodemstat.obj
 0003:00001b28       ?m_MainWndH@CModemStatus@@1PAUHWND__@@A 0004cb28     winmodemstat.obj
 0003:00001b2c       ?m_hCurrModPowerState@CModemStatus@@2PAXA 0004cb2c     winmodemstat.obj
 0003:00001b30       ?m_hEquipmentStateOn@CModemStatus@@2PAXA 0004cb30     winmodemstat.obj
 0003:00001b34       ?m_bDMMode@CModemStatus@@1HA 0004cb34     winmodemstat.obj
 0003:00001b38       ?m_cFuncResultList@CModemStatus@@1V?$list@VCResultListElement@@V?$allocator@VCResultListElement@@@std@@@std@@A 0004cb38     winmodemstat.obj
 0003:00001b50       ?m_bInitFailed@CAtlBaseModule@ATL@@2_NA 0004cb50     winmodemstat.obj
 0003:00001cf8       ?_pAtlRawDllMain@@3P6AHPAXK0@ZA 0004ccf8     atlsd:atlbase.obj
 0003:00001cfc       ?_AtlModuleInstance@ATL@@3PAUHINSTANCE__@@A 0004ccfc     atlsd:atlbase.obj
 0003:00001d00       ?_AtlBaseModule@ATL@@3VCAtlBaseModule@1@A 0004cd00     atlsd:atlbase.obj
 0003:00001d84       ?atlTraceGeneral@ATL@@3VCTraceCategory@1@A 0004cd84     atlsd:atltrace.obj
 0003:00001d88       ?atlTraceCOM@ATL@@3VCTraceCategory@1@A 0004cd88     atlsd:atltrace.obj
 0003:00001d8c       ?atlTraceQI@ATL@@3VCTraceCategory@1@A 0004cd8c     atlsd:atltrace.obj
 0003:00001d90       ?atlTraceRegistrar@ATL@@3VCTraceCategory@1@A 0004cd90     atlsd:atltrace.obj
 0003:00001d94       ?atlTraceRefcount@ATL@@3VCTraceCategory@1@A 0004cd94     atlsd:atltrace.obj
 0003:00001d98       ?atlTraceWindowing@ATL@@3VCTraceCategory@1@A 0004cd98     atlsd:atltrace.obj
 0003:00001d9c       ?atlTraceControls@ATL@@3VCTraceCategory@1@A 0004cd9c     atlsd:atltrace.obj
 0003:00001da0       ?atlTraceHosting@ATL@@3VCTraceCategory@1@A 0004cda0     atlsd:atltrace.obj
 0003:00001da4       ?atlTraceNotImpl@ATL@@3VCTraceCategory@1@A 0004cda4     atlsd:atltrace.obj
 0003:00001da8       ?atlTraceAllocation@ATL@@3VCTraceCategory@1@A 0004cda8     atlsd:atltrace.obj
 0003:00001dac       ?atlTraceException@ATL@@3VCTraceCategory@1@A 0004cdac     atlsd:atltrace.obj
 0003:00001db0       ?atlTraceTime@ATL@@3VCTraceCategory@1@A 0004cdb0     atlsd:atltrace.obj
 0003:00001db4       ?atlTraceCache@ATL@@3VCTraceCategory@1@A 0004cdb4     atlsd:atltrace.obj
 0003:00001db8       ?atlTraceStencil@ATL@@3VCTraceCategory@1@A 0004cdb8     atlsd:atltrace.obj
 0003:00001dbc       ?atlTraceString@ATL@@3VCTraceCategory@1@A 0004cdbc     atlsd:atltrace.obj
 0003:00001dc0       ?atlTraceMap@ATL@@3VCTraceCategory@1@A 0004cdc0     atlsd:atltrace.obj
 0003:00001dc4       ?atlTraceUtil@ATL@@3VCTraceCategory@1@A 0004cdc4     atlsd:atltrace.obj
 0003:00001dc8       ?atlTraceSync@ATL@@3VCTraceCategory@1@A 0004cdc8     atlsd:atltrace.obj
 0003:00001dcc       ?atlTraceUser@ATL@@3VCTraceCategory@1@A 0004cdcc     atlsd:atltrace.obj
 0003:00001dd0       ?atlTraceUser2@ATL@@3VCTraceCategory@1@A 0004cdd0     atlsd:atltrace.obj
 0003:00001dd4       ?atlTraceUser3@ATL@@3VCTraceCategory@1@A 0004cdd4     atlsd:atltrace.obj
 0003:00001dd8       ?atlTraceUser4@ATL@@3VCTraceCategory@1@A 0004cdd8     atlsd:atltrace.obj
 0003:00001ddc       ?g_Allocator@@3VCAtlAllocator@@A 0004cddc     atlsd:Externs.obj
 0003:00001e10       ?s_trace@CTrace@ATL@@2V12@A 0004ce10     atlsd:Externs.obj
 0003:00001e18       __onexitend                0004ce18     <common>
 0003:00001e1c       __onexitbegin              0004ce1c     <common>
 0003:00001e20       _exitflag                  0004ce20     <common>
 0003:00001e24       _pfnReportHook             0004ce24     <common>
 0003:00001e28       _pReportHookListW          0004ce28     <common>
 0003:00001e2c       _pReportHookList           0004ce2c     <common>

 entry point at        0001:000152f8

 Static symbols

 0001:000001c8       __unwind$43713             000111c8 f   aam.obj
 0001:00000c50       __unwind$43900             00011c50 f i aam.obj
 0001:00000e8c       __unwind$46763             00011e8c f   arbitrator.obj
 0001:00000ea4       __unwind$46764             00011ea4 f   arbitrator.obj
 0001:00003030       __unwind$48067             00014030 f   mainfrm.obj
 0001:00003050       __unwind$48068             00014050 f   mainfrm.obj
 0001:00003070       __unwind$48069             00014070 f   mainfrm.obj
 0001:0000308c       __unwind$48070             0001408c f   mainfrm.obj
 0001:000030ac       __unwind$48071             000140ac f   mainfrm.obj
 0001:000030cc       __unwind$48072             000140cc f   mainfrm.obj
 0001:000030ec       __unwind$48073             000140ec f   mainfrm.obj
 0001:00003108       __unwind$48074             00014108 f   mainfrm.obj
 0001:00003128       __unwind$48075             00014128 f   mainfrm.obj
 0001:00003148       __unwind$48076             00014148 f   mainfrm.obj
 0001:00003168       __unwind$48077             00014168 f   mainfrm.obj
 0001:00003184       __unwind$48078             00014184 f   mainfrm.obj
 0001:000031a4       __unwind$48079             000141a4 f   mainfrm.obj
 0001:000031c4       __unwind$48080             000141c4 f   mainfrm.obj
 0001:000031e4       __unwind$48081             000141e4 f   mainfrm.obj
 0001:00003200       __unwind$48082             00014200 f   mainfrm.obj
 0001:00003220       __unwind$48083             00014220 f   mainfrm.obj
 0001:00003240       __unwind$48084             00014240 f   mainfrm.obj
 0001:000033b4       __unwind$48180             000143b4 f   mainfrm.obj
 0001:000033d4       __unwind$48181             000143d4 f   mainfrm.obj
 0001:000033f4       __unwind$48182             000143f4 f   mainfrm.obj
 0001:00003410       __unwind$48183             00014410 f   mainfrm.obj
 0001:00003430       __unwind$48184             00014430 f   mainfrm.obj
 0001:00003450       __unwind$48185             00014450 f   mainfrm.obj
 0001:00003470       __unwind$48186             00014470 f   mainfrm.obj
 0001:0000348c       __unwind$48187             0001448c f   mainfrm.obj
 0001:000034ac       __unwind$48188             000144ac f   mainfrm.obj
 0001:000034cc       __unwind$48189             000144cc f   mainfrm.obj
 0001:000034ec       __unwind$48190             000144ec f   mainfrm.obj
 0001:00003508       __unwind$48191             00014508 f   mainfrm.obj
 0001:00003528       __unwind$48192             00014528 f   mainfrm.obj
 0001:00003548       __unwind$48193             00014548 f   mainfrm.obj
 0001:00003568       __unwind$48194             00014568 f   mainfrm.obj
 0001:00003584       __unwind$48195             00014584 f   mainfrm.obj
 0001:000035a4       __unwind$48196             000145a4 f   mainfrm.obj
 0001:000035c4       __unwind$48197             000145c4 f   mainfrm.obj
 0001:00009d2c       __unwind$44020             0001ad2c f   sessionmanager.obj
 0001:00009d48       __unwind$44021             0001ad48 f   sessionmanager.obj
 0001:00009d60       __unwind$44022             0001ad60 f   sessionmanager.obj
 0001:00009d78       __unwind$44023             0001ad78 f   sessionmanager.obj
 0001:00009ef4       __unwind$44172             0001aef4 f   sessionmanager.obj
 0001:0000a15c       __unwind$44208             0001b15c f   sessionmanager.obj
 0001:0000a174       __unwind$44209             0001b174 f   sessionmanager.obj
 0001:0000a18c       __unwind$44210             0001b18c f   sessionmanager.obj
 0001:0000a38c       __unwind$44290             0001b38c f   sessionmanager.obj
 0001:0000a3a4       __unwind$44291             0001b3a4 f   sessionmanager.obj
 0001:0000a3bc       __unwind$44293             0001b3bc f   sessionmanager.obj
 0001:0000a9c4       __unwind$44095             0001b9c4 f i sessionmanager.obj
 0001:0000ab4c       __unwind$44131             0001bb4c f i sessionmanager.obj
 0001:0000ac04       __unwind$44150             0001bc04 f i sessionmanager.obj
 0001:0000ad9c       __unwind$44361             0001bd9c f i sessionmanager.obj
 0001:0000ade4       __unwind$44379             0001bde4 f i sessionmanager.obj
 0001:0000b0ac       __unwind$44430             0001c0ac f i sessionmanager.obj
 0001:0000b0c4       __unwind$44431             0001c0c4 f i sessionmanager.obj
 0001:0000b0dc       __unwind$44432             0001c0dc f i sessionmanager.obj
 0001:0000b420       __unwind$44556             0001c420 f i sessionmanager.obj
 0001:0000b4ec       __catch$44579              0001c4ec f i sessionmanager.obj
 0001:0000b810       __unwind$44662             0001c810 f i sessionmanager.obj
 0001:0000b828       __unwind$44663             0001c828 f i sessionmanager.obj
 0001:0000bd78       __catch$44782              0001cd78 f i sessionmanager.obj
 0001:0000beb4       __unwind$44809             0001ceb4 f i sessionmanager.obj
 0001:0000bf78       __unwind$44844             0001cf78 f i sessionmanager.obj
 0001:0000c128       __unwind$44909             0001d128 f i sessionmanager.obj
 0001:0000c17c       __unwind$44929             0001d17c f i sessionmanager.obj
 0001:0000c954       __unwind$45133             0001d954 f i sessionmanager.obj
 0001:0000cad0       __unwind$45178             0001dad0 f i sessionmanager.obj
 0001:0000cb5c       __unwind$45201             0001db5c f i sessionmanager.obj
 0001:0000cd8c       __catch$45232              0001dd8c f i sessionmanager.obj
 0001:0000cdc4       __catch$45230              0001ddc4 f i sessionmanager.obj
 0001:0000f724       __unwind$63602             00020724 f   winmodemstat.obj
 0001:0000f73c       __unwind$63603             0002073c f   winmodemstat.obj
 0001:0000fb48       __catch$63745              00020b48 f   winmodemstat.obj
 0001:0000fe60       __catch$63817              00020e60 f   winmodemstat.obj
 0001:0001003c       __catch$63851              0002103c f   winmodemstat.obj
 0001:00010938       __unwind$63894             00021938 f   winmodemstat.obj
 0001:00010958       __unwind$63895             00021958 f   winmodemstat.obj
 0001:00010978       __unwind$63896             00021978 f   winmodemstat.obj
 0001:00010998       __unwind$63898             00021998 f   winmodemstat.obj
 0001:0001142c       __catch$64158              0002242c f   winmodemstat.obj
 0001:000116c0       __catch$64188              000226c0 f   winmodemstat.obj
 0001:00012b70       __catch$64423              00023b70 f   winmodemstat.obj
 0001:00012d90       __catch$64454              00023d90 f   winmodemstat.obj
 0001:00012f40       __catch$64490              00023f40 f   winmodemstat.obj
 0001:00013518       __unwind$64545             00024518 f i winmodemstat.obj
 0001:00013530       __unwind$64547             00024530 f i winmodemstat.obj
 0001:00013714       __unwind$64573             00024714 f i winmodemstat.obj
 0001:0001372c       __unwind$64574             0002472c f i winmodemstat.obj
 0001:00013744       __unwind$64575             00024744 f i winmodemstat.obj
 0001:00013854       __unwind$64626             00024854 f i winmodemstat.obj
 0001:0001386c       __unwind$64627             0002486c f i winmodemstat.obj
 0001:00013a28       __unwind$64678             00024a28 f i winmodemstat.obj
 0001:00013ebc       __catch$64817              00024ebc f i winmodemstat.obj
 0001:00013ff8       __unwind$64844             00024ff8 f i winmodemstat.obj
 0001:000140dc       __unwind$65165             000250dc f i winmodemstat.obj
 0001:000146e4       __unwind$65694             000256e4 f i winmodemstat.obj
 0001:000147f0       __catch$65737              000257f0 f i winmodemstat.obj
 0001:00014a58       __unwind$65960             00025a58 f i winmodemstat.obj
 0001:000154fc       doexit                     000264fc f   corelibc:crt0dat.obj
 0001:000158d4       __unwind$18810             000268d4 f   libcpmtd:string.obj
 0001:00015964       __unwind$19010             00026964 f   libcpmtd:string.obj
 0001:00015d08       ?FindHandler@@YAEPAUEHExceptionRecord@@PAKPAU_CONTEXT@@PAU_DISPATCHER_CONTEXT@@PBU_s_FuncInfo@@H@Z 00026d08 f   LIBCMTD:frame_ce.obj
 0001:000162fc       ?TypeMatch@@YAHPBU_s_HandlerType@@PBU_s_CatchableType@@PBU_s_ThrowInfo@@@Z 000272fc f   LIBCMTD:frame_ce.obj
 0001:000166c0       ?FrameUnwindFilter@@YAHPAU_EXCEPTION_POINTERS@@@Z 000276c0 f   LIBCMTD:frame_ce.obj
 0001:0001674c       ?CallCatchBlock@@YAPAXPAUEHExceptionRecord@@PAKPAU_CONTEXT@@PBU_s_FuncInfo@@PAXHK@Z 0002774c f   LIBCMTD:frame_ce.obj
 0001:00016ce8       ?CanThisExceptionObjectBeDestructed@@YAEPAUEHExceptionRecord@@E@Z 00027ce8 f   LIBCMTD:frame_ce.obj
 0001:00016f74       ?BuildCatchObject@@YAXPAUEHExceptionRecord@@PAKPBU_s_HandlerType@@PBU_s_CatchableType@@@Z 00027f74 f   LIBCMTD:frame_ce.obj
 0001:000172c4       ?AdjustPointer@@YAPAXPAXABUPMD@@@Z 000282c4 f   LIBCMTD:frame_ce.obj
 0001:0001a634       __crtInitCritSecNoSpinCount 0002b634 f   LIBCMTD:initcrit.obj
 0001:0001b1cc       xtow_s                     0002c1cc f   LIBCMTD:xtows.obj
 0001:0001e074       ?_ATLLoadOle32API@ATL@@YAP6AHXZPB_W@Z 0002f074 f   atlsd:atlbase.obj
 0001:000200b8       ?Init@@YA_NXZ              000310b8 f   atlsd:Externs.obj
 0001:00022100       ?ShouldTraceOutput@ATL@@YA_NKKIPAPBVCAtlTraceCategory@@PAP6AHHPB_WH11ZZ@Z 00033100 f   atlsd:AtlDebugAPI.obj
 0001:000252b0       ??__EtheApp@@YAXXZ         000362b0 f   aam.obj
 0001:000252d0       ??__EtheMainWnd@@YAXXZ     000362d0 f   aam.obj
 0001:000252f0       ??__EIOTA_EXIT_MESSAGE@@YAXXZ 000362f0 f   arbitrator.obj
 0001:00025320       ??__EIOTA_BEGIN_MESSAGE@@YAXXZ 00036320 f   mainfrm.obj
 0001:00025350       ??__EIOTA_END_MESSAGE@@YAXXZ 00036350 f   mainfrm.obj
 0001:00025380       ??__EIOTA_BEGIN_ACK@@YAXXZ 00036380 f   mainfrm.obj
 0001:000253b0       ??__EIOTA_BEGIN_NACK@@YAXXZ 000363b0 f   mainfrm.obj
 0001:000253e0       ??__EIOTA_EXIT_MESSAGE@@YAXXZ 000363e0 f   mainfrm.obj
 0001:00025410       ??__EIOTA_DIAL@@YAXXZ      00036410 f   mainfrm.obj
 0001:00025440       ??__EIOTA_1012_MIP_ERR@@YAXXZ 00036440 f   mainfrm.obj
 0001:00025470       ??__EPHONEUTILS_BEGIN_MESSAGE@@YAXXZ 00036470 f   mainfrm.obj
 0001:000254a0       ??__EPHONEUTILS_END_MESSAGE@@YAXXZ 000364a0 f   mainfrm.obj
 0001:000254d0       ??__EPHONEUTILS_BEGIN_ACK@@YAXXZ 000364d0 f   mainfrm.obj
 0001:00025500       ??__EPHONEUTILS_BEGIN_NACK@@YAXXZ 00036500 f   mainfrm.obj
 0001:00025530       ??__EPHONEUTILS_EXIT_MESSAGE@@YAXXZ 00036530 f   mainfrm.obj
 0001:00025560       ??__EAW_BEGIN_MESSAGE@@YAXXZ 00036560 f   mainfrm.obj
 0001:00025590       ??__EAW_END_MESSAGE@@YAXXZ 00036590 f   mainfrm.obj
 0001:000255c0       ??__EAW_BEGIN_ACK@@YAXXZ   000365c0 f   mainfrm.obj
 0001:000255f0       ??__EAW_BEGIN_NACK@@YAXXZ  000365f0 f   mainfrm.obj
 0001:00025620       ??__EAW_EXIT_MESSAGE@@YAXXZ 00036620 f   mainfrm.obj
 0001:00025650       ??__EUPDATER_BEGIN@@YAXXZ  00036650 f   mainfrm.obj
 0001:00025680       ??__EUPDATER_END@@YAXXZ    00036680 f   mainfrm.obj
 0001:000256b0       ??__EUPDATER_BEGIN_ACK@@YAXXZ 000366b0 f   mainfrm.obj
 0001:000256e0       ??__EUPDATER_BEGIN_NACK@@YAXXZ 000366e0 f   mainfrm.obj
 0001:00025710       ??__EUPDATER_END_ACK@@YAXXZ 00036710 f   mainfrm.obj
 0001:00025740       ??__EUPDATER_END_NACK@@YAXXZ 00036740 f   mainfrm.obj
 0001:00025770       ??__EIOTA_BEGIN_NACK@@YAXXZ 00036770 f   sessionmanager.obj
 0001:000257a0       ??__EPHONEUTILS_EXIT_MESSAGE@@YAXXZ 000367a0 f   sessionmanager.obj
 0001:000257d0       ??__EPOWER_ON@@YAXXZ       000367d0 f   stdafx.obj
 0001:00025800       ??__EPOWER_OFF@@YAXXZ      00036800 f   stdafx.obj
 0001:00025830       ??__EIOTA_BEGIN_MESSAGE@@YAXXZ 00036830 f   stdafx.obj
 0001:00025860       ??__EIOTA_END_MESSAGE@@YAXXZ 00036860 f   stdafx.obj
 0001:00025890       ??__EIOTA_BEGIN_ACK@@YAXXZ 00036890 f   stdafx.obj
 0001:000258c0       ??__EIOTA_BEGIN_NACK@@YAXXZ 000368c0 f   stdafx.obj
 0001:000258f0       ??__EIOTA_END_ACK@@YAXXZ   000368f0 f   stdafx.obj
 0001:00025920       ??__EIOTA_EXIT_MESSAGE@@YAXXZ 00036920 f   stdafx.obj
 0001:00025950       ??__EIOTA_ALIVE_MESSAGE@@YAXXZ 00036950 f   stdafx.obj
 0001:00025980       ??__EIOTA_PING_MESSAGE@@YAXXZ 00036980 f   stdafx.obj
 0001:000259b0       ??__EIOTA_PING_ACK@@YAXXZ  000369b0 f   stdafx.obj
 0001:000259e0       ??__EIOTA_CRITICAL_ERROR@@YAXXZ 000369e0 f   stdafx.obj
 0001:00025a10       ??__EIOTA_NON_CRITICAL_ERROR@@YAXXZ 00036a10 f   stdafx.obj
 0001:00025a40       ??__EIOTA_KILL_ME@@YAXXZ   00036a40 f   stdafx.obj
 0001:00025a70       ??__EIOTA_UPDATE_STATUS@@YAXXZ 00036a70 f   stdafx.obj
 0001:00025aa0       ??__EIOTA_DATAPORT_INUSE@@YAXXZ 00036aa0 f   stdafx.obj
 0001:00025ad0       ??__EIOTA_DONE@@YAXXZ      00036ad0 f   stdafx.obj
 0001:00025b00       ??__EIOTA_DIAL@@YAXXZ      00036b00 f   stdafx.obj
 0001:00025b30       ??__EIOTA_1012_MIP_ERR@@YAXXZ 00036b30 f   stdafx.obj
 0001:00025b60       ??__EPHONEUTILS_BEGIN_MESSAGE@@YAXXZ 00036b60 f   stdafx.obj
 0001:00025b90       ??__EPHONEUTILS_END_MESSAGE@@YAXXZ 00036b90 f   stdafx.obj
 0001:00025bc0       ??__EPHONEUTILS_BEGIN_ACK@@YAXXZ 00036bc0 f   stdafx.obj
 0001:00025bf0       ??__EPHONEUTILS_BEGIN_NACK@@YAXXZ 00036bf0 f   stdafx.obj
 0001:00025c20       ??__EPHONEUTILS_END_ACK@@YAXXZ 00036c20 f   stdafx.obj
 0001:00025c50       ??__EPHONEUTILS_EXIT_MESSAGE@@YAXXZ 00036c50 f   stdafx.obj
 0001:00025c80       ??__EPHONEUTILS_ALIVE_MESSAGE@@YAXXZ 00036c80 f   stdafx.obj
 0001:00025cb0       ??__EPHONEUTILS_PING_MESSAGE@@YAXXZ 00036cb0 f   stdafx.obj
 0001:00025ce0       ??__EPHONEUTILS_PING_ACK@@YAXXZ 00036ce0 f   stdafx.obj
 0001:00025d10       ??__EAW_BEGIN_MESSAGE@@YAXXZ 00036d10 f   stdafx.obj
 0001:00025d40       ??__EAW_END_MESSAGE@@YAXXZ 00036d40 f   stdafx.obj
 0001:00025d70       ??__EAW_BEGIN_ACK@@YAXXZ   00036d70 f   stdafx.obj
 0001:00025da0       ??__EAW_BEGIN_NACK@@YAXXZ  00036da0 f   stdafx.obj
 0001:00025dd0       ??__EAW_END_ACK@@YAXXZ     00036dd0 f   stdafx.obj
 0001:00025e00       ??__EAW_EXIT_MESSAGE@@YAXXZ 00036e00 f   stdafx.obj
 0001:00025e30       ??__EAW_ALIVE_MESSAGE@@YAXXZ 00036e30 f   stdafx.obj
 0001:00025e60       ??__EAW_PING_MESSAGE@@YAXXZ 00036e60 f   stdafx.obj
 0001:00025e90       ??__EAW_PING_ACK@@YAXXZ    00036e90 f   stdafx.obj
 0001:00025ec0       ??__EUPDATER_BEGIN@@YAXXZ  00036ec0 f   stdafx.obj
 0001:00025ef0       ??__EUPDATER_END@@YAXXZ    00036ef0 f   stdafx.obj
 0001:00025f20       ??__EUPDATER_BEGIN_ACK@@YAXXZ 00036f20 f   stdafx.obj
 0001:00025f50       ??__EUPDATER_BEGIN_NACK@@YAXXZ 00036f50 f   stdafx.obj
 0001:00025f80       ??__EUPDATER_END_ACK@@YAXXZ 00036f80 f   stdafx.obj
 0001:00025fb0       ??__EUPDATER_END_NACK@@YAXXZ 00036fb0 f   stdafx.obj
 0001:00025fe0       ??__ERIL_STATUS_CHANGED@@YAXXZ 00036fe0 f   stdafx.obj
 0001:00026010       ??__ERIL_DBG_NOTIFY@@YAXXZ 00037010 f   stdafx.obj
 0001:00026040       ??__ERIL_TECHHDR_NOTIFY@@YAXXZ 00037040 f   stdafx.obj
 0001:00026070       ??__ERIL_IOTA_STATUS_CHANGED@@YAXXZ 00037070 f   stdafx.obj
 0001:000260a0       ??__ERIL_IOTA_WAP_URI@@YAXXZ 000370a0 f   stdafx.obj
 0001:000260d0       ??__ERIL_PDSM_PD_DATA@@YAXXZ 000370d0 f   stdafx.obj
 0001:00026100       ??__ERIL_PDSM_PD_DONE@@YAXXZ 00037100 f   stdafx.obj
 0001:00026130       ??__ERIL_PDSM_PD_END@@YAXXZ 00037130 f   stdafx.obj
 0001:00026160       ??__ERIL_PDSM_PD_BEGIN@@YAXXZ 00037160 f   stdafx.obj
 0001:00026190       ??__ERIL_PDSM_PD_UPDATE_FAILURE@@YAXXZ 00037190 f   stdafx.obj
 0001:000261c0       ??__ERIL_PDSM_PD_DLD_DATA@@YAXXZ 000371c0 f   stdafx.obj
 0001:000261f0       ??__ERIL_PDSM_PD_DLD_DONE@@YAXXZ 000371f0 f   stdafx.obj
 0001:00026220       ??__ERIL_PDSM_PD_DLD_END@@YAXXZ 00037220 f   stdafx.obj
 0001:00026250       ??__ERIL_PDSM_PD_DLD_BEGIN@@YAXXZ 00037250 f   stdafx.obj
 0001:00026280       ??__ERIL_PDSM_PA_PARAM@@YAXXZ 00037280 f   stdafx.obj
 0001:000262b0       ??__ERIL_CALL_BYTE_CTR@@YAXXZ 000372b0 f   stdafx.obj
 0001:000262e0       ??__E?m_cFuncResultList@CModemStatus@@1V?$list@VCResultListElement@@V?$allocator@VCResultListElement@@@std@@@std@@A@@YAXXZ 000372e0 f   winmodemstat.obj
 0001:00026300       ??__Einitlocks@std@@YAXXZ  00037300 f   libcpmtd:xlock.obj
 0001:0002633c       ??__E_AtlBaseModule@ATL@@YAXXZ 0003733c f   atlsd:atlbase.obj
 0001:00026378       ??__EatlTraceGeneral@ATL@@YAXXZ 00037378 f   atlsd:atltrace.obj
 0001:000263a8       ??__EatlTraceCOM@ATL@@YAXXZ 000373a8 f   atlsd:atltrace.obj
 0001:000263d8       ??__EatlTraceQI@ATL@@YAXXZ 000373d8 f   atlsd:atltrace.obj
 0001:00026408       ??__EatlTraceRegistrar@ATL@@YAXXZ 00037408 f   atlsd:atltrace.obj
 0001:00026438       ??__EatlTraceRefcount@ATL@@YAXXZ 00037438 f   atlsd:atltrace.obj
 0001:00026468       ??__EatlTraceWindowing@ATL@@YAXXZ 00037468 f   atlsd:atltrace.obj
 0001:00026498       ??__EatlTraceControls@ATL@@YAXXZ 00037498 f   atlsd:atltrace.obj
 0001:000264c8       ??__EatlTraceHosting@ATL@@YAXXZ 000374c8 f   atlsd:atltrace.obj
 0001:000264f8       ??__EatlTraceNotImpl@ATL@@YAXXZ 000374f8 f   atlsd:atltrace.obj
 0001:00026528       ??__EatlTraceAllocation@ATL@@YAXXZ 00037528 f   atlsd:atltrace.obj
 0001:00026558       ??__EatlTraceException@ATL@@YAXXZ 00037558 f   atlsd:atltrace.obj
 0001:00026588       ??__EatlTraceTime@ATL@@YAXXZ 00037588 f   atlsd:atltrace.obj
 0001:000265b8       ??__EatlTraceCache@ATL@@YAXXZ 000375b8 f   atlsd:atltrace.obj
 0001:000265e8       ??__EatlTraceStencil@ATL@@YAXXZ 000375e8 f   atlsd:atltrace.obj
 0001:00026618       ??__EatlTraceString@ATL@@YAXXZ 00037618 f   atlsd:atltrace.obj
 0001:00026648       ??__EatlTraceMap@ATL@@YAXXZ 00037648 f   atlsd:atltrace.obj
 0001:00026678       ??__EatlTraceUtil@ATL@@YAXXZ 00037678 f   atlsd:atltrace.obj
 0001:000266a8       ??__EatlTraceSync@ATL@@YAXXZ 000376a8 f   atlsd:atltrace.obj
 0001:000266d8       ??__EatlTraceUser@ATL@@YAXXZ 000376d8 f   atlsd:atltrace.obj
 0001:00026708       ??__EatlTraceUser2@ATL@@YAXXZ 00037708 f   atlsd:atltrace.obj
 0001:00026738       ??__EatlTraceUser3@ATL@@YAXXZ 00037738 f   atlsd:atltrace.obj
 0001:00026768       ??__EatlTraceUser4@ATL@@YAXXZ 00037768 f   atlsd:atltrace.obj
 0001:00026798       ??__Eg_Allocator@@YAXXZ    00037798 f   atlsd:Externs.obj
 0001:000267d4       ??__Eg_bInitialized@@YAXXZ 000377d4 f   atlsd:Externs.obj
 0001:0002680c       ??__E?s_trace@CTrace@ATL@@2V12@A@@YAXXZ 0003780c f   atlsd:Externs.obj
 0001:00026850       ??__FtheApp@@YAXXZ         00037850 f   aam.obj
 0001:00026864       ??__FtheMainWnd@@YAXXZ     00037864 f   aam.obj
 0001:00026878       ??__F?m_cFuncResultList@CModemStatus@@1V?$list@VCResultListElement@@V?$allocator@VCResultListElement@@@std@@@std@@A@@YAXXZ 00037878 f   winmodemstat.obj
 0001:0002688c       ??__Finitlocks@std@@YAXXZ  0003788c f   libcpmtd:xlock.obj
 0001:000268b0       ??__F_AtlBaseModule@ATL@@YAXXZ 000378b0 f   atlsd:atlbase.obj
 0001:000268d4       ??__Fg_Allocator@@YAXXZ    000378d4 f   atlsd:Externs.obj
 0001:000268f8       ??__F?s_trace@CTrace@ATL@@2V12@A@@YAXXZ 000378f8 f   atlsd:Externs.obj
